:020000040800F2
:100000000004022001020008910F0008950F00086B
:10001000E90F0008950F0008BD0F00080302000853
:100020000302000803020008030200082928000850
:10003000030200080302000803020008030200088C
:10004000030200080302000803020008030200087C
:100050000302000803020008393A0008653A000864
:10006000913A0008BD3A0008E93A00080302000886
:10007000030200080302000803020008030200084C
:10008000030200080302000803020008030200083C
:10009000030200080302000803020008153B0008E1
:1000A000030200080302000803020008030200081C
:1000B0005D3800080302000803020008030200087C
:1000C00003020008030200080302000803020008FC
:1000D00003020008030200088D1100080302000853
:1000E0007D3B000803020008030200080302000829
:1000F00003020008030200080302000803020008CC
:1001000003020008030200080302000803020008BB
:1001100003020008030200080302000803020008AB
:10012000030200080302000803020008030200089B
:10013000030200080302000803020008030200088B
:10014000030200080302000803020008952F0008BC
:10015000030200080302000803020008030200086B
:10016000030200080302000803020008030200085B
:10017000030200080302000803020008030200084B
:100180000302000803020008A1110008030200088E
:10019000030200080302000803020008030200082B
:1001A000030200080302000803020008030200081B
:1001B000030200080302000803020008030200080B
:1001C00003020008030200080302000803020008FB
:1001D00003020008030200080302000803020008EB
:1001E00003020008030200080302000803020008DB
:1001F00003020008030200080302000803020008CB
:1002000002E000F000F8FEE772B6394880F3088893
:10021000384880F3098838484EF60851CEF200017C
:10022000086040F20000CCF200004EF63471CEF2CD
:1002300000010860BFF34F8FBFF36F8F40F20000E3
:10024000C0F2F0004EF68851CEF200010860BFF314
:100250004F8FBFF36F8F4FF00000E1EE100A4EF6A4
:100260003C71CEF200010860062080F31488BFF3D1
:100270006F8F02F017FB03F079FA4FF055301F49EA
:100280001B4A91423CBF41F8040BFAE71C49194A4A
:1002900091423CBF41F8040BFAE71A491A4A1B4B3A
:1002A0009A423EBF51F8040B42F8040BF8E70020D5
:1002B0001749184A91423CBF41F8040BFAE702F093
:1002C00035FB03F0BDFA144C144DAC4203DA54F87C
:1002D000041B8847F9E700F03FF8114C114DAC4280
:1002E00003DA54F8041B8847F9E702F01DBB00004D
:1002F0000004022000240220000000080000022068
:1003000000040220E83F00080024022050240220BC
:100310005024022048390220000200080002000890
:1003200000020008000200082DE9F04F2DED108AB0
:10033000C1F80CD0D0F80CD0BDEC108ABDE8F08F1D
:10034000002383F311882846A047002001F0F6FE21
:1003500001F0A6FE00DFFEE770B532231F4C00253A
:100360006FF07F0623701F236570A570E5702571FF
:100370006571A571E57125726672A372E57200F070
:1003800029FD20B10F2325726672A372E57202F077
:100390000DFA044602F042FA0546D0B9104B9C42D1
:1003A00019D001339C4241F2883412BF0546002423
:1003B0000125002002F004FA0DB100F0B7F800F0BA
:1003C00087FD00F05DFC204600F050F900F0AEF82B
:1003D000F9E70024EDE70446EBE700BF50240220D4
:1003E000010007B008B500F0C9FBA0F12003584296
:1003F000584108BD054B07B51B88022101A8ADF87F
:10040000043000F027FC03B05DF804FB643C0008F6
:10041000064991F8243033B100230822086A81F894
:10042000243000F04FBC0120704700BF7024022030
:100430002DE9F84F234C05468846174694F824309A
:100440008BBB2E46DFF87C90002F38D094F824A088
:10045000BAF1000F05D12022FF214846266200F0A4
:1004600025FDCAF10805414604EB8A00BD4228BFBC
:100470003D465FFA85FBAD00A7EB0B072A462E44ED
:1004800000F0ECFC94F82430A844FFB29B445FFADF
:100490008BFBBBF1080F84F824B0D5D1FFF7B8FF70
:1004A0000028D1D108E0266A06EB8306B042C9D005
:1004B000FFF7AEFF0028C4D10020BDE8F88F01206F
:1004C000BDE8F88F7024022010B5202383F3118833
:1004D0001248C3680BB101F0B7FE0023104A4FF475
:1004E0007A710E4801F074FE002383F311880D4CDD
:1004F000236813B12368013B2360636813B1636809
:10050000013B6360084B1B7833B9636823B9022051
:1005100000F092FC3223636010BD00BF5C24022017
:10052000C9040008A025022098240220454B464912
:100530002DE9F04153F8042F013201D1BDE8F081DB
:100540008B42F7D1414C424B22689A4278D9414BB9
:100550009B6803F1006303F500439A4270D20020C8
:1005600000F0A8FB02203C4B187000F059FC3B4BFC
:100570001A6C00221A64196E1A66196E596C5A6444
:10058000596E5A66596E596941F08001596159692D
:1005900021F0800159615969196941F000511961CF
:1005A000196921F0005119611B6972B62C4B2D4954
:1005B0000B601D682468BFF34F8FBFF36F8F2A4B0A
:1005C000C3F88420BFF34F8F5A6922F480325A61F6
:1005D000BFF34F8FD3F8802043F6E07EC2F3C90605
:1005E000C2F34E32B707520102EA0E0838463146CE
:1005F000013948EA000C00F14040B1F1FF3FC3F877
:1006000074C2F5D1203A12F1200FEDD1BFF34F8F14
:10061000BFF36F8FBFF34F8FBFF36F8F5A6922F411
:1006200000325A610022C3F85022BFF34F8FBFF34C
:100630006F8F202383F31188AD4685F30888204708
:10064000BDE8F081FC7F00081C80000804800008E1
:10065000FF7F000850240220982402200038024026
:100660000080000808ED00E000ED00E02DE9F04F0B
:1006700099B0B34C2022FF21019010A8A66800F089
:1006800015FCB04AA3461378A3B90121AE481170F6
:10069000C360202383F31188C3680BB101F0D4FD3C
:1006A0000023AA4A4FF47A71A74801F091FD002374
:1006B00083F31188019B13B1A54B019A1A600023A3
:1006C000A44AA349019F99461C461D4698461370AB
:1006D0004B600292012000F0A3FB002F00F0128279
:1006E0009B4B1B68002B40F00D8219B0BDE8F08FCA
:1006F0000220FFF777FE002840F0FB81019BB9F153
:10070000000F08BF1F46944B1B8802210BA8ADF8B1
:100710002C3000F09FFADDE74FF47A7000F02EFAEB
:10072000031E0393EADB0220FFF75CFE82460028EB
:10073000E4D0039B581E042800F2DD81DFE800F0BE
:10074000030E1114170018A80523042140F8343DA6
:1007500000F080FA54464FF0000856E00421784833
:10076000F6E704217D48F3E704217D48F0E71C24E7
:100770002046043400F0A0FA04210B900BA800F0EE
:1007800069FA2C2CF4D1E5E7002DB7D0002CB5D0B8
:100790000220FFF727FE0546002800F0AF81012068
:1007A0006C4C00F087FA4FF000090220207000F036
:1007B00037FB5FFA89FA504600F08CFA074658B1C9
:1007C000504609F1010900F095FA0028F1D12C46B4
:1007D000A9460027634B97E701233E46022023707A
:1007E00000F010FBDBF808309E4206D2304600F0E5
:1007F00063FA0130EBD10436F4E70026029BA946E8
:100800002C461E703746524B5E6000F057FB15B108
:10081000002C18BF0027FFF7EDFD5BE7002D3FF42C
:100820006DAF002C3FF46AAF0220029B187000F0FD
:10083000F7FA322000F0A2F9B0F1000AC0F25E81AE
:100840001AF0030540F05A8106EB0A03DBF8082092
:10085000934200F25381BAF5807F00F24F815545F3
:100860000DDA4FF47A7000F089F90490049B002BA4
:10087000C0F24481049B3C4AAB540135EFE7C820E9
:10088000FFF7B0FD0546002800F038811F2E11D873
:10089000C6F1200410AB26F0030033495445184438
:1008A00028BF5446224600F0D9FA2246FF212E489E
:1008B00000F0FCFA4FEAAA0A2B4930465FFA8AF2A6
:1008C000FFF7B6FD0446002800F01A8106EB8A0601
:1008D00005469AE70220FFF785FD00283FF40EAF9A
:1008E000FFF796FD00283FF409AF4FF0000A53468A
:1008F000DBF8082092451CD2BAF11F0F12D8109ACB
:1009000001320FD02AF0030218A90A4452F8202C11
:100910000B92184604220BA90AF1040A00F078FB96
:100920000346E5E75046039300F0C6F9039B0B909E
:10093000EFE718A8042140F84C3D00F08BF964E77C
:10094000502402209C2502205C240220C9040008B7
:10095000A025022098240220663C0008542402208E
:1009600058240220683C00089C24022018A8002378
:10097000642140F8343D00F039F900287FF4BEAE20
:100980000220FFF72FFD00283FF4B8AE0B9800F0CF
:10099000C3F918AB43F8480D04211846CDE718A851
:1009A0000023642140F8343D00F020F900287FF452
:1009B000A5AE0220FFF716FD00283FF49FAE0B986E
:1009C00000F0B8F918AB43F8440DE5E70220FFF753
:1009D00009FD00283FF492AE00F0B2F918AB43F8DD
:1009E000400DD9E70220FFF7FDFC00283FF486AE5A
:1009F0000BA9142000F0AAF9824618A8042140F897
:100A00003CAD00F027F951460BA896E7322000F0E4
:100A1000B5F8B0F1000AFFF671AE1AF0030F7FF4DB
:100A20006DAE0AEB0803DBF8082093423FF666AE92
:100A30000220FFF7D7FC00283FF460AE2AF0030A3B
:100A4000C244D0453FF4E1AE404608F1040800F04E
:100A500033F904210A900AA800F0FCF8F1E74FF4FA
:100A60007A70FFF7BFFC00283FF448AEFFF7D0FCD8
:100A700000283FF4AFAE109B01330CD0082210A920
:100A80000020FFF7D5FC00283FF4A4AE2022FF2170
:100A900010A800F00BFAFFF7ADFC374801F054FB4B
:100AA00023E6002D3FF42AAE002C3FF427AE18A811
:100AB0000023642140F8343D00F098F88246002875
:100AC0007FF41CAE0220FFF78DFC00283FF416AE29
:100AD0000390FFF78FFC41F28830574601F034FB5A
:100AE0000B9800F035FA00F0E9F9039B1C461D460F
:100AF000F0E5054689E64FF00008FFE52546FDE5EF
:100B00002C4667E6002000F039F80490049B002B87
:100B1000FFF6E3AD012000F075F9049B213B122B99
:100B20003FF6D8AD01A252F823F000BFF10600084D
:100B30001907000889070008D5060008D50600082F
:100B4000D50600081D0800080D0A0008D508000891
:100B50006D0900089F090008CD090008D5060008A6
:100B6000E5090008D50600085F0A00080B08000820
:100B7000D5060008A30A0008A08601002DE9F34766
:100B80004FF47A75002402AE154F4543DFF85880C4
:100B900006F8014D97F900305FFA84F95A1C01D02C
:100BA000A34212D158F82400012231460368D3F839
:100BB00020A02B46D047012807D10A4B9DF80700FB
:100BC00083F8009002B0BDE8F0870134032CE1D136
:100BD0004FF4FA7001F0B8FA4FF0FF30F2E700BFBF
:100BE00000240220C4250220743C00082DE9F047AF
:100BF0004FF47A7506460024134F4D43DFF85080BA
:100C000097F900305FFA84F95A1C01D0A34210D141
:100C100058F82400042231460368D3F820A02B465C
:100C2000D047042805D1094B002083F80090BDE887
:100C3000F0870134032CE3D14FF4FA7001F084FA09
:100C40004FF0FF30BDE8F08700240220C4250220C9
:100C5000743C0008074B30B41A78074B53F8224015
:100C60000A46014623682046DD69044BAC4630BC89
:100C7000604700BFC4250220743C0008A086010024
:100C800070B50A4C00250A4E01F096FC20703068C1
:100C90002378834208D901F089FC33680544013385
:100CA000B5F5004F3360F2D370BD00BFC5250220FB
:100CB000A825022001F02CBD00F1006000F50040E5
:100CC0000068704700F10060920000F5004001F0FC
:100CD000B9BC0000054B1A68054B1B789B1A834270
:100CE00002D9104401F062BC00207047A825022000
:100CF000C525022038B5074D04462868204401F078
:100D00005DFC28B928682044BDE8384001F06EBC7D
:100D100038BD00BFA825022010F0030308D1B0F5AC
:100D2000806F05D800F10050A0F571200068704771
:100D300000207047014BC058704700BF20F4F01FDF
:100D4000014B1868704700BF002004E01F4BF0B54E
:100D50001E681F4BC6F30B02360C1F885D68BA4233
:100D600093F9084022D09F89BA4221D01F8BBA4202
:100D700006D102220C2404FB02335D6893F908407B
:100D8000B6F5805F16D041F201039E4208BF5A2497
:100D9000421E013D0B460A44934215D215F9016FDC
:100DA000581C4EB1034600F8016CF5E70022E1E75C
:100DB0000122DFE74124EBE72C2582421D7001D997
:100DC000981C5C70401AF0BD1846FBE7002004E058
:100DD00004240220094B5B88B3F5805F09D041F2FF
:100DE0000102934207D10122054B03EB8203D8781D
:100DF00070470022F8E70020704700BF002004E0A1
:100E00006C3C0008022804D14FF48002034B9A6125
:100E100070470128FCD14FF40002F7E700080240B8
:100E2000022803D14022034B9A6170470128FCD16C
:100E30008022F8E700080240022805D1064A5369DB
:100E400083F04003536170470128FCD1024A536983
:100E500083F08003F6E700BF00080240002310B5CE
:100E6000934203D0CC5CC4540133F9E710BD0000B9
:100E700030B5441E14F9010F0B4658B193F90050D8
:100E80000131854206D11AB993F90020801A30BD8C
:100E9000013AEFE7002AF7D1104630BD024603467B
:100EA000981A13F9011B0029FAD17047024403462E
:100EB000934202D003F8011BFAE77047024B1A78FD
:100EC000024B1A70704700BFC42502200024022084
:100ED00038B5184C184D204600F076FC29462046BF
:100EE00000F09EFC2D681548EA6ED2F8043843F0F5
:100EF0000203C2F8043801F027F91149284600F02E
:100F00009DFDEA6E0F48D2F804380F49A04223F045
:100F10000203C2F804384FF4E1330B6001D000F053
:100F2000B1FB0A48A04204D00749BDE8384000F0B0
:100F3000A9BB38BD602F0220683D000840420F0069
:100F4000903D000848260220AC250220B42602204D
:100F500038B50B4B05461A780A4B53F822400A4B1A
:100F60009C420CD0094B002118221846FFF79EFF27
:100F7000056001462046BDE8384000F083BB38BD1F
:100F8000C4250220743C0008602F0220AC250220FA
:100F9000FEE7000000B59BB0EFF3098168226846C8
:100FA000FFF75CFFEFF30583034B9A6B9A6A9A6A2B
:100FB0009A6A9A6A9B6AFEE700ED00E000B59BB072
:100FC000EFF3098168226846FFF748FFEFF30583D6
:100FD000044B9A6B9A6A9A6A9A6A9A6A9A6A9B6AA4
:100FE000FEE700BF00ED00E000B59BB0EFF3098124
:100FF00068226846FFF732FFEFF30583034B5A6B15
:101000009A6A9A6A9A6A9A6A9B6AFEE700ED00E019
:1010100030B50A44074D91420BD011F8013B092429
:101020005840013CF7D040F300032B4083EA5000C6
:10103000F7E730BD2083B8ED002304491A465A5023
:10104000C81808334260802BF9D17047C8250220A8
:10105000026843681143016003B1184770470000FC
:10106000024A136843F0C003136070470044004015
:10107000024A136843F0C0031360704700780040D1
:101080002DE9F047C66D05463768F46920073462DC
:101090001AD014F0080F0CBF00218021E20748BFCE
:1010A00041F02001A3074FF0200348BF41F0400169
:1010B000600748BF41F4807183F31188281DFFF752
:1010C000C7FF002383F31188E2050AD5202383F3A9
:1010D00011884FF40071281DFFF7BAFF002383F336
:1010E00011884FF020094FF0000A14F0200831D188
:1010F0003B0616D54FF0200905F1380A200610D519
:1011000089F31188504600F031FA00282FDA0821BF
:10111000281DFFF79DFF27F080033360002383F332
:10112000118879060DD562060BD5202383F311882B
:10113000EA6C2B6D9A4201D12B6CEBB9002383F33F
:101140001188E30620D5AA6E1369EBB15069BDE89A
:10115000F047184789F31188736A284695F8641098
:10116000194000F09DFA8AF31188F469BDE7B06276
:1011700088F31188F469C1E727F040071021281D82
:10118000FFF766FF3760D9E7BDE8F08708B5034889
:10119000FFF776FFBDE8084001F056BB4826022065
:1011A00008B50348FFF76CFFBDE8084001F04CBBF1
:1011B000B426022037B51F4C1F4D204600F056FACA
:1011C000009404F1140000234FF400721B4900F056
:1011D00017F94FF40072009404F13800184B1949C4
:1011E00000F090F9184B25660B21E3652620174C7B
:1011F00000F090F8204600F039FA04F11400009451
:1012000000234FF40072124900F0FAF804F138009C
:1012100000944FF400720F4B0F4900F073F90F4B1D
:101220000B215220E365256603B0BDE8304000F095
:1012300071B800BF4826022080F93703202702201A
:1012400061100008202B022000440040B426022038
:101250002029022071100008202D02200078004073
:10126000284B002908BF1946037C012B816630B545
:101270000CD1254B984235D1244B1A6C42F40032E4
:101280001A641A6E42F400321A661B6E0A68036E04
:10129000C46D03EB5203B3FBF2F34A68150442BF7B
:1012A00023F0070503F0070343EA4503E3608B6877
:1012B00043F040036360CB68510543F00103A36032
:1012C00042F4967343F0010323604FF0FF3323622F
:1012D00005D512F0102211D0B2F1805F10D080F845
:1012E000643030BD0A4B9842D0D1084B1A6C42F0A2
:1012F00080421A641A6E42F08042C5E77F23EEE70F
:101300003F23ECE7AC3C00084826022000380240AE
:10131000B426022000F1604300F01F0209014009D9
:1013200003F56143C9B2800083F80013012300F183
:101330006040934000F56140C0F880310360704721
:10134000F8B51546826804460B46AA4200D2856865
:10135000A1692669761AB54207D218462A46FFF7D0
:101360007DFDA3692B44A3610DE011D9AF1B32466B
:101370001846FFF773FD3A46E1683044FFF76EFD0B
:10138000E2683A44A261A36828465B1BA360F8BDEB
:1013900018462A46FFF762FDE368E4E78368934254
:1013A0002DE9F04104460F46154600D28568606974
:1013B0002669361AB54207D22A463946FFF74EFD4E
:1013C00063692B4463610EE013D9A5EB060832462E
:1013D0003946FFF743FD4246B919E068FFF73EFD85
:1013E000E26842446261A36828465B1BA360BDE8D3
:1013F000F0812A463946FFF731FDE368E2E7000055
:1014000010B50A440024C361029B00604060846000
:10141000C160816141610261036210BD08B58269EA
:101420004369934201D1826882B982680132826045
:101430005A1C42611970426903699A4201D3C36818
:101440004361002100F09CFE002008BD4FF0FF30FA
:1014500008BD000070B5202304460E4683F31188B2
:10146000A568A5B1A368A269013BA360531CA36151
:1014700015782269934224BFE368A361E3690BB145
:1014800020469847002383F31188284670BD3146D3
:10149000204600F065FE0028E2DA85F3118870BD71
:1014A0002DE9F74F05460F4690469A46D0F81C9016
:1014B000202686F311884FF0000B144664B12246B3
:1014C00039462846FFF73CFF034668B9514628468F
:1014D00000F046FE0028F1D0002383F31188A8EB2A
:1014E000040003B0BDE8F08FB9F1000F03D0019004
:1014F0002846C847019B8BF31188E41A1F4486F3E2
:101500001188DBE7C160816141611144C361009BC7
:10151000006040608260016103627047F8B5044674
:101520000E461746202383F31188A568A5B1A3684A
:10153000013BA36063695A1C62611E702369626982
:101540009A4224BFE3686361E3690BB12046984780
:10155000002080F31188F8BD3946204600F000FED7
:101560000028E2DA85F31188F8BD0000836942693A
:101570009A4210B501D182687AB9826801328260DC
:101580005A1C82611C7803699A4201D3C368836143
:10159000002100F0F5FD204610BD4FF0FF3010BDDA
:1015A0002DE9F74F05460F4690469A46D0F81C9015
:1015B000202686F311884FF0000B144664B12246B2
:1015C00039462846FFF7EAFE034668B951462846E1
:1015D00000F0C6FD0028F1D0002383F31188A8EBAA
:1015E000040003B0BDE8F08FB9F1000F03D0019003
:1015F0002846C847019B8BF31188E41A1F4486F3E1
:101600001188DBE7026843681143016003B11847A2
:10161000704700001430FFF743BF00004FF0FF3366
:101620001430FFF73DBF00003830FFF7B9BF0000AE
:101630004FF0FF333830FFF7B3BF00001430FFF72F
:1016400009BF00004FF0FF311430FFF703BF000067
:101650003830FFF763BF00004FF0FF323830FFF73C
:101660005DBF000000207047FFF7A4BD044B03607E
:10167000002343608360C36001230374704700BF8D
:10168000C43C000810B52023044683F31188FFF7FB
:10169000E7FD02232374002383F3118810BD0000AB
:1016A00038B5C36904460D461BB904210844FFF749
:1016B000A9FF294604F11400FFF7B0FE002806DA5E
:1016C000201D4FF48061BDE83840FFF79BBF38BD57
:1016D000026843681143016003B118477047000076
:1016E00013B5446BD4F894341A681178042915D1D1
:1016F000217C022912D11979012312898B401342CE
:101700000CD101A904F14C0001F0A6FED4F89444D8
:101710000246019B2179206800F0E0F902B010BD7B
:10172000143001F029BE00004FF0FF33143001F0F7
:1017300023BE00004C3001F0FBBE00004FF0FF3331
:101740004C3001F0F5BE0000143001F0F7BD000090
:101750004FF0FF31143001F0F1BD00004C3001F0CA
:10176000C7BE00004FF0FF324C3001F0C1BE000098
:10177000D0F8942438B5136805461978042901D0A7
:10178000012038BD017C0229FAD1127901205C893F
:1017900090400440F4D105F1140001F089FD0246A7
:1017A0000028EDD0D5F894544FF4807328686979F7
:1017B00000F082F9204638BD406BFFF7D9BF00002A
:1017C00000207047704700007FB5124B01250226AC
:1017D000044603600023057400F184024360294637
:1017E0008360C3600C4B0290143001934FF48073FC
:1017F000009601F039FD094B04F523722946019347
:1018000004F14C004FF480730294009601F000FE46
:1018100004B070BDEC3C0008B9170008E1160008E0
:101820000B68202282F311880A7903EB820210628E
:101830004A790D3243F822008A7912B103EB820310
:1018400018620223C0F894140374002383F31188F0
:101850007047000038B5037F044613B190F8543048
:10186000ABB90125201D0221FFF732FF04F114005E
:1018700025776FF0010100F08FFC84F8545004F1DB
:101880004C006FF00101BDE8384000F085BC38BD68
:1018900010B5012104460430FFF71AFF0023237717
:1018A00084F8543010BD000038B5044600251430CB
:1018B00001F0F2FC04F14C00257701F0C1FD201D80
:1018C00084F854500121FFF703FF2046BDE838405B
:1018D000FFF74EBF90F85C3003F06003202B19D166
:1018E00090F85D20212A0AD0222A4FF000030ED062
:1018F000202A0FD1084A02650722426504E0064B00
:101900000365072343650023836501207047036552
:101910004365F9E70020704728240220D0F894346A
:1019200037B51A680446117804291AD1017C0229B6
:1019300017D11979012312898B40134211D100F17B
:101940004C05284601F03CFE58B101A9284601F09B
:1019500083FDD4F894440246019B2179206800F06D
:10196000BDF803B030BD000000EB8103F7B51C6A81
:1019700005460E46F4B1202383F3118805EB860754
:10198000201D08214C34FFF7A3FEFB685B691B6830
:1019900013B1204601F06EFD01A9204601F05CFD67
:1019A000024648B1019B3146284600F097F80023D3
:1019B00083F3118803B0F0BDFB685A691268002AEE
:1019C000F5D01B8A013B1340F1D105F15C02EAE737
:1019D0000D3138B550F82140DCB1202383F3118854
:1019E000D4F894241368527903EB8203DB689B6973
:1019F0005D6845B104216018FFF76AFE294604F1CD
:101A0000140001F05FFC2046FFF7B2FE002383F3D1
:101A1000118838BD7047000001F00EB8012300F1B5
:101A2000240200F1380103700023436042F8043BB4
:101A30008A421361FAD103814381704738B5044665
:101A4000202383F3118800254160C560056145614D
:101A50008561C561056200F0FFFF0223237085F3F5
:101A6000118838BD70B500EB8103054650690E46FC
:101A70001446DA6018B110220021FFF717FAA069A6
:101A800018B110220021FFF711FA31462846BDE8AF
:101A9000704001F0ABB80000028902F0010202813F
:101AA000428902F0010242810022026142618261A8
:101AB000C261026201F02EB9F0B4012500EB81048D
:101AC00047898D40E4683D43A46945812360002334
:101AD000A2606360F0BC01F049B90000F0B40125D8
:101AE00000EB810407898D40E4683D43646905810A
:101AF00023600023A2606360F0BC01F0C3B9000062
:101B000070B50223002504460370A0F8645080F8E5
:101B1000665080F8675005814581C5600561456163
:101B20008561C561056280F84C5000F0FBFF636879
:101B30001B6823B129462046BDE87040184770BD98
:101B40000278436880F8682005221B6802700BB198
:101B50000421184770470000436890F868201B680C
:101B600002700BB1052118477047000090F84C3007
:101B700070B5044613B1002380F84C3004F15C02C8
:101B8000204601F0E9F863689B6863BB94F85C50F9
:101B900015F0600615D194F85D3005F07F0545EA33
:101BA000032540F202339D4200F00E815BD8022DE6
:101BB00000F0DC803FD8002D00F08780012D00F080
:101BC000CF800021204601F031FB0021204601F0AA
:101BD00023FB63681B6813B1062120469847062340
:101BE00084F84C3070BD204698470028CED094F839
:101BF000632094F8623043EA0223626D934238BF57
:101C0000636594F95C30656D002B4FF0200380F222
:101C1000FD80002D00F0EC80092284F84C2083F335
:101C200011880021636D226D2046FFF757FF0023C6
:101C300083F3118870BDB5F5817F00F0B180B5F5F3
:101C4000407F49D0B5F5807FBBD194F85E30012B41
:101C5000B7D1B4F8643023F00203A4F864302665E9
:101C60006665A665C3E740F201639D421ED8B5F5DF
:101C7000C06F3BD2B5F5A06FA3D1B4F85C30B3F51B
:101C8000A06F0ED194F85E30204684F8663000F0E4
:101C9000A1FF63681B6813B1012120469847032305
:101CA0002370002323656365A365A0E7B5F5106F76
:101CB00032D040F602439D4252D0B5F5006F80D13C
:101CC00004F167032365012324E004F16403A5659F
:101CD0002365022363658AE794F85E30012B7FF465
:101CE00070AFB4F8643043F00203B6E794F86120B3
:101CF0002046616894F860304D6843EA022394F806
:101D00005F1094F85E20A84700283FF45AAF43685C
:101D1000236503686365A4E72378042B10D120238F
:101D200083F311882046FFF7B7FE86F311886368B6
:101D3000032184F867601B6821700BB12046984727
:101D400094F85E30002BACD084F867300423237005
:101D500063681B68002BA4D0022120469847A0E7A7
:101D6000374B23650223636500239DE794F86010D9
:101D7000204611F0800F01F00F010ED000F0DEFFC1
:101D8000012806D002287FF41CAF2E4B6065236526
:101D900067E72D4B6565236563E700F0C1FFEFE75B
:101DA00094F85E30002B7FF40CAF94F8603013F0A1
:101DB0000F013FF476AF1A06204602D501F04AFA29
:101DC0006FE701F03DFA6CE794F85E30002B7FF48A
:101DD000F8AE94F8603013F00F013FF462AF1B06C9
:101DE000204602D501F022FA5BE701F015FA58E728
:101DF000142284F84C2083F311882B462A46294666
:101E00002046FFF759FE85F3118870BD5DB115229C
:101E100084F84C2083F311880021636D226D2046E5
:101E2000FFF74AFE03E70B2284F84C2083F3118866
:101E30002B462A4629462046FFF750FEE3E700BF1F
:101E40001C3D0008143D0008183D000838B590F806
:101E50004C300446152B29D8DFE803F03E2828280B
:101E600028283E28280B29392828282828282828E7
:101E70003E3E90F8631090F86220436D42EA0122E2
:101E80009A4214D9C268128AB3FBF2F502FB1535E7
:101E90006DB9202383F311882B462A462946FFF784
:101EA0001DFE85F311880A2384F84C3038BD1423B5
:101EB00084F84C30202383F31188002320461A46EF
:101EC0001946FFF7F9FD002383F3118838BD836DB0
:101ED00003B198470023E7E7002101F0A7F90021AB
:101EE000204601F099F963681B6813B1062120466A
:101EF00098470623D8E7000090F84C20152A38B5FB
:101F0000044622D80123934040F6416213421DD17A
:101F100013F480150FD19B0217D50B2380F84C309A
:101F2000202383F311882B462A462946FFF7D6FD46
:101F300085F3118838BDC3689B695B682BB9836DD5
:101F400003B19847002384F84C3038BD002101F0DC
:101F50006DF90021204601F05FF963681B6813B139
:101F60000621204698470623EDE70000024B002299
:101F70001B605B609A607047202F022000238268FC
:101F80000374054B1B6899689142FBD25A68036041
:101F90004260106058607047202F022008B520234F
:101FA00083F31188037C032B05D0042B0DD02BB9B0
:101FB00083F3118808BD436900221A604FF0FF3394
:101FC0004361FFF7DBFF0023F2E790E80C001A60A3
:101FD00002685360F2E70000002382680374054B37
:101FE0001B6899689142FBD85A6803604260106090
:101FF00058607047202F0220054B19690874186833
:10200000026853601A60186101230374FEF78CB9EB
:10201000202F02204B1C30B5054687B00A4C10D04B
:10202000236901A8094A00F0D3F82846FFF7E4FF26
:10203000049B13B101A800F007F92369586907B0A0
:1020400030BDFFF7D9FFF8E7202F02209D1F0008C1
:1020500038B50C4D044641612B6981689A689142FC
:1020600003D8BDE83840FFF789BF1846FFF786FF61
:1020700001232C61014623742046BDE83840FEF759
:1020800053B900BF202F0220044B1A681B699068C7
:102090009B68984294BF002001207047202F0220A7
:1020A00010B5084C236820691A6854602260012228
:1020B00023611A74FFF790FF01462069BDE81040C4
:1020C000FEF732B9202F0220826002220274002221
:1020D000427470478368A3F17C0243F80C2C0269B8
:1020E00043F83C2C426943F8382C074A43F81C2C2F
:1020F000C268A3F1180043F8102C022203F8082C40
:10210000002203F8072C70474103000810B5202374
:1021100083F31188FFF7DEFF00210446FFF798FFE5
:10212000002383F31188204610BD0000024B1B6979
:1021300058610F20FFF760BF202F0220202383F378
:102140001188FFF7F3BF000008B50146202383F391
:1021500011880820FFF75EFF002383F3118808BD74
:1021600049B1064B42681B6918605A6013604360AE
:102170000420FFF74FBF4FF0FF307047202F0220A1
:102180000368984206D01A68026050601846596188
:10219000FFF7F4BE7047000038B504460D462068CE
:1021A000844200D138BD036823605C604561FFF75D
:1021B000E5FEF4E7054B03F114025A619A614FF012
:1021C000FF32DA6100221A62704700BF202F02201E
:1021D000F8B503614FF08043C26002295C6A06468D
:1021E000184B38BF02211A461F4652F8145F954219
:1021F0000AD1586198611C620560456081600819C8
:10220000BDE8F84001F0FEB9186AAB68241A0C1951
:1022100002D3E41A2D6804E09C4202D2204401F06B
:10222000FFF9AB689C42F4D86B68356073601E6040
:102230004FF0FF336E60B460A968091BA960FB61B1
:10224000F8BD00BF202F022010B41B4C234653F8CA
:10225000141F814210D0416802680A600268516010
:102260009A424FF00001C16003D0936881680B442B
:1022700093605DF8044B70470A6800209A426261DF
:102280005360C86003D15DF8044B01F0C3B9936893
:1022900088680344206A93604FF08042526A121AA1
:1022A0009342E6D9991A5DF8044B012998BF931C13
:1022B000184401F0B5B900BF202F0220002070475C
:1022C000FEE70000704700004FF0FF30704700004D
:1022D000022906D0032906D00129064818BF00208C
:1022E000704705487047032A9ABF044800EBC200B4
:1022F00000207047EC3D0008A03D0008302402207B
:1023000070B59AB006460846144601AD294600F05D
:1023100095F82846FEF7C2FDC0B2431C5B0086E874
:10232000180023700323023404F8013C00231946EB
:10233000DAB20234904201D81AB070BDEA5C0133BF
:1023400004F8011C04F8022CF2E7000008B5202371
:1023500083F311880348FFF7E1FA002383F3118820
:1023600008BD00BF602F022010B50446052916D80D
:10237000DFE801F016150316161D202383F31188DC
:102380000E4A0121FFF76EFB20460D4A0221FFF79E
:1023900069FB0C48FFF788FA002383F3118810BD0E
:1023A000202383F311880748FFF754FAF4E720232A
:1023B00083F311880348FFF76BFAEDE7203D00082F
:1023C000443D0008602F022038B50C4D0C4C2A46C5
:1023D0000C4904F10800FFF793FF05F1CA0204F16C
:1023E00010000949FFF78CFF05F5CA7204F11800C7
:1023F0000649BDE83840FFF783BF00BF28340220FC
:1024000030240220703D00087A3D0008853D000818
:1024100070B5044608460D46FEF740FDC6B220469C
:10242000013403780BB9184670BD32462946FEF7D1
:102430001FFD0028F3D1012070BD00002DE9F84FE9
:1024400005460C46FEF72AFD2A49C6B22846FFF784
:10245000DFFF08B1013EF6B227492846FFF7D8FF53
:1024600008B11036F6B2632E0DD8DFF88890DFF889
:1024700088A0224FDFF88CB0DFF88C802E7846B928
:102480002670BDE8F88F29462046BDE8F84F01F0D8
:10249000E1BB252E2AD1072249462846FEF7E8FC53
:1024A00050B9D8F800300735063444F8063CB8F87F
:1024B000043024F8023CE1E7082251462846FEF7A2
:1024C000D7FC98B9A21C0E4B13F8011F0232090960
:1024D0005B45C95D02F8041C197801F00F01C95D64
:1024E00002F8031CF0D118340835C7E7267001350F
:1024F0000134C3E70C3E0008853D00081B3E000880
:102500001FF4F01F2BF4F01F143E0008BFF34F8F91
:10251000024AD368DB03FCD4704700BF003C024092
:1025200008B5074B1B7853B9FFF7F0FF054B1A6945
:10253000002A04DA044A5A6002F188325A6008BD5F
:1025400086360220003C02402301674508B5054B52
:102550001B7833B9FFF7DAFF034A136943F00043EE
:10256000136108BD86360220003C02400B2870B57E
:1025700013D80B4A0B4C137863B94FF000610A4E25
:1025800044F8231056F8235001330C2B2944F7D17B
:102590000123137054F8200070BD002070BD00BFEF
:1025A000B8360220883602202C3E0008014B53F832
:1025B000200070472C3E00080C2070470B2810B5F7
:1025C000044601D9002010BDFFF7D0FF064B53F899
:1025D00024301844C21A0BB9012010BD1268013210
:1025E000F0D1043BF6E700BF2C3E00080B2810B5E5
:1025F000044621D8FFF78AFFFFF792FF0F4AF32323
:10260000D360C300DBB243F4007343F002031361F1
:10261000136943F480331361FFF778FFFFF7A6FFD8
:10262000074B53F8241000F0DBF8FFF78FFF20462C
:10263000BDE81040FFF7C2BF002010BD003C0240C3
:102640002C3E00082DE9F84312F0010315463FD156
:102650008218B2F1026F3BD22B4B1B6813F00103BF
:1026600036D0FFF75DFF294CF32340F20127E360EA
:10267000FFF74CFF032D01D9830712D00F46401AF4
:10268000224C40F20118EB1BC6190B44012B2369A5
:1026900024D823F001032361FFF758FF0120BDE890
:1026A000F883236923F44073236123693B43236147
:1026B00051F8046B0660BFF34F8FFFF727FF0368E5
:1026C0009E4208D0236923F001032361FFF73EFFF8
:1026D0000020BDE8F883043D0430CBE723F44073C9
:1026E000B9462361236943EA0803236137F8023BB3
:1026F0003380BFF34F8FFFF709FF3688B6B2B9F8C2
:102700000030B342BFD0DDE700380240003C024059
:10271000084908B50B7828B153B9FFF701FF012329
:102720000B7008BD23B10870BDE80840FFF70EBF6D
:1027300008BD00BF8636022002440439064BD2B2DF
:1027400010B5904200D110BD441C00B253F82000D7
:1027500041F8040FE0B2F4E750280040104B30B5C8
:102760001C6F240407D41C6F44F400741C671C6F96
:1027700044F400441C670B4C024404392368D2B271
:1027800043F480732360084B904200D130BD441C59
:1027900051F8045F00B243F82050E0B2F4E700BF04
:1027A00000380240007000405028004007B5012268
:1027B00001A90020FFF7C0FF019803B05DF804FBFA
:1027C00013B50446FFF7F2FFA04206D002A901228A
:1027D000002041F8044DFFF7C1FF02B010BD00001A
:1027E0000144BFF34F8F064B884204D3BFF34F8F92
:1027F000BFF36F8F7047C3F85C022030F4E700BF6F
:1028000000ED00E0034B1B689B0042BF0122024B1E
:102810001A70704774380240B9360220014B18789C
:10282000704700BFB9360220064A536823F00103FF
:102830005360EFF30983683383F30988002383F33C
:102840001188704730EF00E010B5202383F3118822
:10285000104B5B6813F4006318D0F1EE103AEFF3FD
:1028600009844FF0807344F84C3C0B4BDB6844F810
:10287000083CA4F1680383F30988FFF705FC18B14D
:10288000064B44F8503C10BD054BFAE783F3118822
:1028900010BD00BF00ED00E030EF00E05103000884
:1028A00054030008F0B5BFF34F8FBFF36F8F1D4B7C
:1028B0000021C3F85012BFF34F8FBFF36F8F5A69D7
:1028C00042F400325A61BFF34F8FBFF36F8FC3F8EA
:1028D0008410BFF34F8FD3F8802043F6E076C2F325
:1028E000C904C2F34E32A507520102EA060E284679
:1028F00021464EEA0007013900F14040C3F86072FA
:102900004F1CF6D1203A12F1200FEED1BFF34F8FBA
:102910005A6942F480325A61BFF34F8FBFF36F8F11
:10292000F0BD00BF00ED00E0FEE70000084A094BE3
:1029300009498B4204D3094A0021934205D37047C9
:1029400052F8040F43F8040BF3E743F8041BF4E7D1
:102950003440000848390220483902204839022012
:10296000036F002230B51146C46E9D684FF0FF30F2
:1029700004EB421301329542C3F80019C3F8101951
:10298000C3F80809C3F8001BC3F8101BC3F8080BF1
:10299000EED24FF00113C4F81C3830BD890141F06C
:1029A0002001016103699B06FCD4122000F0C4BE23
:1029B000204B03EB80022DE9F047D2F80CE0461CD7
:1029C000DD6EDEF8142005EB0636D2F800C005EB0C
:1029D0004018516861450BD30123D5F8342803FA18
:1029E00000F022EA0000C5F834081846BDE8F08778
:1029F000ACEB0103BEF81040A34228BF2346D8F831
:102A00001849A4B2B3EB840F10D894681F46A4F100
:102A1000040959F804AF042FC6F800A001D9043FF7
:102A2000F7E71C440B4494605360D2E70020BDE8F4
:102A3000F08700BFBC36022010B5054C2046FEF7DB
:102A4000EDFF4FF0A043E366024B236710BD00BFCC
:102A5000BC360220803E00080378012B70B5054685
:102A600050D12A4BC46E98421BD1294B0E214320D2
:102A70005A6B42F080025A635A6D42F080025A65E6
:102A80005A6D5A6942F080025A615A6922F08002F6
:102A90005A615B69FEF73EFC1E4BE3601E4BC4F8B7
:102AA00000380023EE6EC4F8003EC02323604FF4CC
:102AB0000413A3633369002BFCDA01230C20336178
:102AC00000F03AFE3369DB07FCD4122000F034FE3C
:102AD0003369002BFCDA00262846A660FFF740FF8A
:102AE0006B68C4F81068DB68C4F81468C4F81C6824
:102AF0004BB90A4BA3614FF0FF336361A36843F006
:102B00000103A36070BD064BF4E700BFBC36022092
:102B1000003802404014004003002002003C30C056
:102B2000083C30C0F8B5C46E054600214FF0006681
:102B30002046FFF733FF296F00234FF001128F6803
:102B40004FF0FF30C4F83438C4F81C2804EB4312AB
:102B500001339F42C2F80069C2F8006BC2F808094D
:102B6000C2F8080BF2D20B68EA6E6B67636210233F
:102B70001361166916F01006FBD1122000F0DCFD7F
:102B8000D4F8003823F4FE63C4F80038A36943F492
:102B9000402343F01003A3610923C4F81038C4F89C
:102BA00014380A4BEB604FF0C043C4F8103B084B9D
:102BB000C4F8003BC4F81069C4F800396B6F03F126
:102BC000100243F480136A67A362F8BD5C3E0008FC
:102BD00040800010C26E90F86610D2F8003823F4DE
:102BE000FE6343EA0113C2F8003870472DE9F04153
:102BF0000EB20D4600EB8608D8F80C100F6807F0EF
:102C00000303022B50D0032B50D03D4A3D4F012BE4
:102C100018BF1746C46E4FEA451E002205F1100C7E
:102C200004EB0E03C3F8102B8A69002A40D04A8AAD
:102C300005F158033A435B01E2500123D4F81C2804
:102C400003FA0CF31343C4F81C38A64400234A6962
:102C5000CEF8103905F13F03002A39D00A8A04EB77
:102C60008303898B9208012988BF4A43416F561814
:102C700041EA02422946466720465A60FFF78EFE27
:102C8000D8F80C301B8A43EA85531F4305F14803EB
:102C90005B01E7500123D4F81C2803FA05F515431E
:102CA000C4F81C58BDE8F081174FB3E7174FB1E7E0
:102CB00004EB4613D3F8002B22F40042C3F8002B98
:102CC0000123D4F81C2803FA0CF322EA0303BAE721
:102CD00004EB83030E4A04EB461629465A6020464D
:102CE000FFF75CFED6F80039012223F4004302FA14
:102CF00005F5C6F80039D4F81C3823EA0505CFE7F6
:102D000000800010008004100080081000800C106B
:102D100000040002026F12684267FFF721BE000044
:102D20005831C36E49015B5813F4004004D013F4CA
:102D3000001F14BF01200220704700004831C36EFD
:102D400049015B5813F4004004D013F4001F14BF72
:102D5000012002207047000000EB8101CB68196A56
:102D60000B6813604B6853607047000000EB8103F1
:102D700030B5DD68AA691368D36019B9402B84BFE8
:102D8000402313606B8A1468C26E1C4402EB41102E
:102D9000013C09B2B4FBF3F46343033323F00303B0
:102DA00043EAC44343F0C043C0F8103B2B6803F030
:102DB0000303012B0ED1D2F8083802EB411013F4B3
:102DC000807FD0F8003B14BF43F0805343F00053A2
:102DD000C0F8003B02EB4112D2F8003B43F0044341
:102DE000C2F8003B30BD00002DE9F041244D0446FF
:102DF000EE6E06EB4013D3F8087B3807C3F8087B68
:102E00000AD5D6F81438190706D505EB84032146F0
:102E10002846DB685B689847FA072FD5D6F8143840
:102E2000DB072BD505EB8403D968CCB98B69488ABD
:102E30005E68B6FBF0F200FB12628AB91868DA68C5
:102E400090420DD2121A83E81400202383F31188D4
:102E50000B482146FFF78AFF84F31188BDE8F08113
:102E6000012303FA04F26B8923EA02036B81CB6826
:102E700023B121460248BDE8F0411847BDE8F08182
:102E8000BC36022000EB81034A0170B5DD68C36ED9
:102E90006C692668E66056BB1A444FF40020C2F8FD
:102EA00010092A6802F00302012A0AB20ED1D3F8EF
:102EB000080803EB421410F4807FD4F8000914BF13
:102EC00040F0805040F00050C4F8000903EB42127B
:102ED000D2F8000940F00440C2F800090122D3F8FA
:102EE000340802FA01F10143C3F8341870BD19B96E
:102EF000402E84BF4020206020681A442E8A841906
:102F000040F00050013CB4FBF6F440EAC440C6E790
:102F1000F8B504461E48C56E05EB4413D3F808699E
:102F2000F107C3F8086917D5D5F81038DA0713D5B3
:102F300000EB8403D9684B691F68DA68974218D29E
:102F4000D21B00271A605F60202383F3118821467B
:102F5000FFF798FF87F31188330617D50123D5F8BB
:102F60003428A340134211D02046BDE8F840FFF7B3
:102F70001FBD012303FA04F2038923EA020303813C
:102F80008B68002BE8D021469847E5E7F8BD00BFE5
:102F9000BC3602209F482DE9F84FC56E04466E6985
:102FA000AB691E4016F4805F6E6105D0FEF7A8FD88
:102FB000BDE8F84FFFF748BC002E12DAD5F8003E06
:102FC0009B0705D0D5F8003E23F00303C5F8003E6B
:102FD000D5F804388F4823F00103C5F80438FEF70C
:102FE000BBFD370502D58B48FEF7AAFDB0040CD512
:102FF000D5F8083813F0060FEB6823F470530CBFB4
:1030000043F4105343F4A053EB60310704D56368D5
:10301000DB680BB17F489847F2026FD4B3020CD53E
:10302000D4F86C8000274FF00109DFF8E8A1236F86
:10303000F9B29B688B4280F09C80F70619D5E16E4F
:103040000A6AC2F30A1702F00F0302F4F012B2F593
:10305000802F00F0B580B2F5402F0AD104EB830336
:1030600001F58051DB68186A00231A469F4240F040
:103070009C803303D5F818481DD5E70302D50020FE
:10308000FFF7B2FEA50302D50120FFF7ADFE6003F6
:1030900002D50220FFF7A8FE210302D50320FFF787
:1030A000A3FEE20202D50420FFF79EFEA30202D592
:1030B0000520FFF799FE77037FF57AAFE60702D583
:1030C0000020FFF725FFA50702D50120FFF720FF0D
:1030D000600702D50220FFF71BFF210702D503205E
:1030E000FFF716FFE20602D50420FFF711FFA30643
:1030F0007FF55EAF0520FFF70BFF59E7D4F86C8032
:1031000000274FF00109DFF80CA1236F5FFA87FB5E
:103110009B685B4582D308EB4B13D3F8002902F47C
:103120004022B2F5802F22D1D3F80029002A1EDADE
:10313000D3F8002942F09042C3F80029D3F80029BF
:10314000002AFBDB5946E06EFFF728FC228909FACA
:103150000BF322EA0303238104EB8B03DB689B68F8
:1031600013B15946504698475846FFF721FC01379E
:10317000CBE708EB4112D2F8003B03F44023B3F550
:10318000802F10D1D2F8003B002B0CDA628909FAAB
:1031900001F322EA0303638104EB8103DB68DB684C
:1031A0000BB150469847013741E79C0700D10A68A8
:1031B000072B03F101039EBF0270120A013055E78D
:1031C000023301F5805104EB830252689069026872
:1031D000D0F808C04068A2EB000E002210469742CB
:1031E0000AD104EB830463689B699A683A449A6045
:1031F0005A6817445F603CE712F0030F00D108687B
:10320000964502F1010282BF8CF80000000A0CF121
:10321000010CE4E7BC360220C36E03EB4111D1F888
:10322000003B43F40013C1F8003B7047C36E03EB4F
:103230004111D1F8003943F40013C1F80039704747
:10324000C36E03EB4111D1F8003B23F40013C1F826
:10325000003B7047C36E03EB4111D1F8003923F4F2
:103260000013C1F80039704730B50433039C017274
:10327000002104FB0325C361049B00600363059BDD
:103280004060C160426102618561046242628162A4
:10329000C162436330BD00000022416AC2604161E7
:1032A00001616FF001018262C262FEF775BF00002A
:1032B00003694269934203D1C2680AB10020704792
:1032C000181D7047036919600021C2680132C2608D
:1032D000C269134482699342036124BF436A036154
:1032E000FEF74EBF38B504460D46E3683BB1626950
:1032F0000020131D1268A3621344E36238BD237AD1
:1033000033B929462046FEF72BFF0028EDDA38BDF9
:103310006FF00100FBE70000C368C269013BC360B6
:103320004369134482699342436124BF436A436102
:1033300000238362036B03B11847704770B52023E5
:10334000044683F31188866A3EB9FFF7CBFF054632
:1033500018B186F31188284670BDA36AE26A13F893
:10336000015B9342A36202D32046FFF7D5FF0023FF
:1033700083F31188EFE700002DE9F84F04460E466D
:1033800090469946202787F311880025AA46D4F84D
:1033900028B0BBF1000F09D149462046FFF7A2FF34
:1033A00020B18BF311882846BDE8F88FA16AA8EBFD
:1033B000050BE36A5B1A9B4528BF9B46BBF1400F98
:1033C0001BD9334601F1400251F8040B914243F8F6
:1033D000040BF9D1A36A403640354033A362A26A98
:1033E000E36A9A4202D32046FFF796FF8AF31188D8
:1033F0004545D8D287F31188C9E730465A46FDF7CC
:103400002DFDA36A5E445D445B44A362E7E70000D0
:1034100010B5029C04330172C36103FB0421002335
:1034200000608362C362039B40600363049BC460CB
:1034300042610261816104624262436310BD000027
:10344000026A6FF00101C260426A426102610022B9
:103450008262C262FEF7A0BE436902699A4203D14A
:10346000C2680AB100207047184650F8043B0B6050
:1034700070470000C3680021C2690133C36043691B
:10348000134482699342436124BF436A4361FEF758
:1034900077BE000038B504460D46E3683BB12369AA
:1034A00000201A1DA262E2691344E36238BD237A48
:1034B00033B929462046FEF753FE0028EDDA38BD21
:1034C0006FF00100FBE7000003691960C268013A70
:1034D000C260C269134482699342036124BF436A94
:1034E000036100238362036B03B118477047000038
:1034F00070B5202304460E4683F31188856A35B9DA
:103500001146FFF7C7FF10B185F3118870BDA36A9C
:103510001E70A36AE26A01339342A36204D3E16995
:1035200020460439FFF7D0FF002080F3118870BDDA
:103530002DE9F84F04460D4691469A464FF0200873
:1035400088F311880026B346A76A4FB95146204632
:10355000FFF7A0FF20B187F311883046BDE8F88F50
:10356000A06AA9EB0603E76A3F1A9F4228BF1F46DD
:10357000402F1BD905F1400355F8042B9D4240F81C
:10358000042BF9D1A36A40364033A362A26AE36AEE
:103590009A4204D3E16920460439FFF795FF8BF383
:1035A00011884E45D9D288F31188CDE729463A468D
:1035B000FDF754FCA36A3D443E443B44A362E5E767
:1035C000026943699A4203D1C3681BB91846704720
:1035D0000023FBE7836A002BF8D0043B9B1AF5D04D
:1035E0001360C368013BC360C3691A4483699A428C
:1035F000026124BF436A0361002383620123E5E77C
:1036000000F040B94FF08043002258631A61022253
:10361000DA60704700224FF08043DA6070470000A4
:103620004FF0804358637047FEE7000010B5194C17
:10363000FEF79CFCFEF7BEFD802217492046FEF7F0
:1036400043FD012344F8180C0374144B144AD96841
:1036500021F4E0610904090C0A431249DA60CA68DE
:1036600042F08072CA60104A1049C2F8B01F116857
:1036700041F0010111601022DA77202283F8222024
:10368000002383F3118862B60948BDE81040FEF7B5
:103690003DBD00BF482F02208C3E000800ED00E039
:1036A0000003FA05F0ED00E0001000E055CEACC5D7
:1036B000943E00082DE9F84F1E4C4FF00008656954
:1036C00004F11407C1464FF08043266AAA685B6A7A
:1036D0009E1B96421CD34FF0200AAA68236AD5F895
:1036E0000CB0B61A134423622B68BB425F6063615F
:1036F000C5F80C8001D1FFF78DFF89F31188286987
:10370000D8478AF311886569AB689E42E5D2DAE74B
:103710006269BA420CD0916823628E1B9660A868D9
:1037200002282CBF1818981CBDE8F84FFFF778BF87
:10373000BDE8F88F202F0220034B59685A68521AAF
:103740009042FBD8704700BF001000E04B68436018
:103750008B688360CB68C3600B6943614B6903620C
:103760008B6943620B6803607047000008B5274B04
:1037700040F2FF7126481A690A431A611A6922F455
:10378000FF6222F007021A611A691A6B0A431A6370
:103790001A6D0A431A651F4A1B6D1146FFF7D6FFC3
:1037A0001D4802F11C01FFF7D1FF1C4802F138014E
:1037B000FFF7CCFF1A4802F15401FFF7C7FF194881
:1037C00002F17001FFF7C2FF174802F18C01FFF709
:1037D000BDFF164802F1A801FFF7B8FF144802F137
:1037E000C401FFF7B3FF134802F1E001FFF7AEFF9A
:1037F000114802F1FC01FFF7A9FF104802F58C7196
:10380000FFF7A4FFBDE8084000F09EB80038024072
:1038100000000240B43E00080004024000080240DC
:10382000000C024000100240001402400018024048
:10383000001C0240002002400024024000280240F8
:1038400008B500F0F5F9FFF7F1FEFEF7DBFFBDE884
:103850000840FEF7B9BD0000704700004FF08043FC
:103860001A69920710B508D500241C61202383F340
:103870001188FFF71FFF84F31188BDE81040FEF7A1
:10388000E3BF0000104B08211C201A6C42F001021B
:103890001A641A6E42F001021A660C4A1B6E936893
:1038A00043F0010393604FF080436B229A624FF024
:1038B000FF32DA6200229A615A63DA605A600122AA
:1038C0005A611A60FDF726BD00380240002004E06E
:1038D0001B4B4FF0FF3000211A696FEA42526FEA2A
:1038E00052521A611A69C2F30A021A611A695A69B4
:1038F00058615A6959615A691A6A62F080521A62AB
:103900001A6A02F080521A621A6A5A6A58625A6A2D
:1039100059625A6A0B4A106840F480701060186F40
:1039200000F44070B0F5007F03D04FF4803018678A
:103930001967536823F40073536000F059B900BF4E
:103940000038024000700040354B4FF44041354A8A
:103950001A64354A11601A6842F001021A601A6846
:103960009207FCD59A6822F003029A602C4B194604
:103970009A6812F00C02FBD1186800F0F900186088
:103980009A601A6842F480321A600B689B03FCD577
:103990004B6F43F001034B67214B5A6F9007FCD5E7
:1039A000224A5A601A6842F080721A601E4B1A4608
:1039B00059684904FCD5196841F48031196053688D
:1039C000D803FCD5136843F400331360164A5368D8
:1039D0009903FCD5124B1A689201FCD5144A40F2A7
:1039E00007319A6040F20112C3F88C200022C3F81C
:1039F0009020104A11609A6842F002029A60084BC7
:103A00009A6802F00C02082AFAD15A6C42F48042F9
:103A10005A645A6E42F480425A665B6E704700BF29
:103A200000380240000400100070004008364009D1
:103A300000948838003C0240084A08B55369116870
:103A40000B4003F00103536123B1054A13680BB126
:103A500050689847BDE80840FEF7F6BE003C0140BC
:103A6000C8250220084A08B5536911680B4003F0C5
:103A70000203536123B1054A93680BB1D06898479C
:103A8000BDE80840FEF7E0BE003C0140C82502202A
:103A9000084A08B5536911680B4003F004035361E9
:103AA00023B1054A13690BB150699847BDE8084036
:103AB000FEF7CABE003C0140C8250220084A08B5EE
:103AC000536911680B4003F00803536123B1054AA1
:103AD00093690BB1D0699847BDE80840FEF7B4BEC2
:103AE000003C0140C8250220084A08B55369116806
:103AF0000B4003F01003536123B1054A136A0BB165
:103B0000506A9847BDE80840FEF79EBE003C014061
:103B1000C8250220174B10B55C691A68144004F4DC
:103B200078725A61A30604D5134A936A0BB1D06A1E
:103B30009847600604D5104A136B0BB1506B984739
:103B4000210604D50C4A936B0BB1D06B9847E20564
:103B500004D5094A136C0BB1506C9847A30504D5E2
:103B6000054A936C0BB1D06C9847BDE81040FEF746
:103B70006BBE00BF003C0140C82502201A4B10B5A7
:103B80005C691A68144004F47C425A61620504D5E9
:103B9000164A136D0BB1506D9847230504D5134A8F
:103BA000936D0BB1D06D9847E00404D50F4A136EA6
:103BB0000BB1506E9847A10404D50C4A936E0BB11B
:103BC000D06E9847620404D5084A136F0BB1506F4A
:103BD0009847230404D5054A936F0BB1D06F9847DB
:103BE000BDE81040FEF730BE003C0140C825022071
:103BF000062108B50846FDF78DFB06210720FDF7D5
:103C000089FB06210820FDF785FB06210920FDF729
:103C100081FB06210A20FDF77DFB06211720FDF719
:103C200079FB06212820BDE80840FDF773BB0000A2
:103C300008B5FFF74DFEFDF7FFF9FDF715FDFDF7A0
:103C4000EBFEFDF7BFFDFFF707FEBDE80840FFF7FD
:103C5000D7BC0000034611F8012B03F8012B002A02
:103C6000F9D1704712101213121100000010410018
:103C700001105A00602F022048260220B42602209C
:103C800053544D3332463F3F3F3F3F3F0053544D27
:103C9000333246375B347C355D780053544D3332D4
:103CA00046375B367C375D780000000000960000E8
:103CB0000000000000000000000000000000000004
:103CC0000000000000000000311600081D1600086A
:103CD0005916000845160008511600083D16000840
:103CE00029160008151600086516000800000000D7
:103CF0003D1700082917000865170008511700082C
:103D00005D1700084917000835170008211700083B
:103D1000C1170008000000000100000000000000C2
:103D2000020000000000000069190008D119000815
:103D300040004000F8330220083402200200000056
:103D4000000000000300000000000000151A000839
:103D500000000000100000001834022000000000E5
:103D60000100000000000000BC360220010102003A
:103D70004172647550696C6F740025424F41524422
:103D8000252D424C002553455249414C2500000049
:103D900069230008D1220008D51800084D23000827
:103DA00043000000A83D000809024300020100C0D2
:103DB000320904000001020201000524001001057F
:103DC00024010001042402020524060001070582E3
:103DD000030800FF09040100020A000000070501B2
:103DE00002400000070581024000000012000000B0
:103DF000F43D000812011001020000400912415771
:103E000000020102030100000403090425424F419E
:103E10005244250043554156763500303132333413
:103E2000353637383941424344454600008000006A
:103E30000080000000800000008000000000020000
:103E40000000040000000400000004000000040062
:103E50000000040000000400000004000000000056
:103E60006D1B00084D1E0008F91E000840004000B0
:103E7000343702203437022001000000443702208A
:103E80008000000040010000050000006D61696EC7
:103E900000000000AC3E00085037022048390220E4
:103EA00001000000293600080000000069646C650C
:103EB000000000000000802A00000000AAAAAAAAB0
:103EC00000000000FFFF00000000000000A00A004A
:103ED0000000000000000000AAAAAAAA000000003A
:103EE000FFFF000000000000000000000050000084
:103EF00000000000AAAAAAAA00000000FFFF00001C
:103F00000000000000000000802900000000000008
:103F1000AAAAAAAA40150000FFFF000000707007BF
:103F2000000000000000020000000000AAAAAAAAE7
:103F300000000100FFFF000000000000080000007A
:103F400050255000000000000AA2AAAA50155000F7
:103F5000FFFF00000000000800000000000010004B
:103F600000000000AAAAAAAA00001000FFFF00009B
:103F7000000000000000000000040000000000003D
:103F8000AAAAAAAA00040000FFFF00000000000087
:103F9000000000000051510000000000AAAAAAAAD7
:103FA00000515100FFFF0000000000000000000071
:103FB0000000000000000000000000000000000001
:103FC00000000000000000000000000000000000F1
:103FD00000000000000000000000000000000000E1
:103FE0000000000000000000FF00000000000000D2
:103FF000803C00083F000000490400008D3C0008A0
:104000003F000000510400009B3C00083F000000FE
:10401000009600000000080004000000083E0008B0
:104020000000000000000000000000000000000090
:104030000000000000000000FFFFFFFFFFFFFFFF88
:10404000FFFFFFFFFFFFFFFFFFFFFFFFFFFFFFFF80
:10405000FFFFFFFFFFFFFFFFFFFFFFFFFFFFFFFF70
:10406000FFFFFFFFFFFFFFFFFFFFFFFFFFFFFFFF60
:10407000FFFFFFFFFFFFFFFFFFFFFFFFFFFFFFFF50
:1080000000060220ED8C00088DF30F08A182000805
:108010000DF30F0805F30F0809F30F08EF8C0008A4
:10802000EF8C0008EF8C0008EF8C00087D541608D8
:10803000EF8C0008EF8C0008EF8C0008EF8C000834
:10804000EF8C0008EF8C0008EF8C0008EF8C000824
:10805000EF8C0008EF8C00089DCE1608C5CE1608E0
:10806000EDCE160815CF16083DCF1608E95E1608A6
:10807000115F16083D5F1608695F1608955F1608C0
:10808000BD5F1608E95F1608555D160815E20F0872
:1080900045E20F0875E20F08EF8C000865CF16085F
:1080A000C5D01608D9D01608EDD01608F1D016089C
:1080B00005D11608EF8C000815D11608C166160800
:1080C0002967160891671608F9671608EF8C0008EB
:1080D000EF8C000839D016084DD0160861D016086C
:1080E000C9CF1608EF8C0008EF8C000829D11608BC
:1080F000EF8C0008EF8C0008EF8C00081560160864
:10810000EF8C0008ED6E1608EF8C0008EF8C00086D
:1081100075D01608EF8C0008EF8C0008EF8C000873
:10812000416016086960160895601608C160160857
:10813000ED601608EF8C0008EF8C0008A5E20F0830
:10814000D5E20F0805E30F08EF8C0008FDC81608FC
:1081500015611608416116086D61160889D0160868
:1081600061681608C9681608EF8C0008EF8C0008D3
:10817000EF8C0008EF8C0008EF8C0008EF8C0008F3
:10818000EF8C0008EF8C00089DD01608B1D01608BF
:10819000EF8C0008EF8C0008EF8C0008EF8C0008D3
:1081A000EF8C0008EF8C0008EF8C0008EF8C0008C3
:1081B000EF8C0008EF8C0008EF8C0008316916087E
:1081C00099691608EF8C0008EF8C0008EF8C000806
:1081D000EF8C0008EF8C0008EF8C0008EF8C000893
:1081E000EF8C0008EF8C0008EF8C0008EF8C000883
:1081F000EF8C0008EF8C0008EF8C0008EF8C000873
:1082000049CA0008E10701084D5101087DC2010873
:108210005D350208D10203084560030849EF0308F1
:1082200011780508E1F00708D1F7070835A208081A
:1082300045210908DD290908692D090835B609080D
:10824000D5E1090809ED0908358E0A08F9BA0B08C5
:10825000156F0C08917E0C0835E60F0871EB0F08BE
:10826000B50A100819B211089103120871581208C2
:1082700059AC1208C95314080D94140851B11408CC
:1082800031F4140865141508A54415085D51150846
:10829000F18A15080D951508000000000000000087
:1082A000EFF30383EFF30982EFF30881DFF814D0D3
:1082B0002DE9FE4F684600F0EFFFBDE8FE4F8D460A
:1082C00070470000AC330220F1EE101AA0EC200A37
:1082D00001607047A0EC108A704700BF81F0004138
:1082E00002E000BF83F0004330B54FEA41044FEA9B
:1082F000430594EA050F08BF90EA020F1FBF54EA36
:10830000000C55EA020C7FEA645C7FEA655C00F0D1
:10831000E2804FEA5454D4EB5555B8BF6D420CDDA2
:108320002C4480EA020281EA030382EA000083EA25
:10833000010180EA020281EA0303362D88BF30BDC5
:1083400011F0004F4FEA01314FF4801C4CEA11311B
:1083500002D0404261EB410113F0004F4FEA03337A
:108360004CEA133302D0524263EB430394EA050F05
:1083700000F0A780A4F10104D5F1200E0DDB02FA74
:108380000EFC22FA05F2801841F1000103FA0EF208
:10839000801843FA05F359410EE0A5F120050EF1CE
:1083A000200E012A03FA0EFC28BF4CF0020C43FAFF
:1083B00005F3C01851EBE37101F0004507D54FF00C
:1083C000000EDCF1000C7EEB00006EEB0101B1F55C
:1083D000801F1BD3B1F5001F0CD349085FEA3000A2
:1083E0004FEA3C0C04F101044FEA445212F5800FAD
:1083F00080F09A80BCF1004F08BF5FEA500C50F14A
:10840000000041EB045141EA050130BD5FEA4C0C2C
:10841000404141EB0101013C28BFB1F5801FE9D289
:1084200091F0000F04BF01460020B1FA81F308BFAC
:108430002033A3F10B03B3F120020CDA0C3208DD78
:1084400002F1140CC2F10C0201FA0CF021FA02F153
:108450000CE002F11402D8BFC2F1200C01FA02F1C3
:1084600020FA0CFCDCBF41EA0C019040E41AA2BFE8
:1084700001EB0451294330BD6FEA04041F3C1CDAB0
:108480000C340EDC04F11404C4F1200220FA04F0D0
:1084900001FA02F340EA030021FA04F345EA03017A
:1084A00030BDC4F10C04C4F1200220FA02F001FA3C
:1084B00004F340EA0300294630BD21FA04F02946BE
:1084C00030BD94F0000F83F4801306BF81F4801157
:1084D0000134013D4EE77FEA645C18BF7FEA655CCA
:1084E00029D094EA050F08BF90EA020F05D054EA9C
:1084F000000C04BF1946104630BD91EA030F1EBFA1
:108500000021002030BD5FEA545C05D140004941A4
:1085100028BF41F0004130BD14F580043CBF01F597
:10852000801130BD01F0004545F0FE4141F470017D
:108530004FF0000030BD7FEA645C1ABF1946104658
:108540007FEA655C1CBF0B46024650EA013406BF59
:1085500052EA033591EA030F41F4002130BD00BF18
:1085600090F0000F04BF0021704730B54FF48064D5
:1085700004F132044FF000054FF0000150E700BF56
:1085800090F0000F04BF0021704730B54FF48064B5
:1085900004F1320410F0004548BF40424FF00001A2
:1085A0003EE700BF42004FEAE2014FEA31014FEAE5
:1085B00002701FBF12F07F4393F07F4F81F0605134
:1085C000704732F07F4208BF704793F07F4F04BF7F
:1085D00041F40021704730B54FF4607401F000455C
:1085E00021F000411CE700BF50EA010208BF7047BC
:1085F00030B54FF000050AE050EA010208BF7047AD
:1086000030B511F0004502D5404261EB41014FF415
:10861000806404F132045FEA915C3FF4D8AE4FF01D
:1086200003025FEADC0C18BF03325FEADC0C18BF00
:10863000033202EBDC02C2F1200300FA03FC20FA51
:1086400002F001FA03FE40EA0E0021FA02F114449E
:10865000BDE600BF80F0004002E000BF81F00041B5
:1086600042001FBF5FEA410392EA030F7FEA226CD8
:108670007FEA236C6AD04FEA1262D2EB1363C1BF68
:10868000D218414048404140B8BF5B42192B88BFD7
:10869000704710F0004F40F4000020F07F4018BFFA
:1086A000404211F0004F41F4000121F07F4118BF1A
:1086B000494292EA030F3FD0A2F1010241FA03FCC2
:1086C00010EB0C00C3F1200301FA03F100F00043AA
:1086D00002D5494260EB4000B0F5000F13D3B0F172
:1086E000807F06D340084FEA310102F10102FE2AE1
:1086F00051D2B1F1004F40EBC25008BF20F0010051
:1087000040EA03007047490040EB0000013A28BFEF
:10871000B0F5000FEDD2B0FA80FCACF1080CB2EB72
:108720000C0200FA0CF0AABF00EBC25052421843F0
:10873000BCBFD0401843704792F0000F81F4000195
:1087400006BF80F400000132013BB5E74FEA410368
:108750007FEA226C18BF7FEA236C21D092EA030FD4
:1087600004D092F0000F08BF0846704790EA010F4E
:108770001CBF0020704712F07F4F04D1400028BF7B
:1087800040F00040704712F100723CBF00F500005D
:10879000704700F0004343F0FE4040F40000704793
:1087A0007FEA226216BF08467FEA2363014642023F
:1087B00006BF5FEA412390EA010F40F48000704752
:1087C0004FF0000304E000BF10F0004348BF4042F8
:1087D0005FEA000C08BF704743F0964301464FF034
:1087E00000001CE050EA010208BF70474FF0000390
:1087F0000AE000BF50EA010208BF704711F00043D1
:1088000002D5404261EB41015FEA010C02BF8446A0
:108810000146002043F0B64308BFA3F18053A3F5FF
:108820000003BCFA8CF2083AA3EBC25310DB01FA46
:1088300002FC634400FA02FCC2F12002BCF1004FCA
:1088400020FA02F243EB020008BF20F0010070475B
:1088500002F1200201FA02FCC2F1200250EA4C00AF
:1088600021FA02F243EB020008BF20EADC707047F5
:108870007BB972B90029BEBF00204FF0004106E06D
:1088800008BF00281CBF6FF000414FF0FF3000F020
:108890002BBAADF1080C6DE904CE002909DB002BE1
:1088A0001ADB00F0B9F8DDF804E0DDE9022304B0DA
:1088B0007047404261EB4101002B1BDB00F0ACF83C
:1088C000DDF804E0DDE9022304B0404261EB410140
:1088D000524263EB43037047524263EB430300F0A1
:1088E0009BF8DDF804E0DDE9022304B0404261EBCF
:1088F00041017047524263EB430300F08DF8DDF80D
:1089000004E0DDE9022304B0524263EB4303704705
:1089100053B94AB9002908BF00281CBF4FF0FF31E6
:108920004FF0FF3000F0E0B9ADF1080C6DE904CE76
:1089300000F072F8DDF804E0DDE9022304B07047CE
:10894000430803F05533C01A830803F0333300F0B3
:108950003330184400EB101000F00F3000EB002013
:1089600000EB0040000E704708B502460B4643EC92
:10897000172BB5EEC07BF1EE10FA03D4BDE808402A
:1089800000F02AB8B1EE477B51EC170B00F024F849
:10899000404261EB410108BD9FED0B6B07EE900A71
:1089A0009FED0B5BB7EEE77A27EE066BBCEEC66B6E
:1089B000B8EE464BA4EE457BFCEEC77B16EE101AD4
:1089C00017EE900A704700BF000000000000F03D65
:1089D000000000000000F0419FED0B6B41EC170B15
:1089E0009FED0B5B27EE066BBCEEC66BB8EE464BFD
:1089F000A4EE457BFCEEC77B16EE101A17EE900A2C
:108A0000704700BFAFF30080000000000000F03DA1
:108A1000000000000000F0412DE9F047089D0446E9
:108A20008E46002B4DD18A42944669D9B2FA82F221
:108A300052B101FA02F3C2F1200120FA01F10CFA5D
:108A400002FC41EA030E94404FEA1C48210CBEFB95
:108A5000F8F61FFA8CF708FB16E341EA034306FB1E
:108A600007F199420AD91CEB030306F1FF3080F0AD
:108A70001F81994240F21C81023E63445B1AA4B2FA
:108A8000B3FBF8F008FB103344EA034400FB07F79C
:108A9000A7420AD91CEB040400F1FF3380F00A81DD
:108AA000A74240F207816444023840EA0640E41BD2
:108AB00000261DB1D4400023C5E900433146BDE87E
:108AC000F0878B4209D9002D00F0EF800026C5E920
:108AD000000130463146BDE8F087B3FA83F6002E38
:108AE0004AD18B4202D3824200F2F980841A61EBB0
:108AF000030301209E46002DE0D0C5E9004EDDE7CE
:108B000002B9FFDEB2FA82F2002A40F09280A1EBB5
:108B10000C014FEA1C471FFA8CFE0126200CB1FB0A
:108B2000F7F307FB131140EA01410EFB03F0884203
:108B300008D91CEB010103F1FF3802D2884200F290
:108B4000CB804346091AA4B2B1FBF7F007FB101122
:108B500044EA01440EFB00FEA64508D91CEB0404C0
:108B600000F1FF3102D2A64500F2BB800846A4EB1B
:108B70000E0440EA03409CE7C6F12007B34022FA06
:108B800007FC4CEA030C20FA07F401FA06F31C4335
:108B9000F9404FEA1C4900FA06F3B1FBF9F8200C42
:108BA0001FFA8CFE09FB181140EA014108FB0EF088
:108BB000884202FA06F20BD91CEB010108F1FF3AD8
:108BC00080F08880884240F28580A8F102086144E4
:108BD000091AA4B2B1FBF9F009FB101144EA0141F2
:108BE00000FB0EFE8E4508D91CEB010100F1FF349D
:108BF0006CD28E456AD90238614440EA0840A0FB35
:108C00000294A1EB0E01A142C846A64656D353D00A
:108C10005DB1B3EB080261EB0E0101FA07F722FA2E
:108C200006F3F1401F43C5E9007100263146BDE857
:108C3000F087C2F12003D8400CFA02FC21FA03F3BA
:108C4000914001434FEA1C471FFA8CFEB3FBF7F03B
:108C500007FB10360B0C43EA064300FB0EF69E4260
:108C600004FA02F408D91CEB030300F1FF382FD2F9
:108C70009E422DD9023863449B1B89B2B3FBF7F6A1
:108C800007FB163341EA034106FB0EF38B4208D97A
:108C90001CEB010106F1FF3816D28B4214D9023EBB
:108CA0006144C91A46EA004638E72E46284605E7D9
:108CB0000646E3E61846F8E64B45A9D2B9EB0208AA
:108CC00064EB0C0E0138A3E74646EAE7204694E73A
:108CD0004046D1E7D0467BE7023B614432E730466D
:108CE00009E76444023842E7704700BF02E000F041
:108CF00000F8FEE772B6374880F30888364880F3FC
:108D0000098836483649086040F20000CCF200007D
:108D10004EF63471CEF200010860BFF34F8FBFF3FF
:108D20006F8F40F20000C0F2F0004EF68851CEF294
:108D300000010860BFF34F8FBFF36F8F4FF000004B
:108D4000E1EE100A4EF63C71CEF2000108600620FA
:108D500080F31488BFF36F8F63F1E8F961F1FAFFD4
:108D60004FF055301F491B4A91423CBF41F8040B5C
:108D7000FAE71D49184A91423CBF41F8040BFAE753
:108D80001A491B4A1B4B9A423EBF51F8040B42F84A
:108D9000040BF8E700201849184A91423CBF41F8FB
:108DA000040BFAE763F104FA62F1DEF8144C154D96
:108DB000AC4203DA54F8041B8847F9E703F034FEA9
:108DC000114C124DAC4203DA54F8041B8847F9E702
:108DD00063F1ECB9000602200022022000800008A6
:108DE00008ED00E0000002200006022028D31B0846
:108DF00000220220B8310220B83102202C1E0420AB
:108E00000082000898820008988200089882000872
:108E10002DE9F04F2DED108AC1F80CD0D0F80CD010
:108E2000BDEC108ABDE8F08F002383F3118828463B
:108E3000A047002061F1BCFCFEE761F1BBFA00DF56
:108E4000FEE7000070B54FF0FF0C4CF4E06C1CEA3C
:108E500011541DBF1CEA135594EA0C0F95EA0C0F30
:108E600000F0DEF82C4481EA030621EA4C5123EAA3
:108E70004C5350EA013518BF52EA033541F48011D2
:108E800043F4801338D0A0FB02CE4FF00005E1FB85
:108E900002E506F00042E0FB03E54FF00006E1FBCF
:108EA00003569CF0000F18BF4EF0010EA4F1FF0412
:108EB000B6F5007F64F5407404D25FEA4E0E6D4152
:108EC00046EB060642EAC62141EA55514FEAC52063
:108ED00040EA5E504FEACE2EB4F1FD0C88BFBCF5DF
:108EE000E06F1ED8BEF1004F08BF5FEA500E50F190
:108EF000000041EB045170BD06F0004646EA010156
:108F000040EA020081EA0301B4EB5C04C2BFD4EB87
:108F10000C0541EA045170BD41F480114FF0000E80
:108F2000013C00F3AB8014F1360FDEBF002001F0EE
:108F3000004170BDC4F10004203C35DA0C341BDC68
:108F400004F11404C4F1200500FA05F320FA04F03A
:108F500001FA05F240EA020001F0004221F000416E
:108F600010EBD37021FA04F642EB06015EEA430EE1
:108F700008BF20EAD37070BDC4F10C04C4F1200511
:108F800000FA04F320FA05F001FA04F240EA0200C4
:108F900001F0004110EBD37041F100015EEA430E95
:108FA00008BF20EAD37070BDC4F1200500FA05F2B5
:108FB0004EEA020E20FA04F301FA05F243EA020334
:108FC00021FA04F001F0004121FA04F220EA020043
:108FD00000EBD3705EEA430E08BF20EAD37070BD89
:108FE00094F0000F0FD101F00046400041EB010169
:108FF00011F4801F08BF013CF7D041EA060195F04B
:10900000000F18BF704703F00046520043EB030304
:1090100013F4801F08BF013DF7D043EA06037047F1
:1090200094EA0C0F0CEA135518BF95EA0C0F0CD0FC
:1090300050EA410618BF52EA4306D1D181EA030142
:1090400001F000414FF0000070BD50EA410606BF3C
:109050001046194652EA430619D094EA0C0F02D181
:1090600050EA013613D195EA0C0F05D152EA0336C6
:109070001CBF104619460AD181EA030101F00041E4
:1090800041F0FE4141F470014FF0000070BD41F02D
:10909000FE4141F4780170BD4FEA410212F5001221
:1090A00015D211D56FF47873B3EB625212D94FEA2F
:1090B000C12343F0004343EA505311F0004F23FA19
:1090C00002F018BF404270474FF00000704750EA6E
:1090D000013005D111F0004008BF6FF0004070472B
:1090E0004FF00000704700BF4FEA4102B2F1E04389
:1090F00024BFB3F5001CDCF1FE5C0DD901F0004C7F
:109100004FEAC0024CEA5070B2F1004F40EB8300CE
:1091100008BF20F00100704711F0804F21D113F1FA
:109120003872BCBF01F00040704741F480114FEA33
:109130005252C2F11802C2F1200C10FA0CF320FABC
:1091400002F018BF40F001004FEAC1234FEAD323D9
:1091500003FA0CFC40EA0C0023FA02F34FEA430343
:10916000CCE77FEA625307D150EA01331EBF4FF0CC
:10917000FE4040F44000704701F0004040F0FE40E7
:1091800040F40000704700BF01F0FF01102A2BDB04
:1091900010F0070F08D010F8013B013A8B422DD098
:1091A00010F0070F42B3F6D1F0B441EA012141EAD1
:1091B000014122F007047FF000070023F0E8025687
:1091C000083C85EA010586EA010685FA47F5A3FA17
:1091D00087F586FA47F6A5FA87F68EB9EED1F0BC88
:1091E00001F0FF0102F0070232B110F8013B013A31
:1091F00083EA010313B1F8D10020704701387047AA
:10920000002D06BF35460338073815F0010F07D18A
:10921000013015F4807F02BF013015F4C03F0130EA
:10922000F0BC0138704700BFEC46A0E8F05F4FF09B
:1092300000007047B0E8F05FE546080008BF012075
:10924000704700BF10F8012B11F8013B012A28BF1D
:109250009A42F7D0D01A7047034613F8012B002A20
:10926000FBD1181A01387047A8B110B504460AE0BE
:1092700000F08CFA14F8041C54E903031B1AB3FB26
:10928000F1F200F083FA204654F80C3B0822012149
:109290000133EDD110BD70472DE9F04F0023A7B089
:1092A0000293C36A009013F0040FD0E9002118BFA5
:1092B0000A46D9064FF0E021D3694CBF02F12000E5
:1092C00002F168000192DB0903F0040303430393F6
:1092D000D1F8883D03F4A003B3F5A00F01D1012319
:1092E000029393694FF004094F4D4FF001081B881A
:1092F0004E4C03F47F43A3F53E43B3FA83F35B097B
:10930000049329E000F036F9FFF7AEFF4FF0E023B9
:10931000D3F8003D03F47023B3F5402F0ED0444A38
:109320004FF0FF3305A88DF81C90059214328DF88C
:1093300028800692CDE90833FFF796FF2B68A342F9
:1093400006D03C4B0422012105A8059300F01EFA2B
:1093500000F066FB00285ED103A82C6000F002FC40
:1093600004220121344800F011FA0422012102A84C
:1093700000F00CFA10220121019800F007FA009881
:10938000202201210C3000F001FA01980422012171
:10939000103000F0FBF90422012103A800F0F6F9D7
:1093A00001980C220121143000F0F0F90C22012167
:1093B000009800F0EBF9029BDA07A3D5009BDB6A6B
:1093C000DB0622D415A80DF1140AFEF783FFDDF8A1
:1093D00004E0D4460EF120060EF1600B3068103622
:1093E00056F80C1C674656F8082C0CF1100C56F871
:1093F000043C5E450FC7F1D1DEF86030259384222E
:109400005046012100F0C2F97CE70DF1140A5046E4
:10941000FEF75AFFF3E7049B1BB1019A93690233ED
:10942000936127B0BDE8F08FB8310220ED55CEAC86
:1094300028ED00E0ACCE55ED5064170838B5272074
:109440003B255FF14BF80F4B0F4A4FF0FF34196A81
:109450000D2041F480211962196A21F480211962DA
:10946000196A196C41F480211964196E41F4802144
:10947000196601211B6E054BD560146210601970CE
:1094800038BD00BF0038024000480040E4330220ED
:10949000002953D02DE9F84F074689460026284D6C
:1094A000DFF8A480274C17F801AB2B784FEA1A128B
:1094B00018F802B0002B3CD0C4F828B0E369580675
:1094C00004D462F1F9FDE3695906FAD50AF00F0AEE
:1094D0002B7818F80AA04BB3C4F828A0E3695A0601
:1094E00004D462F1E9FDE3695B06FAD50136B145C2
:1094F00022D03107D7D12B784FF00D0BDFF84CA0DD
:109500008BB1C4F828B0E3695A0604D462F1D4FDE3
:10951000E3695B06FAD51AF801BFBBF1000FC2D0B0
:109520002B78002BEDD1FFF789FFEAE7FFF786FFE5
:10953000D2E7FFF783FFBFE7BDE8F88F704700BFB2
:10954000E433022000480040D8641708B0A7180888
:10955000014B1868704700BFFCFF1F08014B024811
:10956000C01A7047E0E21B0800002008004870475E
:10957000E0E21B08774943F69822774B09682DE90A
:10958000F04F0A441B7883B0744F02EB030960F17B
:109590000FFE734B0446002800F0C8800225FF1A16
:1095A000DFF8E0810126DFF8CCB130E01846019108
:1095B00062F1FEF90199002836D1206AAA460AF123
:1095C00001030AEB4A0E04F13C058944DBB2014475
:1095D0000BEB8E0CB94503EB43034BF82E40CCF854
:1095E00004500AF102058CF808600BEB830CEDB215
:1095F0004BF823008CF80860CCF8041023D22046E6
:1096000060F1E6FD0446002835D04E2D33D8206A9F
:10961000404505D0211AE369002BC7D1AA46CEE701
:10962000504BA3EB0801F6E705EB450C01350BEBBE
:109630008C005FFA85FA0672E3694BF82C300D3323
:109640004360206ABBE74F2D63D94FF0FF330122FF
:10965000CBF8B4338BF8BC23CBF8B833424B1B7830
:109660002BB1424A424B12681B68CBE900234148A8
:1096700003B0BDE8F08FB7EB0900E4D44E2DE2D87B
:109680000AF1030A3C4EDFF800C15FFA8AFAA6EB42
:109690000C03BAF14E0F514694BF002401248342BB
:1096A0002BDC05EB450503EB090201200BEB8503E1
:1096B0004BF825C05E601872BA1A12D48CB92F48C4
:1096C00001EB41052E4BC41A944224DD1A440AF1E1
:1096D00001014BF825300BEB8503C9B25A6001221A
:1096E0001A7201EB41054FF0FF3201210BEB8503AC
:1096F0004BF8252019725A60B0E705EB45050122A9
:1097000060440BEB85034BF825C01A723A4658604B
:10971000D2E72946E5E70AF1010101224BF825309D
:109720000BEB8503C9B258601A72DAE7FF1AB7EB80
:1097300009000BD4104E4FF0030ADFF84CC002258D
:10974000DFF830B05146A6EB0C03A8E70221DFF8A2
:1097500024B0C6E7D4330220AC3302200000200836
:10976000E0E21B080022022000220220D83302205F
:10977000D0330220042202202C1E042000000820E6
:10978000301E042000060220B83102209A4B1B78BC
:109790002DE9F04F824685B00E4693462BB9974B84
:1097A0001B782BBB05B0BDE8F08F022900F0EE80DE
:1097B000042900F0B580012900F0AE80904D2B788F
:1097C0000D27DFF858828F4C7BB1A762E3695A06F8
:1097D00004D462F171FCE3695B06FAD518F8017FE5
:1097E000002FDCD02B78002BEFD1FFF727FEECE722
:1097F000854B4FF00009854A9B1A0093CB45D1D089
:10980000834F844C38682578031D009A2B4493427B
:1098100079D2202D51D0022E24D0042E0DD0012E2D
:10982000ECD12378DFF8F0815A1C22701AF8092055
:1098300009F1010908F80320E0E7DFF8DC810025E1
:10984000434620789AF80010421CE9400835D2B20D
:1098500008F80010202A227018D0202DF1D109F12B
:109860000109CBE725789AF80030DFF8AC8108F8D9
:1098700005300135EDB2202D257030D06B1C09F17B
:1098800001092370002308F80530B7E738685F49FD
:1098900001920844194661F153FE39684FF0000304
:1098A000019A203123705C4B39600021184667F122
:1098B00095FF62F101FC584BCFE7544B2A465649BD
:1098C000184461F13DFE3B6800212A46203352488E
:1098D00021703B6067F182FF62F1EEFB9BE74B4B2F
:1098E0002A4638684146184461F12AFE3B68002147
:1098F0002A462033404621703B6067F16FFF62F1DA
:10990000DBFB2578BAE7444A4FF0FF312023D161D1
:10991000237005B0BDE8F08F1146FFF7B9FD4DE7A4
:10992000002A3FF44BAF02460027354D0DF10C08DD
:1099300052F8043B334C0092039301910137042108
:109940004046FFF7A5FDBB451ED0009ABE0752F862
:10995000043B00920393F1D12A780D26DFF8BC90E6
:109960007AB1A662E369580604D462F1A5FBE36903
:109970005906FAD519F8016F002EDFD02A78002A8F
:10998000EFD1FFF75BFDECE7019E18E7002A3FF4FB
:1099900015AF024600271A4D0DF10C0832F8023BB4
:1099A000184C0092ADF80C3001910137022140466D
:1099B000FFF76EFDBB45E7D0009A790732F8023B0E
:1099C0000092ADF80C30F0D12A780D26DFF84C90DB
:1099D0007AB1A662E3695A0604D462F16DFBE369C9
:1099E0005B06FAD519F8016F002EDED02A78002A1E
:1099F000EFD1FFF723FDECE7AD3302200022022078
:109A0000E43302200048004000002008E0E21B0888
:109A1000D4330220AC330220B0330220B0A71808A0
:109A2000F8B5324B1A782AB9314A1078F0B90122C8
:109A30001A70F8BD2F4E0D252F4F304C3B7893B147
:109A4000A562E3695A0604D462F136FBE3695B065A
:109A5000FAD516F8015F002DF0D1294B586800386F
:109A600018BF0120F8BDFFF7E9FCE9E7254D264EB8
:109A70002B68264C26481A1D3178241A0A44A24223
:109A800006D239BB9C421CD8002061F115FEE4E7E8
:109A9000204A4FF0FF31D161202232701844202239
:109AA0001C4961F14DFD2A6833780021194813449F
:109AB000202231702B6067F191FE62F1FDFA2B6874
:109AC000E0E7144920221448CB6161F139FD62F1CD
:109AD000F3FAD9E703F120029442DFD81F29DDD839
:109AE0000C4AD36120223270D8E700BFAD33022088
:109AF0000022022054641708E4330220004800408A
:109B0000DC330220D4330220AC33022000002008D2
:109B1000E0E21B08B0330220E0FF1F080E4B1B7869
:109B200010B5B3B1642100200C4A0D4CD3699B06DB
:109B3000FCD5536ADBB28B424FF0640101D00020A8
:109B4000F4E70130C0B20E2801D0015DEEE700203D
:109B500010BDFFF773FCE5E7E43302200048004046
:109B6000646417082DE9F04102680646EFF30581A9
:109B7000D9205369C9B2F5F0CBFB674B1B782BB9E1
:109B8000664C2378002B37D1BDE8F081644B0D275C
:109B9000DFF8B081634D644C96E8030083E803006E
:109BA0002B7833B3A762E3695F0604D462F184FAC9
:109BB000E3695806FAD518F8017F002FF0D17368D1
:109BC0000BB32B784227DFF88081574C73B1A76223
:109BD000E369590604D462F16FFAE3695A06FAD5CB
:109BE00018F8017F1FB32B78002BF0D1FFF726FC6C
:109BF000EDE7FFF723FCD5E73568002D47D10023BB
:109C00002370BDE8F081DFF844814327464C2B7870
:109C1000002B6AD0A762E3695B0604D462F14CFAB8
:109C2000E3695F06FAD518F8017F002FEFD1DFF85E
:109C3000208120273C4C2B78002B53D0A762E3696E
:109C4000580604D462F138FAE3695906FAD518F8CF
:109C5000017F002FEFD1FFF761FF2B78DFF8F48051
:109C60000D27314C83B1A762E3695A0604D462F12F
:109C700023FAE3695B06FAD518F8017F002F3FF459
:109C80007FAF2B78002BEED1FFF7D8FBEBE7284610
:109C900061F18EFE0028B2D0284661F191FE00F2FB
:109CA0001450854231D3214BA5F214521A60284634
:109CB00061F1A6FE05F5E053834220D81C4A1360EB
:109CC00000231C481C4A03601C481D49801A0B7065
:109CD00002D10DE083420BD252F8041B0433013150
:109CE000F8D08CE7FFF7AAFBA8E7FFF7A7FB91E7FF
:109CF00062F1E2F90120BDE8F04161F1DDBC2846E6
:109D000061F17EFE0A4B1860DAE7284661F158FEE1
:109D1000064B1860CBE700BFAD33022000220220C3
:109D2000DC330220E433022000480040D833022014
:109D3000D0330220D4330220E0E21B0800002008C8
:109D4000AC330220746417087C641708D0641708C9
:109D500088641708B0A7180800207047036800221D
:109D60001B681847F0B50D4683B040210646D7F072
:109D70002DFD18B1154F97F99E321BB901242046CD
:109D800003B0F0BD91F07EFF437A93B1104BB7F969
:109D9000A022D3F8D43FB3F906309A42EEDD0D4944
:109DA0002A460D4B3046009140210024D7F016FD85
:109DB000E5E791F067FF847A002CE7D1074B2A464C
:109DC00040213046D7F00AFDD9E700BFE8730220F2
:109DD000E883022010651708FC641708EC64170874
:109DE000F0B50D469DB020210446D7F0EFFC0028C9
:109DF0005DD0644E96F99E32002B5BD196F98D3280
:109E0000022B7ED0B6F8603241F65832A3F57A7351
:109E10009BB293426ED85C4F96EDB37AD7F89C3FD5
:109E2000D3ED097AB4EEE77AF1EE10FA5BDC96ED49
:109E3000B47AD3ED0B7AB4EEE77AF1EE10FA52DC95
:109E4000B6F99A32002B40F3928096F8842D0D2AB1
:109E500004D80123934013F4215F59D14B4813F0E8
:109E600013FF012862D04A4B93F8651411F01001DA
:109E700055D1602204A8039167F1B0FC642303AAC2
:109E80004449D7F8A40FE3F03FFE38B16423D7F874
:109E90009C0F03AA4049E1F0AFF948B9204603AC52
:109EA0003E4B2A4620210094D7F098FC18E0012070
:109EB0001DB0F0BD06F58052B6F9A032D2F8D42F0D
:109EC000B2F90A1003F10A02914203DD40F28D3229
:109ED000934293DC324B2A4620212046D7F07EFC69
:109EE00000201DB0F0BD2F4B2A4620212046D7F080
:109EF00075FCF5E72C4B2A4620212046D7F06EFC56
:109F0000EEE72A4B2A4620212046D7F067FC79E766
:109F1000274B2A4620212046D7F060FCE0E7254B5E
:109F20002A4620212046D7F059FCD9E7D7F8A80FB8
:109F3000E6F06EF810B3012895D11F4B93F8E83F77
:109F4000F3B119211D4876F085FCC8B1D6F87862C6
:109F500019211A4876F0B4FC864284DD184E194B5C
:109F60002A46202120460096D7F038FCB8E7164B49
:109F70002A4620212046D7F031FCB1E7134EEEE708
:109F8000134EECE7E8730220E8A30220F8C8022091
:109F9000E8930220346617084C66170838661708DD
:109FA0001C65170868651708586517083065170895
:109FB0009C6517081C661708E8830220904B022056
:109FC00004661708BC65170884651708E465170858
:109FD000F465170870B500249AB060220E46054655
:109FE000214602A8019467F1F9FB642201A90D48FA
:109FF000B2F020F9044640B99DF9043043B90A4B48
:10A0000031460A4A2846D8F02DF820461AB070BDCD
:10A01000284601AB054A3146D8F024F820461AB04C
:10A0200070BD00BF249102205066170810B31A08B3
:10A030002DE9F043DFF88491A5B007468846D9F8AA
:10A040004C341A6818461369984705461DF010F8F5
:10A050000021064660220CA80B9167F1BFFB642328
:10A060000BAA294630461CF077F9044698B34848B5
:10A07000AFF004FD9DB997F91E30012B0FD010F001
:10A08000060F24D0A9F5C04018F080FA034660B945
:10A09000404A414638461C46D7F0E4FF17E03E48A8
:10A0A00018F074FA0346002852D003A930461BF07A
:10A0B000F1FC18B19DF80D305B0650D4374D0023EC
:10A0C000D5EDAF7AF5EEC07AF1EE10FA0DDC204650
:10A0D00025B0BDE8F08338460BAB314A4146D7F096
:10A0E000C1FF204625B0BDE8F0833046089308AE96
:10A0F00009930A9307AB05AA04A9019306AB00963E
:10A100001CF0F8FB304649F09DFBD5EDAF7AB4EE7C
:10A11000E70AF1EE10FA29DA9DED057AF4EEC77A36
:10A12000F1EE10FA28D99DED047AF4EEC77AF1EE3B
:10A1300010FA27D99DED067AF4EEC77AF1EE10FAFF
:10A14000C5D8184A41463846D7F08CFF0024BEE7F0
:10A15000154A414638461C46D7F084FFB7E7134AF4
:10A16000414638460024D7F07DFFB0E7104A41460B
:10A170003846D7F077FFE9E70E4A41463846D7F030
:10A1800071FFE3E70C4A41463846D7F06BFFDDE745
:10A19000C47102208C661708E8330220E87302209D
:10A1A000686617080C67170874661708B4661708FE
:10A1B000C4661708DC661708F4661708E8930220DF
:10A1C00070B50D469AB020210646D7F0FFFA18B9AF
:10A1D000012420461AB070BDEEF0AAFA0446002809
:10A1E000F6D00021602202A8019167F1F7FA20461B
:10A1F000642201A9EEF064FA04460028E8D101AB1C
:10A20000024A29463046D7F02DFFE2E710B31A087C
:10A2100070B50D4C05460E46D4F84C341A681846F5
:10A220005369984710B10124204670BDA4F5C04081
:10A2300018F0C0F904460028F5D1044A31462846F2
:10A24000D7F010FFF0E700BFE8930220306717084F
:10A25000F0B583B007460E46D7F0F4FA044610B9BD
:10A26000204603B0F0BD02213846D7F0AFFA0546CC
:10A270000028F5D01548E7F09DFDC205C0F307237F
:10A28000C0F3002401D49B0703D42C46204603B01E
:10A29000F0BD0E48E7F09CFD0D4B9FED0E7A03F6E6
:10A2A0004C73D3ED007AF8EEE77A30EE670AF0EE01
:10A2B000C07AF4EEC77AF1EE10FAE6DD064B3246CC
:10A2C00002213846D7F08AFACAE700BF68B30220F5
:10A2D000E8A302200000C8424467170870B505468D
:10A2E00082B00E46D8F020F9102104462846D7F057
:10A2F0006DFA10B9204602B070BD0848E7F05AFD6B
:10A3000010F00100F6D10446054B284632461021D4
:10A31000D7F064FA204602B070BD00BF68B30220D7
:10A320005867170870B506460D46D7F093FE0446E9
:10A3300008B9204670BD80213046D7F047FA002882
:10A34000F7D0074B93F8313A13B90446204670BD55
:10A35000044B2A46802130460024D7F03FFAE8E734
:10A36000E89302206C67170838B50D4D0446D5F800
:10A37000A80FE5F04DFE012810D0D5F8A80FE5F0A4
:10A3800047FE022804D02046BDE83840D7F0A0B9E7
:10A39000044813F079FC0128F5D138BD002038BD00
:10A3A000E8A30220F8C80220F0B5134C85B00F4690
:10A3B000064604F5A0436A4604F5C044D3F8CC5FD2
:10A3C0000095D3F8D05F0195D3F8D45FD3F8D83F88
:10A3D00002950393D8F016FE054639463046D7F06D
:10A3E000D7FB94F84034284060F3C303C3F3C000A4
:10A3F00084F8403405B0F0BDE8330220F8B5264FAC
:10A40000044626480D46AFF039FBD7F84C340646D3
:10A410001A6818461369984716F0060F0ED168B9E6
:10A42000D7F88034022B09D029462046FFF700FEDA
:10A4300068B301231A4A1846D371F8BD294620464D
:10A44000D7F0AEFC18B329462046FFF7F1FDF0B176
:10A4500008212046D7F0BAF90028EAD0114830F098
:10A4600051FA0028E5D0104BB02193F8242601FBC7
:10A47000023203F58043B2F82E24B3F98E329A42A9
:10A48000D7DD0A4B2A4608212046D7F0A7F900233A
:10A49000034A1846D371F8BDE8930220C471022024
:10A4A00068D0022000370220E833022080671708B6
:10A4B00070B588B006460D46D7F0FEFD044610B9CB
:10A4C000204608B070BD20213046D7F07FF9002823
:10A4D000F6D0194B93F8E420002AF1D093F8C0305D
:10A4E0009B07EDD507AA06A91448AAF093FB0028FC
:10A4F000E6D09DED077ADFED127AB4EEE77AF1EE61
:10A5000010FADDD8DDED066AB7EEC77A2A46304686
:10A51000FDEEE66A0B4B202100249FED055BCDED9F
:10A52000006A8DED045B8DED027BD7F057F9C7E72C
:10A53000000000403333E33FE8B30220C477022039
:10A540009A99193F906717082DE9F04182B00D469E
:10A5500006461CF08DFD07461BF034FA88B33846DA
:10A560001CF0ECFC78B1DFF8CC812946D8F84C041B
:10A5700003689B6998470446A0B1B3685BBB20465B
:10A5800002B0BDE8F08127F03DF990F8461327F0BE
:10A590006FF804460028E6D1594A01213046D7F029
:10A5A00061FDECE7D8F84C0403681B6C9847554AEA
:10A5B000034601213046D7F055FD204602B0BDE8E4
:10A5C000F0810446504A30460121D7F04BFD204629
:10A5D00002B0BDE8F08110213046D7F0F7F8E0B1C5
:10A5E000D7ED937A97ED920A20EE270A64F1B0F93D
:10A5F000A8F50053DFED457AB3F9603220EE270A63
:10A600009FED437A07EE903A20EE070AF8EEE77ADC
:10A61000B4EEE70AF1EE10FA69DC20213046D7F0FB
:10A62000D5F818B198F86534DB0658D44021304687
:10A63000D7F0CCF858B1232D18BF012D01D0042D2F
:10A6400014D1D8F84C040368DB6B984770B1314BD8
:10A65000314A1B68D86A0368DB69934235D12946C1
:10A66000304602B0BDE8F041D7F048BA2B4CD4F8E0
:10A67000D43FA4F5A040B3F9083000EE103AB8EE8C
:10A68000C00A00F0AFFCB5EEC00AF1EE10FA12DC21
:10A69000D8F84C0403685B69984730B9D8F84C0483
:10A6A00003681B6898470B28D1D1D4F8D43FB3F97D
:10A6B0000830002BCBDD1A4C01221A4B40210094AC
:10A6C00030460024D7F08AF859E798470128014618
:10A6D000C5D1154A30460024D7F0C4FC4FE7134BD0
:10A6E0000122202130460024D7F078F847E7104BAC
:10A6F0000122102130460024D7F070F83FE700BF58
:10A70000D0671708E4671708BC671708E02E654292
:10A710000000C84288CD0220599D0008E88302202D
:10A7200010651708006817080C6817081C661708DA
:10A73000F8671708E893022070B50E460546FFF744
:10A7400077FC084B04463146D8712846FFF760FD78
:10A75000034631462846002B08BF0024D7F0FCFDF5
:10A76000204070BD68D002202DE9F0439BB00D461B
:10A77000044691F087FA202192F0FEFC002839D09F
:10A7800091F080FA1F2192F0F7FC60B3594F2946EF
:10A79000594A2046D7F066FC97F84234002603F069
:10A7A0001403142B2ED129462046544A0026D7F0F4
:10A7B00059FC29462046D8F0B9FD48BB0146602225
:10A7C000019002A867F10AF8D7F870040DF10408A7
:10A7D0006421036842461B68984700284BD000203C
:10A7E0001BB0BDE8F08391F04DFAA52192F0C4FCB6
:10A7F0000028CBD13F4F012697F8423403F01403D1
:10A80000142BD0D029462046D8F090FD0028D5D072
:10A810004FF00009602202A80DF104084946CDF866
:10A82000049066F1DBFFD7F87004642142460368A8
:10A830001B689847F8B1002ED1D0A3682BBB2368C2
:10A8400029462F4A20469B6B93424AD1FFF7F0FBE3
:10A850002C4B06462946D8712046FFF7D9FC034603
:10A8600029462046002B08BF0026D7F075FD304052
:10A870001BB0BDE8F08320464346234A2946D7F063
:10A88000F1FB00201BB0BDE8F08329462046FFF70E
:10A89000A7FA294606462046FFF79CFB97F8653441
:10A8A00006409B07F6B21ED429462046FFF788FCD7
:10A8B000064029462046FFF755FA0640294620461D
:10A8C000FFF7A6FC294606402046D7F06BFD03465D
:10A8D000294620461E40D8F003FC30401BB0BDE89E
:10A8E000F0839847C4E7094A294620464E46D7F0E8
:10A8F000B9FBD9E7E89302201C68170838681708E5
:10A9000039A7000868D00220506817082067170888
:10A91000F8B5124DD5F8703493F8D54074B9104B92
:10A9200007460E461B68986A03685B6B98470446A7
:10A9300070B131463846FFF717FF044695F84034AA
:10A940002046084A64F30413947185F84034F8BD36
:10A95000054A31463846D7F085FBEFE7E8930220F9
:10A9600088CD022068D002205C6817082DE9F041EC
:10A97000554E3378C3B9554F0124D7F8705434700D
:10A9800095F8D5501DB128463370BDE8F081D8F058
:10A99000A7FD054660B94E4A30702846137843F04B
:10A9A00001031370BDE8F08100252846BDE8F08161
:10A9B00082F02EF8214680F0E7FEA7F5C04008F0AF
:10A9C0009DFC444B1C710B246CF050FD6CF052FC50
:10A9D000611E11F0FF04F7D13F4801F0DBFB1CF0D2
:10A9E00047FBD0F80022C7F8982490F87C32DA07A9
:10A9F0004DD59B0757D50021374801F057FC364805
:10AA000017F0C4FD01463548EDF078FA344B354C6B
:10AA100001211B68D86A03681B68984794F82031A5
:10AA2000D7F870046FF3410384F8203103689B6A00
:10AA300098470121D7F87004E8F03EFF81F0E8FF65
:10AA40008046D7F84C0403681B689847A4F58043F8
:10AA50000146404693F8742081F092F8A4F5004036
:10AA600008F03EFC7CF094FD7CF00CF90023337080
:10AA7000F4F0C2FCB7F8423444F84C0C284623F4F6
:10AA8000087343F02003A7F84234BDE8F0811BF0BF
:10AA90002BFD81F0BDFF3C2181F0AAFC07F58B6303
:10AAA00000221A60A7E721460B4806F003FB0E4878
:10AAB000E7F08EF9DFED0D7A07F58B6320EE270ABC
:10AAC00083ED000A97E700BFE5330220E8930220F8
:10AAD00088D0022068D00220E8330220B48F022000
:10AAE00088CD0220E8B3022068B302200AD7233CB5
:10AAF0002DE9F0433E4D87B0D5F8703493F8D5304A
:10AB0000002B55D01AB1232948D0012946D0D8F0BE
:10AB10006FFD044620B90024204607B0BDE8F0834D
:10AB20001CF0A6FA064626F06DFE804630461AF066
:10AB300077FD18B198F92830022B3ED001212D481D
:10AB400008F072FE01212B4808F09AFD0021D5F88B
:10AB50007004E8F0B1FE284849F078FB81F058FF16
:10AB6000002180F011FE254B00211B68D86A036884
:10AB70001B689847D5F84C14214895F84234091AB7
:10AB80003C306FF34513B1FA81F185F8423449093D
:10AB9000F1F0C2FB204607B0BDE8F08395F94034E0
:10ABA000002BB8DAD8F024FD04460028B3D0B7E76C
:10ABB0000124204607B0BDE8F08300274FF00009CC
:10ABC000F9B203AA3046CDF80C9001910137CDF8C7
:10ABD0001090CDF814901BF009FA019910B9032FC9
:10ABE000EED1ABE703AA404626F044F8F7E700BFF2
:10ABF000E8930220E833022074C1022088CD0220AD
:10AC00007CC4022070B52A4E0D46D6F84C042DEDBA
:10AC1000028B036888B0B0EE408A5B6A98470446AE
:10AC200000283CD0D6F8703493F8D540BCB3B4EECD
:10AC3000488AF1EE10FA37D6DFED1E8ADFED1E7A74
:10AC400068EE288A68EEA78AD5ED027A02A82A68FB
:10AC5000F1EE677A6B689FED180A02920393CDEDCF
:10AC6000047A48F04BF9B4EE488A0022B0EE407AFC
:10AC70000123F0EE607A9FED110AF1EE10FA05A9BA
:10AC8000F0EE680A0E488DED057ACDED067A8DED71
:10AC9000071ACDE9002368BF134610F057FF20467E
:10ACA00008B0BDEC028B70BDDFED048ACCE700BFBD
:10ACB000E8930220E02E65420000C8420000000038
:10ACC00098C7022038B50B4D0C46D5F84C040368E4
:10ACD0005B6A984758B1D5F8703493F8D53033B1E2
:10ACE0002146A5F5C040BDE8384000F0FDBB00207E
:10ACF00038BD00BFE89302200148AFF07BB800BF29
:10AD0000C471022000F5C04008B590F84034C3F388
:10AD100040128A4204D061F3451380F8403401B9EF
:10AD200008BD81F075FE0F21BDE8084081F060BBD1
:10AD300070B500F5C046D6F880348B4208D00129A2
:10AD400005460C4626D0022912D011B1C6F880441F
:10AD500070BD81F05DFE1B2181F04AFB46F2D810E8
:10AD6000144A0621284485F0A5FDC6F88044EFE783
:10AD7000012101F09BFA81F04BFE1D2181F038FB8F
:10AD800046F2D8100C4A0621284485F093FDC6F8F7
:10AD90008044DDE781F03CFE1A2181F029FB46F278
:10ADA000D810064A0621284485F084FDC6F8804460
:10ADB000CEE700BFD4681708F4681708E4681708DE
:10ADC00000F5C04210B592F865340C4603F001015D
:10ADD000A14209D064F3000382F86534DB0704D58F
:10ADE00007F0B0FF024B9C7210BD07F0E9FDF9E7D8
:10ADF00068D0022000F5C040044A90F86534117311
:10AE000061F3410380F86534704700BF68D00220C9
:10AE100010B5044690F036FF202192F0ADF904F50C
:10AE2000C043003893F8422418BF012060F3820227
:10AE300083F8422410BD00BF704700BF9FED010A98
:10AE4000704700BF000000000346B6EE061AF4EE9D
:10AE5000000A302093ED4B0A42F022B810B50446A8
:10AE60007CF096FB436F04F5C04204F5E044D2F851
:10AE70007024D360D4F89C2F9366D4F8A42FC2F822
:10AE80000833D4F89C0F03685B6D9847D4F89C0F87
:10AE9000044A03689B6D934200D110BDBDE8104089
:10AEA000184700BF39AE000870B500F5C0452DED5C
:10AEB000028BD5F8703493F8D530002B3AD095F941
:10AEC0004034002B36DB00F50043044693F8B03CD9
:10AED00083BBD5F84C0403685B69984750BB3A4B79
:10AEE000D3F84C0403681B6898470B2822D004F55C
:10AEF000E0469FED367AD6F8A43FD3EDE47AF0EE43
:10AF0000E77AF4EEC77AF1EE10FA13D5D5F87004AB
:10AF1000443084F029FE0346B7EE001A9F20DFED8F
:10AF20002C0A93ED000A41F0BBFFB5EEC00AF1EE2A
:10AF300010FA02DCBDEC028B70BD04F5FF40E6F0B8
:10AF400053FFB0EEC00ADFED237AB4EEE70AF1EE6C
:10AF500010FAEFD5D6F89C0F04F500561E4AD6F825
:10AF6000383607EE903A0368D3F89830B8EEE78A9F
:10AF7000934224D1B0EEC88ADFED187AB4EEE78AA6
:10AF8000F1EE10FAD6D5D6F83C3640F2E63203F2AE
:10AF9000F3139342CED8D5F870049FED110AEAF06E
:10AFA0003BFBD5F8703404F5E4509FED0D0AD3ED6A
:10AFB0000C0ABDEC028BBDE87040C4F015BD98478B
:10AFC00038EE408AD6E700BFE89302200000003444
:10AFD00000000000000070423DAE00080000FA438F
:10AFE0000AD7233C00F5C04370B52DED028B93F8D2
:10AFF000651411F0010504D09FED370ABDEC028BFA
:10B0000070BDB0EE408A044690F03CFE037F002BFA
:10B01000F2D0DFED328A04F58046DFED2F0AB0EE84
:10B02000480AB0EE681A4E2041F03AFF4FF4C87259
:10B030002946B6F9A202B0EE408A41F09DFF0346D0
:10B040002046A6F8A23217F011F8B6F9A23207EEA0
:10B05000100A07EE903AB8EEC77AF8EEE77A77EE84
:10B06000676AB4EEE68AF1EE10FA17D504F5A0444B
:10B07000B4F9983C43BBB6F99A32002BB8BF5B4297
:10B080009BB207EE903AF8EEE77A38EE668A27EE42
:10B09000888A88EE260ABDEC028B70BD77EE877A2F
:10B0A000B4EEE78AF1EE10FAA6DDB6F99A3238EE80
:10B0B000678A78EEE77A07EE103AB8EEC77A27EE9D
:10B0C000088A88EE270A99E7002BB8BF5B429BB23B
:10B0D00007EE903AD7E700BF0000000000007A4476
:10B0E00000F5C0400F4908B5D0F870341A681269ED
:10B0F0008A4214D1B6EE061A3020F4EE000A93ED1F
:10B100004B0A41F0CDFEF6EE007A20EE270AB5EEAE
:10B11000C00AF1EE10FA48BF9FED030A08BD1846B9
:10B120009047F0E749AE00080000000038B504463B
:10B13000B7EE001A7120DFED1A0A04F5E04504F5B8
:10B14000C0442DED028BD5F89C3F93ED370A41F0BA
:10B15000A7FED5F8A43FD4F87024B0EE408A03F5DA
:10B160000574104913681B698B4215D1B6EE061A97
:10B170003020F4EE000A92ED4B0A41F091FE38EED9
:10B18000408A9FED090A204628EE000ABDEC028B9A
:10B19000BDE83840C0F064B810469847EFE700BFFC
:10B1A0000000000049AE000800007A4400F511508C
:10B1B000D2ED007A91ED006AD0ED946AD0ED975A05
:10B1C00027EEA67A65EEE77AA6EE257AE6EE267AEF
:10B1D000C1ED007A82ED007A704700BF00F5A04310
:10B1E000B3F9983C43B900F58040B0F99A020028C1
:10B1F000B8BF404280B2704783EAE370A0EBE370CF
:10B2000080B27047704700BF704700BF704700BFF3
:10B21000704700BF00207047002070470020704733
:10B2200000207047002070470020704700207047C2
:10B230000020704700207047704700BF034644F26B
:10B24000B0201844704700BF0048704720A7170877
:10B2500000F5C040D0F84C0403681B68184700BFD5
:10B2600010B4044C39200C60082110705DF8044BB8
:10B2700019607047A86F170800F5E0409FED0A7A43
:10B28000D0F8B03F0120D3ED0E7AF4EEC77A9FEDEF
:10B29000077AF1EE10FAB8BFD3ED047A67EE877A39
:10B2A000C1ED007A704700BF000000340AD7233C8C
:10B2B00000F5C040DFED047AD0F84C0420EE270AF8
:10B2C00003685B6E184700BF0000C84200F51043DA
:10B2D00093F85D30002B14BF1B200320081AB0FA2E
:10B2E00080F04009704700BF00F5C04090F8650449
:10B2F000C0F38000704700BF00F5C040D0F84C0498
:10B3000003685B6D184700BF00F5C040D0F84C04DF
:10B310000368DB6C184700BF00F5C040D0F84C0450
:10B3200003689B6C184700BF00F5C04248F65053B5
:10B330000344D2F84C04C01AB0FA80F040097047B8
:10B3400000F5C04010B5D0F84C040C460368DB6D26
:10B35000984707EE900A9FED057A0120F8EE677A8C
:10B3600067EE877AC4ED007A10BD00BF0AD7233C90
:10B3700000F5C04010B5D0F84C040C4603689B6D36
:10B38000984707EE900A9FED057A0120F8EEE77ADC
:10B3900067EE877AC4ED007A10BD00BF0AD7233C60
:10B3A00000F5C04010B5D0F84C040C4603681B6E85
:10B3B0009847DFED047A012020EE270A84ED000A89
:10B3C00010BD00BF0AD7233C9DF070BEEDF096B9CA
:10B3D00018F03EB905F0D2BAA4F0D2BF93F0B0BADB
:10B3E0007CF018B83EF028BE80F08ABB20F01ABE70
:10B3F00094F062B88DF010BC8EF07ABA16F072BA82
:10B4000016F04ABF08F098BC18F0B4B807F008BBB3
:10B4100006F0FABF06F0ECBE16F012BCA0F03CB984
:10B42000AEF004B913F0C0BAFFF73EBD16F0A4BBEE
:10B43000D5F0F6B8A9F0B8BA16F06ABE04F07CB937
:10B4400016F01EBB16F098BA90F09EBA6EF07EBC55
:10B4500031F03EB807F0CCBF03F048BC94F03CB8E4
:10B4600016F098BE08F01EBC05F010BE08F0A8BD8E
:10B4700006F082BF08F07CB816F0B4B9FFF7EEBC56
:10B480003FF0CEB900F5E04008B5D0F8B00FE4F0D9
:10B490001BF9012008BD00BF48F6505C844400F54C
:10B4A000C040D0F84C04604501D0002070470AF03D
:10B4B00097BD00BF48F6505300F5C0420344D2F890
:10B4C0004C04984200D070470AF0A8BD012100F555
:10B4D00011501BF091BC00BF07F0E2BC0CF096BE0F
:10B4E0000CF0C6BB0CF04EBB00F5C04330B50446B3
:10B4F000D3F84C0483B00D4603685B6A984760B18B
:10B500000023DFED070A49F2B0302946B0EE600AA9
:10B510001A462044009310F041FC03B030BD00BF38
:10B520000000000000F5C04310B504462DED028B6D
:10B53000D3F84C04B0EE408A03685B6A984720B9A0
:10B5400000242046BDEC028B10BD9FED080A49F295
:10B55000B03028EE000A20440FF0EEF80446002830
:10B56000EED001210248FFF7CDFBEAE70000C84218
:10B57000E833022070B584B005460C46164668468E
:10B5800023F04EFE05F5C0436946D3F84C0403682A
:10B590005B6D98476946204624F07CFD10B9002079
:10B5A00004B070BD6946204624F082FD0028F6D024
:10B5B000204623F08BFE0446304623F087FE84426B
:10B5C000EDD12B68314628461B6A984704B070BD00
:10B5D0002DE9F0431F4600F5C04304460D461646CC
:10B5E0002DED028BD3F84C0487B0B0EE408A03688F
:10B5F000F0EE608A9DF840805B6A9DF84490984721
:10B6000018B39FED140A49F2B030CDF804903B46D0
:10B61000D5ED006A68EE800A95ED017A2044D5EDFB
:10B62000027A66EE806A27EE007A324667EEC07ACA
:10B6300003A928EE000ACDF80080CDED036A8DED58
:10B64000047ACDED057A10F099FA07B0BDEC028BC3
:10B65000BDE8F0830000C84200F5C04370B5044661
:10B66000D3F84C048EB00E46036815465B6A9847C3
:10B67000D8B3DFED1F7A0020D6ED004A0BAB96ED74
:10B68000015A08AAD6ED025A64EEA74A95ED006A5F
:10B6900025EE275AD5ED016A65EEE75A95ED027A57
:10B6A00026EE276ADFED130A66EEA76A009067EEC2
:10B6B000677AB0EE600A05A9CDED054A8DED065A10
:10B6C000CDED075A8DED086ACDED096ACDED0A7A08
:10B6D000CDED0B0ACDED0C0ACDED0D0ACDE9010043
:10B6E00049F2B030204410F09DFC0EB070BD00BF98
:10B6F0000000C842000000002DE9F0471D4600F59B
:10B70000C04304468A4616462DED028BD3F84C04FE
:10B710008EB0F0EE408A0368B0EE608A9DF86070EB
:10B720005B6A9DF864809DF868909847002846D031
:10B730009FED250A49F2B0300BAB08AA68EE000A6B
:10B74000204405A9CDE901899AED003ADAED013AE4
:10B750009AED024A23EE003AD6ED004A63EE803AB3
:10B7600096ED015A24EE404AD6ED025A64EE804A24
:10B7700095ED006A25EE005AD5ED016A65EEC05AD6
:10B7800095ED027A26EE006A66EE806A009727EE53
:10B79000407A8DED053A28EE800ACDED063A8DED22
:10B7A000074ACDED084A8DED095ACDED0A5A8DEDC7
:10B7B0000B6ACDED0C6A8DED0D7A10F033FC0EB0F6
:10B7C000BDEC028BBDE8F0870000C84200F5C04325
:10B7D00070B50546D3F84C0486B00E4603685B6A24
:10B7E0009847044610B39FED136A0023D6ED006A14
:10B7F000012196ED017A49F2B030D6ED027A66EE7B
:10B80000866A27EE067ADFED0C0A67EEC67A0191AA
:10B81000B0EE600A1A46284403A90093CDED036AEE
:10B820008DED047ACDED057A10F090F9204606B042
:10B8300070BD00BF0000C842000000002DE9F047C5
:10B84000984600F5C04305460F4616462DED028B7F
:10B85000D3F84C048AB0B0EE408A0368F0EE608AF8
:10B860009DF850905B6A9DF854A098470446A8B391
:10B870009FED1D0A012149F2B030434668EE800A6F
:10B8800007AA2844CDE9009AD7ED004A97ED015A5E
:10B89000D7ED025A64EE804A96ED006A25EE005A12
:10B8A000D6ED016A65EEC05A96ED027A26EE006A80
:10B8B00066EE806A029127EE407A04A928EE000A1B
:10B8C000CDED044A8DED055ACDED065A8DED076A92
:10B8D000CDED086A8DED097A10F0C2F820460AB065
:10B8E000BDEC028BBDE8F0870000C84200F5C04304
:10B8F00070B505462DED048BD3F84C0488B0F0EEFE
:10B90000409A0368F0EE608AB0EE419A5B6AB0EE4E
:10B91000618A9847044600B3DFED120A00264FF013
:10B920007E5304A829EEA00A079629EE201A049354
:10B9300068EEA00A0696059645F0AEFC9FED0A0A51
:10B9400049F2B030002304A928EE000A284401AAD5
:10B950000196029603960FF0F9F9204608B0BDEC67
:10B96000048B70BD35FA8E3C0000C84200F5C04320
:10B9700030B505462DED048BD3F84C0489B0F0EEBC
:10B98000409A0368B0EE609AF0EE418A5B6AB0EECE
:10B99000618A98470446F0B100234FF07E5204A814
:10B9A000049207930693059345F0F0FE9FED0C0A71
:10B9B00001A8CDED019A8DED029ACDED038A47F0F5
:10B9C000F1FA49F2B030B0EE480A012301AA04A905
:10B9D00028440FF0BBF9204609B0BDEC048B30BD04
:10B9E00035FA8E3C0A4B93F940240B46002A09DBBA
:10B9F00000F5E040D0F89C2F783207CA83E80700B2
:10BA000001207047002201208A604A600A60704766
:10BA1000E8930220F8B54D4A00F500430546026060
:10BA200093F8342C42B9D3F8304C2CB120463CF07A
:10BA3000E7FA204624F062FC05F5C043444AD3F8F7
:10BA4000D403C3F8D82108B124F05CFC414B43F681
:10BA50005C502B60284423F05FFB05F5405393F8BE
:10BA6000982742B9D3F894472CB120463CF0C8FA45
:10BA7000204624F043FC42F2103041F69C6441F62B
:10BA8000846628442C442E44D3F018F814F8043C5F
:10BA9000083C3BB92768384627B13CF0B1FA384634
:10BAA00024F02CFCB442F1D141F6883041F24474C8
:10BAB00041F2E46628442C442E4493F0B7FB204620
:10BAC000183C3BF035FDA642F9D141F2701441F229
:10BAD0002817214B2C442F44C5F8483C14F8043C4B
:10BAE000083C3BB92668304626B13CF089FA30461E
:10BAF00024F004FCBC42F1D105F60C6083F0F0FCAC
:10BB000005F55E6083F0ECFC05F6B45083F0E8FCCC
:10BB100005F6085083F0E4FC05F6DC4083F0E0FC19
:10BB200005F54B6083F0DCFC0C4A95F8D031C5F884
:10BB3000BC2043B9D5F8CC412CB120463CF060FA8A
:10BB4000204624F0DBFB2846F8BD00BF2C74170804
:10BB500008E31808C8BD18086C5F180848C11A081F
:10BB600010B5044607F0A4FD204616F03BFD204624
:10BB700005F066F82046BDE8104005F0F5B900BFB5
:10BB800010B516F0E1F990F07DF80368BDE81040BB
:10BB90005B68184710B5044607F096FA204607F090
:10BBA00031F8204607F0E6FA204617F077FD2046E8
:10BBB000BDE8104004F01EBEF8B56F4B05460027E7
:10BBC00044F2840440F8043B44F204269DF0C2FB96
:10BBD00005F110001FF088FD05F17000D7F078FD29
:10BBE00005F518707BF0F8F905F546702EF076FD36
:10BBF00005F5EC601DF04CFE05F6FC0024F0DAFBC8
:10BC000005F648403DF010FF41F2D8602C442E4428
:10BC100028449DF021F941F2A870284473F0E2FF16
:10BC200041F6582028447FF0C5FC41F66C3028448A
:10BC3000ACF0A8FE41F68830284493F0DFFA41F6D4
:10BC4000C430284422F070FB05F5E450C2F066FDD4
:10BC500042F210302844D2F01DFF42F22C3028442A
:10BC60007BF0C8FD42F29C3028449EF0D5FF05F5DC
:10BC7000005342F2F030414A83F8E07342F2E0337D
:10BC800028442B4413606BF049F8394605F51150F0
:10BC900019F056F842F638302844A4F081FB42F6F9
:10BCA00068302844C1F0ACFC43F274502844CAF018
:10BCB000EFFC43F28C602844C9F0A8F943F2B46069
:10BCC0002844CDF035F905F55D50D1F063FE43F21F
:10BCD000A4702844D2F0E6FB43F2FC702844BFF085
:10BCE0004FFD43F6A400284418F03AF843F610201C
:10BCF0002844C2F05FFA43F668202844D4F000FAE2
:10BD000043F6BC501E49284471F050FB43F6D45012
:10BD10002844D9F089FD43F6DC502844ADF0ACFD51
:10BD200043F698602844D4F09BF843F6F06028442A
:10BD3000F3F082FB05F5804383F8747020460C34E1
:10BD400083F00EFFB442F9D144F210200D4C284488
:10BD5000D4F0E0F844F23420284483F0BBF923689F
:10BD600033B92846084971F021FB28462560F8BD03
:10BD70000648F3F00FFB00BFC8BD180864DC0220C2
:10BD8000405D1A0884D1022030BC180808691708E1
:10BD900070B546F29C450446054428461FF01AFA41
:10BDA00025F030FD90F9253093B390F844337BB300
:10BDB00004F5C04304F6FC06D3F87004443083F065
:10BDC000D3FE0346B7EE001A9F20DFED120A93ED73
:10BDD000000A41F065F894F9343928460021012B16
:10BDE00004F6583408BF86ED0F0A1EF0CFFF9FED12
:10BDF0000A7ADFED0A7A304620EE070A94ED287AB7
:10BE0000A7EE270A84ED280ABDE8704025F078B92E
:10BE100070BD00BF00000000CDCCCC3D6666663F23
:10BE2000FFF7B6BF10B50121044616F021FC30B172
:10BE3000124BD3F84C0403689B6A9847B8B14FF48F
:10BE40000011204616F014FC60B94FF48021204602
:10BE500016F00EFC00B910BD40F0A0FABDE810408D
:10BE60003DF0CEB840F09AFA3DF0FAF9EDE7204601
:10BE700002F038FE204602F045FEE0E7E89302209B
:10BE8000FFF7D0BF70B500F5E045044684B09FEDE4
:10BE90006F0AD5F89C0F6C3047F030F801A904F513
:10BEA00011508DED010ACDED020A8DED031A18F047
:10BEB00009FE0221204616F0DBFB002874D1012187
:10BEC000204616F0D5FB40B9614BD3F84C0403680B
:10BED0009B6A9847002800F0AC800121204616F0AC
:10BEE000C7FB00285CD04FF40031204616F0C0FBA1
:10BEF00030B104F5C043D3F8700403685B6C984715
:10BF00004021204616F0B4FB00286ED14FF480612A
:10BF1000204616F0ADFB002861D12021204616F006
:10BF2000A7FB58B104F5C046D6F84C0403681B695A
:10BF3000984740B3D5F8A40FE0F0AEFF802120462B
:10BF400016F096FB30B94FF48021204616F090FB96
:10BF5000002872D040F022FA3DF078F810212046F7
:10BF600016F086FB002855D14FF6FF71204616F0DB
:10BF70007FFB002848D14FF40041204616F078FBA3
:10BF800028BB04B070BD204610F058FA0028D1D16B
:10BF9000D6F84C0403685B6998470028CAD0CDE7FF
:10BFA000204602F009FE9EE70121204616F060FBC4
:10BFB000002884D1264BD3F84C0403689B6A984729
:10BFC00000287FF47CAF204602F08CFD77E748F232
:10BFD0003C00204404B0BDE8704093F057BE41F6E9
:10BFE000582020447EF0EAFD97E741F658263019A4
:10BFF0007EF038FD04F5805393F9883B002B85D003
:10C0000030197EF013FF81E745F67C402044ECF0C8
:10C010007FFBB0E7D5F89C0FDCF006FB44F2DC3088
:10C020002044A8F0A1FE44F220302044D4F01CFBB0
:10C030009AE7204602F066FD4FE74FF400212046C4
:10C0400016F016FB002885D188E700BFE02E654278
:10C05000E8930220FFF716BF10B50121044616F041
:10C0600007FB58B98021204616F002FB78B94FF43F
:10C070000011204616F0FCFAD8B910BD204602F097
:10C080009BFD8021204616F0F3FA0028EFD04FF4F4
:10C090008021204616F0ECFA0028E8D140F07EF925
:10C0A0003CF0AEFF4FF40011204616F0E1FA0028F4
:10C0B000E3D004F5E450BDE81040C3F0EBBD00BF91
:10C0C000FFF7CABF70B504464FF6FF7116F0D0FAFD
:10C0D00004F5C04580BBD5F8703493F8D530BBB3B8
:10C0E00092F072F804F5E04691F070FA204617F0ED
:10C0F000C7FA95F8403404F50044224ADB43C3F301
:10C10000C01384F8CD3BD6F89C5F53712B681C6F2D
:10C110007BF03EFA7AF0C2FE1B4B9C4225D1D6F84A
:10C12000A44F7BF035FA7AF0B9FE04F50574204689
:10C13000BDE87040BEF042BE07212046D5F840243D
:10C1400002F070FDD5F8703493F8D530002BC7D1CC
:10C150002046FEF75DFED5F870040C4A03681B6AA2
:10C16000934205D1E9F01AFABAE72846A047D6E784
:10C1700004F5804191F8B62291F8841D9847D5F8CE
:10C180007004EFE768D0022009B2000805B2000889
:10C19000FFF798BF2DE9F04100F5115300F5C044B9
:10C1A00000F500580546D3F8502204F2844704F500
:10C1B000916644F250603A60D3F85C323360D8F84C
:10C1C0004036184440F01AFEC4F88C0404F592631B
:10C1D0003A6804F294444FF6FF711A6028463368B7
:10C1E000236016F045FA08B9BDE8F081D8F840267A
:10C1F00028460921BDE8F04102F0E6BC00F5C04345
:10C20000D3F8801400294AD093F8412412F0010F8A
:10C2100045D06FF30002012983F8412400F5A042C4
:10C22000D2F8CC1FB1F908C007EE10CAB8EEC77A31
:10C2300036D003F5926C03F2944393ED006A00F557
:10C240001150D2F8D03FDCED005AB3F9083007EEB8
:10C25000903AF8EEE77A66EE676A65EEA77AE7EE5F
:10C26000256AE7EE067A90ED977A90ED946A27EECC
:10C27000877AA6EE867ABDEEC77A17EE103A0B8162
:10C2800090ED946A90ED977A67EE867AD2F8D03F77
:10C29000E6EEC77AFDEEE77A17EE902A1A8170472C
:10C2A00003F2844C03F59163C7E700BF38B5044639
:10C2B00000F5C0452DED028B59B9D5F88034022B1D
:10C2C00002D0BDEC028B38BD15F05AFCB0F57A7F78
:10C2D000F7D3204615F078FCD5F88C3440F2E632DE
:10C2E0001B1A03F2F3139342EBD944F25063174A3B
:10C2F000C5F88C04034482FB0312DB17C3EB621303
:10C3000006EE903A9FED0F7BB8EEE60B20EE070BA2
:10C31000B7EEC08BB0EE480A61F1EAFAF0EE407A6F
:10C3200005F5926305F29445B0EE480AC3ED007A34
:10C3300062F17AF985ED000ABDEC028B38BD00BFD1
:10C34000AFF30080000000A046DF913F1F85EB5156
:10C3500010B5044615F090FE1021204616F088F91D
:10C3600000B910BD204602F0F3FA4FF40011204648
:10C3700016F07EF90028F4D140F010F83CF070FF80
:10C3800004F5E450BDE81040C3F084BCFFF7E0BF03
:10C390002DE9F04F89B00446FFF70EFCDC4B44F268
:10C3A000D82045F6E87623604FF07C572044264499
:10C3B00002F00CFE44F2A42304F5A04205A9234494
:10C3C00006F10800059746F23005C2F8E03F062363
:10C3D000254404F5FF4882F8E43F4FF0010B83F059
:10C3E000D5FC06F12000F2F065F80023049704F56F
:10C3F000C04704A905F1080087F820301923C7F8C1
:10C4000028800DF1180987F82C3046F2D81A83F0ED
:10C41000BDFC05F1200046F2F005F2F04BF81823C0
:10C4200046F288002544C7F8708087F874302044AD
:10C4300087F868B0A24492F037F82846D5F052F950
:10C44000B44B4946281DC7F8F03046F208258DF850
:10C4500018B072F0C5FE46F25010AF4E254420448D
:10C460006DF0FEFB46F290102044D3F05FFEAB4B24
:10C4700046F2A8104946C7F890312044069683F04A
:10C4800085FC46F2B41049460696204483F07EFCB3
:10C4900046F2C01049460696204446F2A82683F08C
:10C4A00075FC9F4B0AF10C002644C7F8D831F2F016
:10C4B00001F8284614358AF009FCB542F9D11E234B
:10C4C00040F2CC60C7F8D8330023A7F8DC3323F060
:10C4D0000FFFC7F8D40346F2E0302044F1F0EAFF42
:10C4E00046F224402044F1F0E5FF8E4B1A68002A02
:10C4F00000F0638249F29C568B4B46F250404FF05D
:10C500007E552644C7F8D8312044C7F84C64D7F08C
:10C51000B1F807F2844346F29C4007F592671D602C
:10C520004FF40071814B20443D6004F500470793B0
:10C530007F4B0694009399E80C001EF0AFF946F685
:10C5400034202044B5F070F947F6507003A90395E4
:10C55000204483F045FC47F6647003A9039520440A
:10C5600083F014FC47F67070204422F059FE04F565
:10C57000E042002347F6BC7002F68C71C8F8003028
:10C580002044C8F80430C8F8083048F24C180B6052
:10C590004B60A0448B6004F511534FF40041C2F886
:10C5A000983F002382F8B93F1FF0D8F948F23C00C9
:10C5B000204492F069FF48F2C0002044B0F0B8FA7D
:10C5C00048F2FC00204472F03BFF5A4B48F2101036
:10C5D000C7F8FC302044ACF0CFFF48F22C10564B8B
:10C5E00020445649186070F0E1FEFF23544940464C
:10C5F00087F85C3187F8643170F0D8FE514B1D68C4
:10C60000002D40F0E08148F26C10C3F8008048F63D
:10C61000103820447CF0AAFC48F61420A0442044A2
:10C62000E1F08EFE48F608302044E1F073FC40460D
:10C63000BDF070FC48F6404041462044EAF08EF8D8
:10C64000414B424948F6A040C7F8403C06232044ED
:10C6500087F8943C3E4B19600B7C4BB12B46013361
:10C660009BB203EB830201EB8202127C002AF6D11B
:10C670003849394A0B80D2F8009038490B80B9F11B
:10C68000000F40F09D81106048F6B440344B03A980
:10C69000204448F65058039383F078FB48F6D44082
:10C6A000A0444FF6FF7A4FF0FF3B204404F51045BD
:10C6B00007F086FB2B4B48F61450C7F8D43C2044B7
:10C6C00007F07EFB284B4046C7F8143D07F078FB87
:10C6D000264B48F6D050C7F8A88DC7F8503D244BDC
:10C6E0002044C7F8B08DC7F8AC3D224BC7F8B88DD1
:10C6F00008F13C08C7F8B43D1F4BC7F8BC3D22F019
:10C700008FFD48F6EC50204422F08AFD36E000BF51
:10C710002C7417087C6817080000A040C068170830
:10C7200008E31808FCD5022010751708D9B40008D2
:10C730001C741708D068170870DC0220C80C190890
:10C74000785B1A0830DD022018D01708A8C5170832
:10C7500040D102203CD10220E4D0022014D102209A
:10C76000CDCC4C3D5CD5170804D617087CD91708EA
:10C77000DDB40008E1B40008E5B4000848F608603C
:10C78000204422F04DFD914B48F62460A7F820AEDE
:10C79000C7F81C3E204422F043FD8D4B8D49404696
:10C7A000C7F8D4BFC3F8008070F000FE48F6E87008
:10C7B000A7F8C8BDA7F8E4AD0027204449F25058B7
:10C7C00022F02EFD49F20400A0444FF0010A20445B
:10C7D000DFF850B222F024FD49F22000204422F07C
:10C7E0001FFD49F2940085F834902044C5F8589014
:10C7F00007F0E6FA784B49F2D000C5F894302044AF
:10C80000EEF0A2F8754B49F25420C5F8D030204420
:10C8100007F0D6FA724B49F29820C5F854322044FA
:10C8200007F0CEFA6F4B49F2D82085F8D492C5F8BC
:10C830009832204407F0C4FA6B4B49F21430C5F823
:10C84000D832204407F0BCFA684B49F26830C5F88A
:10C850005073C5F814332044C5F85473C5F85873A1
:10C8600007F0AEFA624B49F2B030C5F8A493C5F8B0
:10C870006833204407F0A4FA5E4B49F2F430C5F85F
:10C88000EC93C5F8B033204407F09AFA5A4B49F2BA
:10C890003C40C5F8F433204407F092FA574B49F274
:10C8A0007C40C5F83C34204407F08AFA544A05F22B
:10C8B000F44349F21050C5F87C2420441F605F60A7
:10C8C00007F07EFA4046A5F84CA5C5F810B522F051
:10C8D000A7FC08F1100022F0A3FC08F1200022F0D0
:10C8E0009FFC08F1300022F09BFC304607F068FA0C
:10C8F000444B49F2D85049F2AC76C5F89C352044F7
:10C90000264412F02BFA49F29460204407F058FABA
:10C910003D4B49F2D860C5F8D096C5F8943620440E
:10C9200007F04EFA394B49F22870A5F81497C5F86C
:10C93000D836204407F044FA354B49F26C70C5F8FC
:10C940006497C5F82837204407F03AFA3046C5F80E
:10C950006CB7A5F8A8A722F063FC06F1100022F03E
:10C960005FFC06F1200022F05BFC06F1300022F0B3
:10C9700057FC05F2FC73274A49F6080085F8F5A72D
:10C98000C5F86C2720441F605F609F600CF044FF77
:10C9900049F6DC00204413F00DFE49F65410204403
:10C9A00007F00EFA05F694131B4A2046C5F85429E1
:10C9B0001F605F6009B0BDE8F08FC3F800A099E583
:10C9C0001648F2F0E7FC1648F2F0E4FC0000FFFF26
:10C9D00034D002201071180824DA1708B8DA1708C2
:10C9E0001CDC1708C0DC170864DD170800DE170818
:10C9F00050E01708F4E017083CE21708E0E21708D7
:10CA000084E3170868E6170878DB1708B0EA170808
:10CA1000A0E11708C0E5170878EB17084069170868
:10CA20001C69170804E5170838B5054C0A46054B7C
:10CA300001462468256820462C68A047002038BDA0
:10CA400088CD0220E833022010B5084CF2F088F8B7
:10CA5000074B024620461A60FFF79AFC2046054A1B
:10CA60000549BDE8104060F13DBF00BFE83302203A
:10CA700088CD0220B07F032015BA0008012070473E
:10CA800090F8D0308B4204D900EB8100D0F8D4006C
:10CA900070470020704700BF90F8D0308B4204D917
:10CAA00000EB8100D0F8D40070470020704700BF31
:10CAB000FA207047014B93F866027047E873022032
:10CAC000044BD3F88004A0F10100B0FA80F04009D3
:10CAD000704700BFE8930220044BD3F88004A0F114
:10CAE0000200B0FA80F04009704700BFE8930220CE
:10CAF000034BD3F8700408B1E6F044BF0148704717
:10CB0000E8930220FC74170838B5D0E90912C36A0B
:10CB10000446544D41F4E05043F4E05342F4E052F3
:10CB20006062C4E90A23D5F8A43FABB141F4F841EF
:10CB30006162D5F8A40FDFF0EFF938B1D4E90A2328
:10CB400042F4804243F48043C4E90A23D5F8A40F99
:10CB5000DFF022FD002871D14348A8F085F818B114
:10CB6000636A43F0806363623F48A8F0A5F818B198
:10CB7000A36A43F08063A3623B48A8F0A3F818B906
:10CB8000E36A43F08063E362384B1D68002D5ED09A
:10CB90001921284673F05EFE18B1636A43F480736E
:10CBA0006362334B93F8E83F002B37D1A36A3149D6
:10CBB00091F9142AF2B9626A91F8101A013901291F
:10CBC00007D8E16A42F4800243F4800341F4800113
:10CBD000E16243F0804342F080422749C4E90923DF
:10CBE000D1F8703493F8C1301BB9E36A43F0804345
:10CBF000E36238BD626A43F0800342F08002C4E918
:10CC0000092391F9140A0028D6D091F8FC0A0028CB
:10CC1000D2D0E06A40F08000E062CDE7A36A19213B
:10CC2000284643F48073A36273F066FE0028BDD0EB
:10CC3000D4E90A3242F48072E262B8E7D4E90A2306
:10CC400042F4005243F40053C4E90A2384E7084B3A
:10CC500093F8E83F002BA9D0A36A43F48073A36242
:10CC6000A5E700BFE8A30220C47702204CD1022030
:10CC7000E8830220E8B30220E893022070B54FF465
:10CC800044700D46164623F02DFB044628B132466B
:10CC9000294687F0A3FA024B2360204670BD00BFEF
:10CCA0007077170800207047704700BF0320704757
:10CCB00008207047014B93F868027047E873022020
:10CCC000034B93F9780D003818BF0120704700BF5F
:10CCD000E8730220014B93F96A027047E87302205F
:10CCE000704700BF08B50C4BD3F8A40F10B1DFF0AC
:10CCF00013F968B950201022084BD3F8703423B1CF
:10CD000093F8D5300BB142F0C00040F0010008BDEF
:10CD100058201822F0E700BFE8A30220E893022081
:10CD200000B5002389B002930393049305930693FF
:10CD300007931AF09DF902A91AF036F910B909B053
:10CD40005DF804FB1AF094F900F55A7005AB07C8BA
:10CD500083E80700184646F075FDF1EE047A20EEF0
:10CD6000270AFCEEC07ACDED017A9DF8040009B0E7
:10CD70005DF804FB10B5194C84B094F8FA1904F668
:10CD8000A40017F01FFC30B194F8FA1904F6A400BF
:10CD900017F02EFCC8B900230193029303931AF0F5
:10CDA00067F901A91AF000F950B92FF0B9FCB022C7
:10CDB00090F80C3302FB030090ED410A04B010BD63
:10CDC00001A846F03FFD04B010BD94F8FA1904F62E
:10CDD000A40004B0BDE8104017F0A8BDE86302202D
:10CDE00008B50D4BD3F87004A8B1443082F0BCFEF6
:10CDF0000346B7EE001A9F2093ED000ADFED070A05
:10CE000040F04EF8DFED067A20EE270ABDEEC00AAC
:10CE100010EE103A18B208BDE8930220000000009E
:10CE20000000C8422DE9F04F354C8DB0354E4FF023
:10CE3000010B0546E71C06F54059B6F9C0320BF167
:10CE4000FF3A43FA0AF3DB0733D5287C84F03AFF34
:10CE50008046287C85F066FF00F12103984548D381
:10CE6000BAF1030F25D8DFE80AF03C342C02D9F8D8
:10CE7000A43F03F52D7359681A680491D968586A5C
:10CE800006911969039221220791996905915969BF
:10CE90001B6A08916221009203AA0191C221CDF878
:10CEA0002500CDF829301923287C8DF824B084F092
:10CEB00089FFA74202D014F801BBBEE70DB0BDE860
:10CEC000F08FD9F89C0F03681B69984700F1A00305
:10CED000D1E7D9F89C0F0368DB68984700F1A003FD
:10CEE000C9E7D9F89C0F03689B68984700F1A00335
:10CEF000C1E7287C0DB0BDE8F04F83F0B3BF00BFA1
:10CF000061781708E873022010B50446EBF010FCB6
:10CF100020B12146BDE81040EBF0CCBB10BD00BFF6
:10CF200038B5044606480D460AF064FD28B929467E
:10CF30002046BDE8384086F0A3B9042038BD00BFC4
:10CF400038C10220014809F0ADBB00BF38C1022042
:10CF50000E4B30B5D3F87C3D83B004460D46DB075D
:10CF60000CD411460A480192ECF05AFB019A29466A
:10CF7000204603B0BDE830408CF01EBB114605488A
:10CF80000192EAF005F8019AEBE700BFE87302208E
:10CF90008890022028C0022010B588B0044687F08F
:10CFA000FDFF0C4BD3F8700458B169461E22E6F021
:10CFB00045FC6B46084A0621204687F0D7FF08B09B
:10CFC00010BD064A0621204608B0BDE8104087F093
:10CFD000CDBF00BFE893022010B31A0848751708A8
:10CFE000034A92F8C83F013382F8C83F86F058BB25
:10CFF000E88302200148E1F0FDBB00BFFCBD022038
:10D0000000B583B00846019123F092F838B1019938
:10D01000054803F0BDF9002003B05DF804FB0420CF
:10D0200003B05DF804FB00BF94CD022070B58B8B7C
:10D0300082B00C460546CD2B06D02146284602B0CC
:10D04000BDE8704086F0CCBBD1ED067AFCEEE77A05
:10D05000CDED017A9DF80430022BEED10D4E0192F8
:10D0600096F8B51006F13C0092F050FA019A0028AB
:10D07000E3D096F8B51006F13C0092F051FA019A0F
:10D080000028DAD194ED020A034803F061F9019A0D
:10D09000D3E700BFE8B3022094CD0220542A18BF82
:10D0A000162A0CBF0123002303D1032218460A705D
:10D0B000704786F001B900BF70B50C464B7A897A8B
:10D0C0000546E27A43EA012343EA02439D2B05D059
:10D0D00021462846BDE8704086F040BA124E96F8C8
:10D0E000B51006F13C0092F011FA0028F0D096F845
:10D0F000B51006F13C0092F01FFA0228E8D196F82C
:10D10000B51006F13C0092F00BFA0028E0D1D4ED06
:10D11000057A9FED060AF8EEE77A054827EE800AC1
:10D1200003F016F9D4E700BFE8B302200AD7233C86
:10D1300094CD0220074A40F6CD1310B540F6CD3409
:10D1400092F96C21002A08BF1C4686F05FFA204342
:10D1500010BD00BFE8B3022010B584B019F088FFFD
:10D160000446684622F05CF86946204619F004FF40
:10D170000E4B93F8410410F0200014D003F58053B7
:10D18000DDED017A9FED0A7AD3F8A43FF8EEE77A55
:10D19000D3ED0F6A77EEA67A67EE877AFDEEE77A2F
:10D1A00017EE903A18B204B010BD00BFE893022009
:10D1B0000AD7233C10B5044623F0A0F8204610BD42
:10D1C00010B50C4C94F94034002B0FDBD4F84C0410
:10D1D0000368DB6C984758B9D4F84C0403689B6C1F
:10D1E000984700280CBF0220032010BD012010BD6D
:10D1F000042010BDE893022008B5134B93F84104B6
:10D2000010F020001CD0D3F84C040368DB6D984765
:10D2100007EE100ADFED0D6AB8EE477ADFED0C7A03
:10D2200027EE267AB4EEE77AF1EE10FA09D5F2EE9F
:10D23000046AC7EE267AFCEEE77A17EE903A98B2C7
:10D2400008BD41F6991008BDE89302200AD7233C97
:10D2500000FF7F4710B44C69012C03D05DF8044BEC
:10D2600086F038BA01465DF8044B014803F064BF0C
:10D27000E8330220B1F90430002B3EDB9FED1F0A9A
:10D280004FF47A732DE9F041DFF8788082B00027FF
:10D290000C461546009201970646B1F90220D8F8CF
:10D2A000CC1F8CF065FC0123D8F8D01F30460193C9
:10D2B0004FF47A7300959FED110AB4F900208CF0B9
:10D2C00057FC3B46D8F8D41F30469FED0D0ACDE9F8
:10D2D0000057B4F904208CF04BFCB4F906209FED04
:10D2E000070A3046D8F8D81F4FF47A730197009593
:10D2F0008CF03EFC02B0BDE8F08170470000FA44BB
:10D3000000007A44E883022008B50A4B93F84104F0
:10D3100010F020000DD0D3F84C0403689B6D9847A3
:10D320003FF06CFD044B83FB0023C017C0EBA31040
:10D33000C0B208BDE89302201F85EB51044B18785A
:10D3400020B9044B93F84204C0F38010704700BF2B
:10D3500020CF0220E893022000B5002387B003937A
:10D360000493059319F084FE03A919F01DFE10B96A
:10D3700007B05DF804FB19F07BFED0EDDA0A90ED02
:10D38000DB0AF1EE600AB1EE400A61F149FBDFED24
:10D39000097A20EE270A3FF0F3FCF6EE007A20EE41
:10D3A000270AFCEEC07ACDED017A9DF8040007B0A3
:10D3B0005DF804FBE02E6542144B93F8410410F035
:10D3C000200000D1704703F5805300B5D3F8A40FB7
:10D3D00083B000F5657046F035FA9FED0D7ADFED0C
:10D3E0000D7A20EE070AB4EEE70AF1EE10FA03D444
:10D3F000FF2003B05DF804FBFCEEC07ACDED017AAE
:10D400009DF8040003B05DF804FB00BFE893022020
:10D41000CDCC4C3D00007F430B4B93F8312A7AB9B9
:10D4200093F8652492060BD193F94024002A09DB76
:10D4300093F8413413F0200F14BF042001207047EB
:10D440000520704703207047E893022030B52DED8A
:10D45000028B89B0054619F00BFE00F55A7002AC3C
:10D460002D7C07C884E80700DDED020A9DED030A64
:10D47000F1EE600AB1EE400A61F1D2FA2046B0EE58
:10D48000408A46F0DFF9DFED0B7A0C230499012284
:10D4900028EE278A28460791A8218DED060A8DEDF2
:10D4A000058ACDE9003205AA84F08CFC09B0BDECF8
:10D4B000028B30BDE02E654208B5074B93F9B432BC
:10D4C000032B03D0BDE8084087F0F4BD034A0221D6
:10D4D00087F04CFD042008BDE87302206075170832
:10D4E000094BD3F87C2D92070CD503F54053DFEDA3
:10D4F000077A03F6747393ED000AB8EEC00A20EEC3
:10D50000270A704785F0CCBEE87302200AD7233C77
:10D5100030B595B0044603A821F082FE1E4B03A946
:10D52000D3F84C0403685B6D984708B915B030BD5B
:10D53000002103A821F07EFF0028F7D0257CF1F020
:10D540005BFFDDED047A9621059C0022F8EEE77A78
:10D550009FED127A01914FF6F8510894002467EE7E
:10D56000877A3323079028460B920C920D920E92E5
:10D570000F9210921192129207AAADF84C105721F7
:10D580008DF84E40069C0093CDED0A7A099484F004
:10D5900019FC15B030BD00BFE89302200AD7233C28
:10D5A000F0B5884C05462DED0A8BD4F84C3499B073
:10D5B0001A681846536A9847002864D004F5405406
:10D5C000D4F8EC33062B00F2E880DFE803F0040423
:10D5D0000460A3C95C007C480BAC0EF043FE03461C
:10D5E0009FED7A8A20469FED7A0A40F6F8579FED24
:10D5F000799AF0EE489AF0EE48AAF0EE498AF0EEF9
:10D6000048BA93ED025B93ED046B93ED007BB7EEAC
:10D61000C55BB7EEC66BB7EEC77B8DED0C5A8DEDD3
:10D620000D6A8DED0B7A45F069FCB0EE40CAB0EEA4
:10D6300060BAB1EE41AA2E7CF1F0DEFE8C22002110
:10D640003323054601922246012415911691304656
:10D6500055210093ADF85C700B958DED0CCA8DEDE6
:10D660000DBA8DED0EAACDED0FBACDED10AACDED10
:10D67000118ACDED129A8DED138A8DED149A8DF8E5
:10D680005E4084F09FFB19B0BDEC0A8BF0BD4E48A4
:10D690000BAC0EF0E7FD03469FED4D0A20464FF41C
:10D6A000406793ED025B93ED046B93ED007BB7EE67
:10D6B000C55BB7EEC66BB7EEC77B8DED0C5A8DED33
:10D6C0000D6A8DED0B7A45F019FC3F48B0EE41AA8A
:10D6D000B0EE60BAB0EE40CA0EF0C8FD9FED3C0A55
:10D6E000B1EE4AAA45F00AFC3748F0EE418AF0EE66
:10D6F00040BAF0EE60AA0EF0BDFD9FED350AF1EEE6
:10D70000688A45F0FBFBB1EE419AF0EE409AB0EE2C
:10D71000608A90E72C4840F607470EF0A7FD9FED82
:10D720002C0A45F0EBFB2848F0EE418A9FED27BA22
:10D73000F0EE40BA9FED27AAF0EE60AA0EF09AFD37
:10D740009FED230AF1EE688A45F0D8FBB0EE4BCA94
:10D75000F0EE409A0BACB1EE419AB0EE608A6AE707
:10D76000194840F63F470EF085FDDFED18AA9FED02
:10D77000180A0BACDFED178A45F0C0FBF0EE6ABA71
:10D78000B0EE68AAF0EE409AB0EE608AB1EE419A2F
:10D79000B0EE6ABAB0EE6ACA4DE79FED0C8A002778
:10D7A0009FED0C9A0BACF0EE489AF0EE498AB0EE81
:10D7B00049AAF0EE48AAF0EE48BAB0EE48BAB0EE88
:10D7C00048CA38E7E893022098C70220000000000A
:10D7D0000AD7233C000000802DE9F043404D2DED99
:10D7E000048B95F841348DB09B0604D40DB0BDEC8C
:10D7F000048BBDE8F08305F5805804469FED398A17
:10D80000D8F89C0F9FED380A6C3045F077FB61EE3D
:10D81000087AD5F84C6420EE089A8DED020A60EE85
:10D82000888AFDEEE77A3368CDED030A30469B6DBA
:10D8300017EE902A8DED041A94F8109017B29847BD
:10D8400007EE900A3046F8EEE77A67EE887AFDEE4A
:10D85000E77A17EE903A1CB23368DB6D984707EE13
:10D86000900A9FED227AF8EE677A67EE887AF4EEF6
:10D87000C77AF1EE10FA30D5FCEEE77A17EE903A5F
:10D880009DB2D8F8A43F3046DFED169A93ED0F8A8B
:10D89000336828EE298A1B6E98471A23B72220EE98
:10D8A000290A48463E21ADF828708DED059ACDED48
:10D8B000068A8DED078A8DED090AADF82A40ADF88C
:10D8C0002C50CDE900320022089205AA84F07AFAA1
:10D8D0000DB0BDEC048BBDE8F0834FF6FF75D0E7CB
:10D8E000E89302200AD7233C9F0CB34500FF7F47F3
:10D8F0001D4B2DE9F04F2DED028BD3F89C3F8DB0E1
:10D90000077CD3F88480D3F88860D3F88C50D3F8A0
:10D91000904093ED258AD3F898B0D3F89CA0D3F823
:10D92000DC90F1F069FD162225234FF0000C0290E7
:10D930000192384602AA532100938DED078ACDF853
:10D9400020B0CDF824A0CDF82890CDF80C80049616
:10D95000059506948DF82CC084F034FA0DB0BDEC1A
:10D96000028BBDE8F08F00BFE8A30220B0EEC00A32
:10D97000DFED157A10B5B4EEE70AF1EE10FA0ED429
:10D98000124CD4F84C0403681B68984704281AD03A
:10D99000D4F84C0403681B689847142813D002225B
:10D9A00011210B4806F07EFE30B140F6C411094843
:10D9B000BDE810400BF0A0B8022205481146BDE8B2
:10D9C000104006F06FBE10BD00000034E893022046
:10D9D000E83302203CC60220A1F11B0370B50446C7
:10D9E00084B0282B16D8DFE803F01A151515151585
:10D9F0001515155915151E4F151515151515151550
:10DA000015151515151515151515151515151529B2
:10DA1000151A1A0004B0BDE870408CF08FBE0125C5
:10DA2000284604B070BD122183F02EFA0546002866
:10DA30004AD0217C26487AF04DFBF1E7262183F07D
:10DA400023FA054600283FD0217C2248BCF0CEFBBB
:10DA5000214B1E68002EE3D02621204683F014FAC5
:10DA600005460028DCD0002301AA40212046ADF85D
:10DA7000043089F0F7FB0028D2D0BDF804203046EE
:10DA8000217CB2F0E1FECBE7162183F0FDF90546DB
:10DA9000D0B1217C0E487AF035FCC1E70C2183F02F
:10DAA000F3F9054680B1002301930293039319F023
:10DAB000DFFA01A919F078FA03460028B0D0204611
:10DAC0001D46FFF7C3FCABE70025284604B070BD38
:10DAD00054B50220F8BE02202CDD0220054BD3F8FD
:10DAE00070342BB193F8CA00002808BF0220704799
:10DAF00002207047E893022008B5034BD3F84C048A
:10DB000003681B68984708BDE8930220024B93F80E
:10DB10004104C0F340107047E8930220F0B52A4F4B
:10DB200087B0D1ED017A0646D7F84C340C46FDEEAD
:10DB3000E77A1A68184617EE905A536A9847EB0727
:10DB400000D440B3D4E9040140F0BAFE18B302A8EF
:10DB500021F066FB02AA214630468AF00FFAD0B1C6
:10DB60001A4902A822F0D0F9A8B9DFED190A034634
:10DB700002460090B0EE600A02A916480EF00EF9B7
:10DB800090B1D7F84C0403685B6A9847044628B103
:10DB9000002007B0F0BD022007B0F0BD0222042132
:10DBA0000D4806F07FFD08B90420F5E7DFED080A0F
:10DBB0002346224602A9B0EE600A064800940EF001
:10DBC000EDF80028E4D1EFE7E893022058B30220F3
:10DBD0000000000098C70220E833022091ED000AFF
:10DBE000B5EEC00AF1EE10FA1EDBDFED1F7AB4EEDF
:10DBF000E70AF1EE10FA17D89FED1C7A10B5D1EDB7
:10DC0000037A82B00C46F0EEE76AF4EEC76AF1EEF2
:10DC100010FA0FD4F7EE000AB0EE670A3EF07AFF72
:10DC200020B9042002B010BD0420704794ED000A12
:10DC3000D4ED037ADFED0D6A94ED027AF4EEE67A24
:10DC4000D4ED010AFDEEC77A0948F1EE10FACDEDE8
:10DC5000017A9DF90410ACBF0122002202F0D4FA2F
:10DC6000002002B010BD00BF0000B443000000342B
:10DC700094CD0220D1ED017AF5EEC07AF1EE10FAE2
:10DC800030DD91ED007ADFED186AB4EEE67A08B582
:10DC9000F1EE10FA0CDD154B9FED150AD3F84C048C
:10DCA00027EE800A0368DB6E9847A0B1002008BD0C
:10DCB000DFED106A0D4BB4EEE67A9FED0D0AD3F856
:10DCC0004C0427EE800AF1EE10FA036805DD9B6E26
:10DCD00098470028EAD1042008BD5B6E98470028C9
:10DCE000E4D1F8E7042070479A993940E89302207C
:10DCF0000000C8423333F33FD1ED007A9FED167A2E
:10DD0000F0EEE77AF4EEC77AF1EE10FA11D5D1ED24
:10DD1000017AF0EEE77AF4EEC77AF1EE10FA08D560
:10DD2000022203210D4808B506F0BCFC18B90420F6
:10DD300008BD0220704709480121FCF7E3FF0848AD
:10DD400090F8903D012B05D000F68C5049F0CCFBAB
:10DD5000002008BD002008BD00000034E833022088
:10DD6000E8B3022010B5154882B00C46EAF0DEFB9D
:10DD700060B1D4ED017AFCEEE77ACDED017A9DF841
:10DD80000400012805D002280BD090B1042002B075
:10DD900010BD94ED020A0948EAF02CFC002002B004
:10DDA00010BD94ED030A0548EAF068FC002002B0BB
:10DDB00010BD034B83F88A0C02B010BD64900220A2
:10DDC000E883022010B5D1ED007A0446FCEEE77A34
:10DDD00017EE903A13F0FF0308D1114BD3F84C041F
:10DDE00003689B6F9847A0B1002010BD012B01D0A4
:10DDF000022010BD0A4BD3F84C040368DB6F984730
:10DE00000028F1D12046074A062187F0AFF8042008
:10DE100010BD2046044A062187F0A8F8042010BD52
:10DE2000E8930220947517088475170838B5194CC3
:10DE300094F86534DB070ED4D4F8703493F8D530F9
:10DE40005BB194F94034002B0FDB02220921A4F5C9
:10DE5000C04006F027FC002038BD012204F1F0008C
:10DE60001146FCF783FD002038BD0D460222052136
:10DE7000A4F5C04006F016FC0028ECD095ED000A91
:10DE80000121DFED057AD4F84C0420EE270A15F0C5
:10DE90000BF8E0E7E89302200000C842F6EE007AB3
:10DEA00091ED007AB4EEE77AF1EE10FA01DC04208D
:10DEB000704701220521034808B5FCF719FE002030
:10DEC00008BD00BFD894022030B58B8B85B08C463E
:10DED0000446D12B12D8B12B2DD8202B22D8102BB1
:10DEE0005AD9113B0F2B57D8DFE803F05D5656681F
:10DEF000894F565656565656565656704AF2124E38
:10DF0000734500F0F0802BD94AF2134E734500F0B0
:10DF1000D3804AF2686E73453ED105B0BDE830400B
:10DF2000FFF720BF552B6AD0732B2CD105B0BDE86D
:10DF30003040FFF753BEB23B1F2B2DD8DFE803F074
:10DF40006D2C2C2C2C2C2C2C2C2CA3AA2C2CB1671B
:10DF50002C2C2C2C2C2C2C2C2C2C2C2C2C2C738660
:10DF6000B3F5967F00F0A3804AF2114E734513D1AA
:10DF70007B4D95F8654414F0010400F0B98000244D
:10DF8000204605B030BD542B06D19CF82030032B21
:10DF900000F0BE800224F3E76146204605B0BDE8EC
:10DFA00030408CF091BF022205216E4806F07AFBCA
:10DFB0000028E4D10424204605B030BD0222062109
:10DFC000684806F06FFB0028D9D1F3E7DCED007A52
:10DFD000F5EEC07AF1EE10FADCDD9FED637AF4EE37
:10DFE000C77AF1EE10FAD5D8FCEEE77A5F4A002442
:10DFF000CDED027A9DF80830A2F8A23CC0E70222DB
:10E000000921584806F04EFB0028B8D1D2E76146F6
:10E0100005B0BDE83040FFF7D5BE614605B0BDE8AC
:10E020003040FFF727BEDCED007AFCEEE77A17EE12
:10E03000903A99B2012904D0022900F08580002984
:10E04000B8D14B4800249FF08BFD99E79CED017AF5
:10E050000146DCED007ABCEEC77A9CF81030FCEE8D
:10E06000E77ADCED030A9CED020A8DED027ACDED34
:10E07000037A00933B489DF808309DF80C2013F07C
:10E0800009FB04467CE702213A4807F035FF0028E7
:10E0900090D074E70221374807F0F8FE002889D0B5
:10E0A0006DE7614605B0BDE83040FFF737BD05B00C
:10E0B000BDE83040FFF720BE294890F8654414F0D1
:10E0C00001047FF45CAFD0F8702492F8D520002AC8
:10E0D0003FF455AF90F94024002A3ADB91ED000A55
:10E0E000FFF744FC4CE705B0BDE83040FFF79EBEAB
:10E0F00002220521A5F5C04006F0D4FA00287FF4DD
:10E100003EAF0222A5F5C040114606F0CBFA37E734
:10E11000DCED027A9FED187AF0EEE77A9CED060AC4
:10E12000DFED166A0E4BF4EEC77A20EE260AD3F81E
:10E130004C04F1EE10FA4CBF0121002114F0B4FEA2
:10E1400000287FF41CAF35E70648002403F03EFEAC
:10E1500016E701220821F030FCF7CAFC10E700BFE7
:10E16000E8930220E833022000007F43E883022086
:10E1700014B5022038C10220000000340000C8425B
:10E1800030B50C46272200212DED028BE57893B0A7
:10E19000954208A828BF154663F120FB04F10C0145
:10E1A00008A82A4663F1D0FA4C4BD3F84C04036814
:10E1B0005B6A9847002841D09DF8464061063DD4EF
:10E1C0004FF07E5200230492220607930693059394
:10E1D00040D40A9804AD0B9A0C9B099905902846E7
:10E1E00004910692079343F0D7FA38B30023E24331
:10E1F00084F0020004F00401019302F00102029392
:10E20000C0F340000393A3071CD052EA000329D1B6
:10E2100041B333480CF092FDB7EE001A044648B300
:10E22000FFEE000A40F2ED409DED100A3EF038FE90
:10E23000234601AA29462A480CF088FD13B0BDECFC
:10E24000028B30BD59B90D990E9A0F9B0191029224
:10E250000393DEE704AD284643F098FAC6E70AB90F
:10E260000028D6D001211E480CF006FD13B0BDECED
:10E27000028B30BDDFED1B0A4FF49E609DED100A4E
:10E280003EF00EFEF6EE000AB0EE408A3EF042FC92
:10E2900090B9B6EE000AB4EEC08AF1EE10FA0EDDC7
:10E2A00038EE408A104BD3F8A83F38EE088A93ED39
:10E2B000070A28EE000ABBE79FED0A0AB8E70A4BF7
:10E2C00030EE488AD3F8A83F38EE088A93ED080A62
:10E2D000B0EEC00A20EE480AAAE700BFE893022089
:10E2E00098C7022000000000E8A302202DE9F047B3
:10E2F0000C46352200212DED028BE5789CB095422D
:10E300000EA828BF154663F169FA04F10C010EA8A6
:10E310002A4663F119FAB94BD3F84C0403685B6AD7
:10E320009847002800F0CA809DF86C50EB1F012D23
:10E33000DBB202D0022B00F2D180BDF8684014F4A9
:10E34000E0780CBF0122002212EA542640F0B68089
:10E35000002214F007090592069207921BD19FED47
:10E36000A86AA5F10802DDED106ADDED117A012A37
:10E370009DED0F7A66EE866A67EEC67A27EE067A1C
:10E38000CDED066ACDED077A8DED057A40F22E814E
:10E39000022B40F22281002714F0380A08970997CF
:10E3A0000A9740D1DDED127ADDED146AF4EE677A5A
:10E3B0009DED137AB1EE666ACDED087A8DED097A9E
:10E3C000F1EE10FA8DED0A6A80F18880F0EEE77ABE
:10E3D0009FED8C6AF4EEC67AF1EE10FA7EDCB4EEB4
:10E3E000477AF1EE10FA79D6B0EEC77AB4EEC67A73
:10E3F000F1EE10FA72DCF4EE666AF1EE10FA6DD608
:10E40000F0EEE66AF4EEC66AF1EE10FA66DC9FED15
:10E410007C8A08A8B0EE480A44F0C4FDA5F10803C0
:10E42000012B40F2A88000230B930C930D93B8F1BD
:10E43000000F18D19FED726AA5F10803DDED166A91
:10E44000DDED177A012B9DED157A66EE866A67EE93
:10E45000C67A27EE067ACDED0C6ACDED0D7A8DEDFC
:10E460000B7A40F2A68014F4806040D014F400636C
:10E470009FED650A4ED1DDED190AA2069FED637A84
:10E48000DFED5F7A60EE870A60EEA70A46D0B9F149
:10E49000000218BF0122BAF1000F14D19AB1B3FAE9
:10E4A00083F40121B0FA80F30BAA640958485B0990
:10E4B0000094CDE9016108A90DF0D2FA1CB0BDECC1
:10E4C000028BBDE8F087BAF1000118BF0121002AD4
:10E4D00038D0002936D0B8F1000F70D001214C4857
:10E4E0000CF0CAFB1CB0BDEC028BBDE8F087A5F1B7
:10E4F00008029DED180A9FED457A012ADFED407A6A
:10E5000020EE070A8CBF0026012614F4006320EEDB
:10E51000270AB0D0A206DFED3C0AB8D1B3FA83F1E6
:10E52000B0FA80F00BAB08AA49094009CDE9011601
:10E5300005A9009036480DF075FD1CB0BDEC028BAE
:10E54000BDE8F087B9F1000F14BF002101F001010F
:10E550000029C3D0B8F1000FC0D00024B0FA80F277
:10E56000B3FA83F305A9520929485B09CDE9006490
:10E570000DF004FBA2E708A909AA2648FCF716FE3D
:10E580000B970C970D97B8F1000F7FF46CAFDDED92
:10E59000166A9DED177ADDED157A66EE886A27EE2C
:10E5A000487A67EE887ACDED0C6A8DED0D7ACDED67
:10E5B0000B7A0CAA0BA91748FCF7F8FD53E70124C6
:10E5C000B0FA80F2B3FA83F30BA9520910485B0941
:10E5D000CDE900640DF0D2F970E705AF0E48E3F025
:10E5E000F3FB0146384644F0A9FCD4E605AF06AA81
:10E5F00008483946FCF7DAFDF0E700BFE89302204F
:10E600000000C84200007A4400000000E02E65428D
:10E6100098C70220E833022068B302202DE9F047B2
:10E620000C463522002106462DED028BE578A0B080
:10E63000954212A828BF154663F1D0F804F10C01E9
:10E6400012A82A4663F180F8A04BD3F84C04036863
:10E650005B6A984730B1BDF87840A30504F4E075D3
:10E6600005D525B920B0BDEC028BBDE8F0870AAF17
:10E6700004F00708384620F0D3FDB8F1000F00F091
:10E68000A580002314F038060493059306933CD12B
:10E69000DDED167ADDED186AF4EE677A9DED177AF6
:10E6A000B1EE666ACDED047A8DED057AF1EE10FAE1
:10E6B0008DED066A80F19980F0EEE77A9FED846A2D
:10E6C000F4EEC67AF1EE10FA00F38F80B4EE477ADA
:10E6D000F1EE10FA80F18980B0EEC77AB4EEC67A16
:10E6E000F1EE10FA00F38180F4EE666AF1EE10FAB2
:10E6F0007BD6F0EEE66AF4EEC66AF1EE10FA74DC50
:10E700009FED740A04A844F04DFC0023079308937E
:10E7100009939DB99FED6F6ADDED1A6ADDED1B7AF5
:10E720009DED197A66EE866A67EEC67A27EE067A5E
:10E73000CDED086ACDED097A8DED077A14F4806A83
:10E7400034D014F400699FED648A3CD1DDED1D8A5C
:10E75000DFED627ADFED5F0A68EEA78A68EEA08AD5
:10E7600014F03F044AD0B8F1000318BF01230EB9DA
:10E77000002B64D1003E18BF0126002B00F08B80D7
:10E78000002E00F0888085BB0120B9FA89F3BAFA1F
:10E790008AF2F0EE680AB0EE480A5B09520907A94E
:10E7A000CDE900504E480DF0E9F85BE79DED1C8A7D
:10E7B00014F40069DFED497A9FED460A28EE278AB6
:10E7C00028EE008AC2D0DFED448AC9E7DDE9139A5A
:10E7D0004846514640F074F838B1304607AA9DF8D3
:10E7E0007C108BF0ADF900283ED101213C480CF0A3
:10E7F00043FA20B0BDEC028BBDE8F087384620F02C
:10E8000065FD0328F1D0002338460EA90E930F931F
:10E81000109320F0D5FE0028E7D0B9FA89F0BAFAB3
:10E820008AF3F0EE680A04AA4009B0EE480A5B09D0
:10E830000EA9CDE900042A480DF078FC12E7B9FAD8
:10E8400089F401200021BAFA8AF36409F0EE680A1B
:10E85000B0EE480A5B0907AA0094CDE9011004A9AB
:10E860001F480DF0FDF8FDE6DDED157A0EAE9FEDCB
:10E87000197A5246079B494667EE877A30460093DD
:10E88000FDEEE77A17EE903A20F0E2FC96E80F00F2
:10E8900087E80F00F5E6B8F1000F14BF002606F078
:10E8A0000106002EA1D0002D9FD00020B9FA89F3D7
:10E8B000BAFA8AF2F0EE680A0090B0EE480A5B09F4
:10E8C0003946520906480DF069FACBE6E893022072
:10E8D00000007A440000C84200000000E02E6542BB
:10E8E00098C7022000B591F80AE04B7A43EA0E235C
:10E8F00091F80BE043EA0E43562B16D00A468446A5
:10E9000007D8522B1BD0542B13D15DF804EBFFF723
:10E91000EDBC0D49194421F07F41012909D8017C42
:10E920005DF804EB094879F0ADBD5DF804EBFFF745
:10E9300075BE114660465DF804EB8BF08BB95DF84F
:10E9400004EBFFF71DBC00BF7AFFFF0054B50220A7
:10E950002DE9F041044648F26C10002301222044C6
:10E960002DED028B90B0694600937AF0A5FC08B9B2
:10E97000584B009304F5C048D8F84C0403685B6911
:10E980009847002840F0968004F5E0479FED528AB2
:10E99000D7F8A43F93EDE07BD3EDE76AFDEEE66A9E
:10E9A000B7EEC77B16EE903A27EE088A1EB246F203
:10E9B000780501A92544284613F006FD00287FD0DC
:10E9C0003722002102A862F109FFA3238DF8083045
:10E9D00095238DF80930F0F017FDD7F89C3FCDF85E
:10E9E0000B00D8F87004D3F8DC20D3F8E0304430C2
:10E9F000CDF81320CDF81730CDF80F1081F0B4F812
:10EA0000B7EE001A90ED000ADFED340A9F203EF0C9
:10EA100047FAD8F8700410EE103A314ACDF81B309E
:10EA200003681B69934250D190ED4B0AB6EE061A6B
:10EA3000F4EE000A30203EF033FA10EE103A04F5FE
:10EA4000FF48CDF81F3018EE103A4046CDF823307D
:10EA5000E3F0BEF9DFED207A2846D7F84C3F20EEF0
:10EA6000270ACDF82B3010EE103ACDF82730019B55
:10EA7000CDF82F3013F0CCFC009A10EE103A40463F
:10EA8000ADF83B60CDF83330CDF83720E3F0ACF98A
:10EA9000BDEEC00A41F65820372202A9204410EEEC
:10EAA000103AADF83D307CF08FFE10B0BDEC028B1B
:10EAB000BDE8F08100269FED098A04F5E04776E77E
:10EAC0007DF0A6FF034B01937AE7984710EE103ACA
:10EAD000B5E700BF2292CA7F0AD7233C000000009E
:10EAE00049AE000810B500F5E044D4F89C0FD8F00A
:10EAF000CBFCD4F8A41FD4F89C0FBDE81040D8F08C
:10EB000029BD00BF70B54FF48051044613F0B0FD2D
:10EB100000284FD004F5E04641F65825D6F89C0F62
:10EB2000254403689B689847692100F1A0022846A4
:10EB30007CF04AFCD6F89C0F0368DB6898476A2192
:10EB400000F1A00228467CF03FFCD6F89C0F036839
:10EB50001B6998476B2100F1A00228467CF034FC29
:10EB6000D6F8A42F6C21284602F52D727CF02CFCDF
:10EB70002021204613F07CFDE0B104F5C043D3F81A
:10EB80004C0403681B69984778B1D6F8A42F28462F
:10EB90006E2190327CF018FCD6F8A42F28466F2105
:10EBA000BC32BDE870407CF00FBC20460DF046FC46
:10EBB0000028EAD170BD00BF08B518F059FABDE8C9
:10EBC000084018F0AFB900BF70B50D4684B04FF6DD
:10EBD000FF710646144613F04BFD08B904B070BD32
:10EBE0000023CDE90033CDE90233A3238DF80030B3
:10EBF00095238DF8013003238DF80230F0F004FCEA
:10EC0000CDF8030041F658200B46102230446946E7
:10EC10008DF80B50CDF8073003947CF06BFE04B0F8
:10EC200070BD00BF70B50D4684B04FF6FF7106464B
:10EC3000144613F01DFD08B904B070BD0023CDE9E2
:10EC40000033CDE90233A3238DF8003095238DF8EE
:10EC5000013004238DF80230F0F0D6FBCDF803002C
:10EC600041F658200B461022304469468DF80B506F
:10EC7000CDF8073003947CF03DFE04B070BD00BFBA
:10EC800030B50023A32204460D462DED048B87B03A
:10EC9000B0EE409AF0EE608A0093B0EE418A0593A0
:10ECA0008DF800209522CDE90133CDE90333062309
:10ECB0008DF801208DF80230F0F0A6FBCDF80300AE
:10ECC00041F658200B461822694620448DF80B5017
:10ECD000CDF807308DED039ACDED048A8DED058AD0
:10ECE0007CF072FD07B0BDEC048B30BD10B54FF465
:10ECF0008011044613F0BCFC00B910BD04F511509E
:10ED0000BDE8104015F0BCBF2DE9F04F2DED028B92
:10ED10008DB080462F2200216846F0EE408AB0EE8A
:10ED2000608A11EE10BA11EE90AA12EE109A12EE4D
:10ED3000907A13EE106A13EE905A14EE104A62F1B4
:10ED40004DFDA3238DF8003095238DF80130092364
:10ED50008DF80230F0F058FB18EE903ACDF8030031
:10ED600041F65820CDF80710CDF80B302F2218EEC1
:10ED7000103A69464044CDF813B0CDF80F30CDF8C5
:10ED800017A0CDF81B90CDF81F70CDF82360CDF8FB
:10ED90002750CDF82B407CF017FD0DB0BDEC028B59
:10EDA000BDE8F08F30B52DED088B8BB028220446DE
:10EDB0000D4668460021B0EE40BAF0EE60AAB0EE13
:10EDC00041AAF0EE619AB0EE429AF0EE628AB0EE9D
:10EDD000438A62F103FDA3238DF8003095238DF85B
:10EDE00001300A238DF80230F0F00EFBCDF803005D
:10EDF00041F658200B462822694620448DF80B50D6
:10EE0000CDF807308DED03BACDED04AA8DED05AA3E
:10EE1000CDED069A8DED079ACDED088A8DED098A24
:10EE20007CF0D2FC0BB0BDEC088B30BD2DE9F0437B
:10EE30008FB01446074689463122002101A8169E4C
:10EE4000179D984662F1CAFCA3238DF804309523E0
:10EE50008DF8053008238DF80630F0F0D5FA2368D8
:10EE60003122CDF8070041F65820049363683844F6
:10EE7000CDF80B1001A90593A3686C68069333685D
:10EE80008DF80F90CDF81D3073688DF81C80CDF88B
:10EE90002130B368CDF82D40CDF825302B68CDF862
:10EEA0002930AB68CDF831307CF08EFC0FB0BDE876
:10EEB000F08300BFF0B52C27144605460E463A46AF
:10EEC00000212DED068B8DB0B0EE409AF0EE608AF9
:10EED00001A8B0EE418AB0EE61AAF0EE429A62F16A
:10EEE0007DFCA3238DF8043095238DF805300B238A
:10EEF0008DF80630F0F088FADFED1A7A0B4694EDC3
:10EF0000006A3A46D4ED016A29EE279A94ED027A16
:10EF100026EE276ACDF8070041F6582066EEA76A6C
:10EF200001A968EEA78A284428EE278A8DF80F6089
:10EF300067EE277ACDF80B308DED049ACDED058A7A
:10EF40008DED068A8DED076ACDED086ACDED097A63
:10EF50008DED0AAACDED0B9A7CF036FC0DB0BDEC20
:10EF6000068BF0BDE02E6542B020704730B50446F8
:10EF700041F6582589B0134B25441E22D3F870045E
:10EF80006946E4F05BFC6A460F4928467CF08CFB3E
:10EF900004F5C043D3F84C0403681B68984704F594
:10EFA00080430146284693F874207CF0E9FD04F57F
:10EFB000115018F0DDFA04F546702CF003FD09B08D
:10EFC00030BD00BFE893022010B31A08F8B54FF027
:10EFD000804105460023404A404C05F6686740489A
:10EFE000A96340496B61AB61EB61EB6329646A64BF
:10EFF0006C6305F66834686005F14800D1F01CF9CF
:10F0000005F58270A5F064FA05F52B608CF0CCFB59
:10F01000354E364BC5F8B03A20468CF03BFE44F8EE
:10F02000306BBC42F8D1204605F580568EF0C8FE04
:10F0300041F6F40000212E4C2844E8F09DFA41F6F8
:10F04000A4102844E9F060FA41F6C810C6F8C44993
:10F050002844EAF00FF9A4F5E76341F66420C6F806
:10F06000583A2844ADF094F8A4F50C7341F62C40BE
:10F07000D434C6F81C3C9FED1F1A2844DFED1E0A4D
:10F080009FED1E0AC6F8284CD9F056FA9FED191AC2
:10F0900041F644409FED1A0AF0EE410A2844D9F0A7
:10F0A0004BFA9FED141A41F65C409FED150AF0EE05
:10F0B000410A2844D9F040FA41F6AC402844DEF039
:10F0C00075FD28460F496EF071F928460E496EF01D
:10F0D0006DF92846F8BD00BF0000E0400000C841BF
:10F0E000C04A02200AD7233CE0CF1708F4CF170804
:10F0F000F0CB0220000000009A99993E0000B44332
:10F1000000804A4328C2170818C517082DE9F043A4
:10F11000ADF50F7D504DD022504981465AA862F17D
:10F1200013FB0DF1380C5AAC8EAE0FCDACE80F00CE
:10F130000FCDACE80F000FCDACE80F0095E80F0045
:10F140008CE80F0020461034B7EE000A00216EF064
:10F150005FFFB442F6D1424B02AC0FCB84E80F0004
:10F1600001A920466EF004FF002844D10EAC0DF139
:10F17000780820461034B7EE000A00216EF048FFF0
:10F180004445F6D136AF90223649384662F1DCFA72
:10F190000022092138466EF0F7FF99F9946D002E90
:10F1A0003DD0314D06AE9FED310A44460FCD0FC61E
:10F1B00095E80F0086E80F0006A800216EF028FFF2
:10F1C000002130469FED290A6EF022FF602205F1F2
:10F1D0001001404662F1B8FA20461034B7EE000A3A
:10F1E00000216EF015FFA742F6D18EF0AFFD0DF5B0
:10F1F0000F7DBDE8F0839DF90430F0EE007ADFED7D
:10F200001C6AB7EE000A07EE103AE068B8EEC77A5B
:10F21000E7EE267A80EE270A6FF052FCA6E7154D3E
:10F2200044460FCD0FC40FCD0FC40FCD0FC495E8CA
:10F230000F0084E80F003246042140466EF0A4FF20
:10F240009FED0D0A0D486FF03BFCB7EE000A0C482D
:10F250006FF036FCA5E700BF645A170894591708E9
:10F26000A45A1708B45A1708845B170800003442E0
:10F27000CDCCCC3D445B1708000000000CC1170842
:10F280001CC1170830B5B5B0D0220849684634AD66
:10F29000044662F159FA20461034B7EE000A002104
:10F2A0006EF0B6FEAC42F6D135B030BD045C170846
:10F2B0002DE9F04391B01D200DF106018EF0F0FB19
:10F2C00010B911B0BDE8F0839DF8063011216F4AE6
:10F2D0000BA80133DBB28DF80630EFF0BDF9002248
:10F2E0000DF107010BA86DF065FC9DF80630684A2A
:10F2F000112104460BA8EFF0AFF900220DF1070130
:10F300000BA86DF057FC9DF80630624A11210546A6
:10F310000BA8EFF0A1F900220DF107010BA86DF089
:10F3200049FC9DF806305C4A112103F03F03074673
:10F330000BA8EFF091F90DF107010BA800226DF079
:10F3400039FC0646002CBCD0002DBAD0002FB8D016
:10F350000028B6D020466DF0E3FF0028B1D1284642
:10F360006DF0DEFF0028ACD138466DF0D9FF0028E3
:10F37000A7D130466DF0D4FF0028A2D1474B0DF144
:10F380000C0C0DF11C0803F1100E0FCB8CE80F00D4
:10F390009EE80F0088E80F0002A960466EF0E8FDC5
:10F3A00002A968B3BDF9089040466EF0E1FD1FFA6E
:10F3B00089F3002857D1002B83D040F2D66842460B
:10F3C0009A4232D228460DF10A01ADF80A906FF048
:10F3D00087FF20460DF10A01ADF80A806FF080FF2B
:10F3E0000DF10A013846ADF80A806FF079FF01236C
:10F3F0000DF10A013046ADF80A306FF08BFF60E77F
:10F4000040466EF0B5FD00283FF45BAFBDF90880C3
:10F410001FFA88F2002A3FF454AF40F2E2494B460B
:10F42000CEE740F2E24940F2D66828460DF10A01E3
:10F43000ADF80A806FF054FF20460DF10A01ADF8D7
:10F440000A906FF04DFF0DF10A013846ADF80A90B1
:10F450006FF046FF00230DF10A013046ADF80A3087
:10F460006FF058FF2DE7BDF908801FFA88F253EAC4
:10F4700002013FF426AF23B1002A9ED00FFA83F990
:10F480009EE7002ACDD040F2E243F7E72CC11708EF
:10F4900038C1170844C1170854C11708D45C1708AD
:10F4A00044F26421782230B5014483B004467AF0F6
:10F4B00065F800220C21294801256EF065FE2046E2
:10F4C000FFF7F6FE44F27820B7EE000A0022022190
:10F4D00020446EF00DFF43F6DC510023204A214406
:10F4E000452000956EF06AFE1E4B1A68D1070DD4B8
:10F4F00043F6102043F6F0611D6041F66C331A4A62
:10F500002044214423441060D160936144F2D82008
:10F5100003221549012520446EF0B2FE41F6582120
:10F520000023124A2144FD2000956EF047FE104B47
:10F530001A68D20705D442F22C320E491D602244CB
:10F540000A6001210B486EF0B9FE6FF0B1FA0A4A69
:10F55000138843F00103138003B030BD68C117085E
:10F56000E0531A088CCD0220C4250220C8C5180813
:10F5700090CD0220E825022020D102200F2904D8B6
:10F58000302303FB0100B83070470020704700BFF4
:10F59000014B93F9AB027047E8730220024B93F8DA
:10F5A000650400F001007047E8930220054BB3F8B2
:10F5B0007032DB0703D40069C0F3401070470020AD
:10F5C000704700BFE8730220014BD3F8D80F704793
:10F5D000E883022038B50C1E05DB1C4DE3B295F81C
:10F5E000E42F9A4200D238BDD5F8E03F0122A5F5BC
:10F5F000A040195D05F056F80028F4D08CF042FBCD
:10F6000003218DF0B9FD0028EDD18CF03BFB0D21DD
:10F610008DF0B2FD0028E6D1A5F5805292F9903226
:10F62000E340DB0706D5A5F5A0400221BDE8384040
:10F63000FBF77EBB92F9AA12A5F5A040E140BDE818
:10F64000384001F00101FBF773BB00BFE8830220E3
:10F65000022910B5044608D00A4BD3F84C040368BD
:10F660001B689847844207D010BD014635220648E2
:10F67000BDE8104005F016B88CF004FBBDE8104062
:10F680008CF0FAB9E8930220E833022008B5036849
:10F690000A4A9B6893420ED1094B93F8650400F027
:10F6A000010030B9064B93F96404B0FA80F04009C8
:10F6B00008BD002008BD9847F3E700BF9DF500088E
:10F6C000E893022000F5A0439FED186ADFED186A69
:10F6D000012110B5D3F8D02F0446D3F8CC3F00F564
:10F6E0001150B2F90820B3F9083007EE102A07EEDE
:10F6F000903AB8EEC77AF8EEE77AC7EE060A87EED8
:10F70000860A60EEA60A20EE260A17F05BFD7DF061
:10F710007FF926217CF06CFE46F2D810054A0621BE
:10F720002044BDE8104081F0C5B800BF0000C842C9
:10F7300035FA8E3C8CCD170870B500F5E04595F88C
:10F74000B81F00294DD0334B0446334AD3F84C043C
:10F75000904247D1D3F87034304E93F8D530002B17
:10F7600041D0012395F8B92F337242B904F5C04254
:10F7700092F94024002A34DB85F8B93F05E004F50E
:10F78000C04393F94034002B2DDB013904F5A0432D
:10F790009FED236A04F51150C9B2DFED226A85F8A6
:10F7A000B81FB1FA81F1D3F8D02FD3F8CC3F490973
:10F7B000B2F90820B3F9083007EE102A07EE903AA4
:10F7C000B8EEC77AF8EEE77AC7EE060A87EE860A41
:10F7D00060EEA60A20EE260A17F0F4FC95F8B83F72
:10F7E00073B170BD0D4E002346F2D8100E4A0621AB
:10F7F000204485F8B83F3372BDE8704081F05AB8B4
:10F8000046F2D8103372094A06212044BDE8704000
:10F8100081F050B8E893022084C9022068D0022009
:10F8200000007A4535FA8E3C98CD1708ACCD170804
:10F830008B1ED92B6ED8DFE803F06F706F6F6D6F82
:10F840006D6D706D6F70706D6F6F6F6D6D706F70CF
:10F850006D70706D6D6D6D6D706F6D6D6D6F6D70C8
:10F860006D6D6F70706F6D6F6F6F6D6D6F6D6D6FB4
:10F870006F6F6D6D6F6F6D6D6D6D6D6D6F6F6F6FA8
:10F880006F6F6D70706D6D6D6D6D6D6F706D6D6D99
:10F890006D6D6D6D6D6D6D6D6D6D6D6F6D6D6D6D96
:10F8A0006D6D6D6D6D706D6D6D6D6D6D6D6D6D6D85
:10F8B0006D6D6D6D6D6D6D6D6D6D6D6D6D6D6D6D78
:10F8C0006D6D6D6D6D6D6D6D6D6D6D6D6D6D6D6F66
:10F8D0006F6D6F6D6D6D6D70706F6D6D6D6D6D6D4C
:10F8E0006D6D6D6D6D6D6D6D6D6D6F6D6F6D6D6D44
:10F8F0006D6D6D6D6D6D6D6D6D6D6D6D6D6D6D6D38
:10F900006D6D6D6D6D6D6D6D6D6D6D6D6D6D6D6D27
:10F910006D6D6D708DF068BA704700238DF02ABA56
:10F920008B1E70B58AB0D92B00F22781DFE813F067
:10F930000A0301031403E8022501DA002501250169
:10F94000DF0225012501D402C1022501BB02B50257
:10F95000AF0225012501A5029D028E02250182022A
:10F960005502250125012501250125010202FC0181
:10F97000250125012501F6012501EA0125012501C1
:10F98000E4012501DB0121012501250125012501D6
:10F9900025012501D501250125014F024902430218
:10F9A000250125013D022202250125012501250110
:10F9B000250125011C0216021002C301BD01C90167
:10F9C0002501AE019A012501250125012501250109
:10F9D00025018C017F012501250125012501250136
:10F9E00025012501250125012501250125012501E7
:10F9F0002501790125012501250125012501250183
:10FA000025012501250125012501250125012501C6
:10FA100025012501250125012501250125012501B6
:10FA200025012501250125012501250125012501A6
:10FA30002501250125012501250125012501250196
:10FA40002501250125012501250125012501250186
:10FA500025012501250125012501730155012501F8
:10FA6000620125012501250125014A013F012501EA
:10FA70002501250125012501250125012501250156
:10FA80002501250125012501250125012501250146
:10FA90002A012501CF012501250125012501250187
:10FAA0002501250125012501250125012501250126
:10FAB0002501250125012501250125012501250116
:10FAC0002501250125012501250125012501250106
:10FAD00025012501250125012501250125012501F6
:10FAE00025012101022A44D1C24CC34AD4F84C1446
:10FAF00091423ED0D4F8702492F8D520002A38D014
:10FB000004F50055B5F9C02D002A40F0AA8254F83A
:10FB10002C2CA4F58054B2F9083053B305AE002361
:10FB200030460993CDE90333CDE90533CDE90733F9
:10FB30001FF076FBB5F9C03DB04D002B00F094826C
:10FB400005F57763D4F8D44F0FCB86E80F00B4F9EE
:10FB5000083003A9AA48002BCCBF10231523ADF809
:10FB60000E3044F079FE20B17CF052FF27217CF06A
:10FB70003FFC012420460AB070BD0AB0BDE87040C9
:10FB80008CF064BC002A00F01682022AF1D1994B55
:10FB9000D3F84C0403689B6F98470028E9D18AF09A
:10FBA0001BFC984A0421012480F084FEE2E7002A2D
:10FBB00000F00982022ADCD10123934A1C4682F814
:10FBC000B03FD7E7002A00F0F181022AD1D101230A
:10FBD000884A1C4682F84834CCE7022AC9D18B48AF
:10FBE0000124FCF7D7FA8AF0F7FB894A062180F056
:10FBF00061FEBFE711468CF09BFB8648D1F0DAFD31
:10FC000004460028B5D07B4A92F8433443F00203FF
:10FC100082F84334AEE711461C200124FFF718FD9B
:10FC2000A8E711461B200124FFF712FDA2E7002AD6
:10FC300000F0B781022A02D16E4BC3F84424764803
:10FC4000012405F0EBFA95E76A49744BD1F84C04AE
:10FC500098428ED1022A4FF0010400F0F38111F096
:10FC600057FB87E7022A00F087816D4B00220124B1
:10FC700083F8B02C7CF0CCFE4B217CF0B9FB8AF0F1
:10FC8000ABFB684A062180F015FE73E7012A00F0FD
:10FC9000A781022A00F09E81002A7FF46AAF012129
:10FCA00061480C4612F0D6FB64E711460720012498
:10FCB000FFF7CEFC5EE7114616200124FFF7C8FCD3
:10FCC00058E711460B200124FFF7C2FC52E711460A
:10FCD00056480124ECF0FAFC4CE70120114604469A
:10FCE000FFF7B6FC46E7012A00F23C81464B0022B2
:10FCF000012483F88A2C3DE7114615200124FFF7E3
:10FD0000A7FC37E7002A00F04781022A7FF431AFD1
:10FD10000123474A1C4682F878342BE7114612200B
:10FD20000124FFF795FC25E7114611200124FFF778
:10FD30008FFC1FE7013A01242E4BA24293F8421494
:10FD40008CBF0022012262F3041183F8421411E7F0
:10FD5000114602200124FFF77BFC0BE7114610201F
:10FD60000124FFF775FC05E7114600200124FFF789
:10FD70006FFCFFE61F49294BD1F84C449C427FF4AD
:10FD8000F8AE2046019211F0D3FA019A012A00F050
:10FD90006281022A00F05981002A7FF4EAAE2046EF
:10FDA0001146012410F0B0FEE4E6114618200124AB
:10FDB000FFF74EFCDEE6114617200124FFF748FC52
:10FDC000D8E6114605200124FFF742FCD2E6114691
:10FDD00004200124FFF73CFCCCE6A2F10201074B12
:10FDE0000124B1FA81F1D3F89C0F4909DBF06CF8DA
:10FDF000C0E600BFE893022038C10220E8A3022039
:10FE000074C10220ECCD1708E8830220E8330220F9
:10FE100008CE1708D8940220BCC00220C4CC02200F
:10FE2000E8B30220D8CD170860940220B8C402209D
:10FE3000E8C30220A2F10202964B0124B2FA82F238
:10FE4000D3F89C3F520983F8202093E6012A00F062
:10FE5000E680022A00F0DE80002A7FF48AAE114696
:10FE60008D4801249DF07CFE84E6022A7FF481AE59
:10FE70008A48012401F0AAFF7CE6A2F1020186482B
:10FE80000124B1FA81F149099DF06AFE72E611463A
:10FE900009200124FFF7DCFB6CE611460F2001244A
:10FEA000FFF7D6FB66E6114603200124FFF7D0FBDF
:10FEB00060E6012A00F0A480022A00F09780002A60
:10FEC0007FF457AE764B012483F8D4227CF0A0FD5A
:10FED0002B217CF08DFA4DE6012A79D0022A14BF3D
:10FEE000002102216D480124FAF722FF42E6022A8E
:10FEF00000F09B806B4B0022012483F8E82F39E649
:10FF0000022A7FF436AE684DD5F84C040368DB6AEC
:10FF10009847044600283FF42CAE55F82C3CB3F922
:10FF20000830002B7FF425AEA5F5C040FFF7CAFBD3
:10FF300020E6111E59484FF0010418BF0121FAF7BD
:10FF4000F7FE17E6022A7FF414AE35220E2153483D
:10FF5000012404F0A7FB0DE6114606200124FFF75B
:10FF600077FB07E6022A7FF404AE9FED500A0124D6
:10FF70004F48E8F083FBFDE54E4B012483F8B04C7D
:10FF80007CF046FD4A217CF033FA8AF025FA4A4A91
:10FF9000062180F08FFCEDE5484B012483F878249E
:10FFA000E8E5414B0122C3F8442448E63E4B0124D6
:10FFB00083F84824DEE53C4B0124D3F84C04036865
:10FFC000DB6F9847D6E5374B012483F8B02FD1E596
:10FFD000114687E711463A48012412F03BFAC9E579
:10FFE00000213748144612F035FAC3E52C4B0124A2
:10FFF00083F8D4227CF00CFD2D217CF0F9F9B9E5D1
:020000040801F1
:10000000274B144683F8D4227CF002FD2C217CF08F
:10001000EFF9AFE5012120489DF0A2FD28E7114648
:100020001D4814469DF09CFDA4E51921254870F05B
:1000300011FC044600283FF45DAF1A4B012283F8FF
:10004000E82F97E511F0E8F894E5012120460C46E9
:1000500010F05AFD8EE520460021144610F0C8FA33
:1000600088E5A4F5805459E5162303A91648ADF890
:100070000E30D5F8743F642BB8BF6423069344F068
:10008000EBFB00283FF45CAD7CF0C2FC27217CF048
:10009000AFF955E5E8A3022014B50220E8330220A9
:1000A000E8730220E8830220E893022000000000A9
:1000B00064900220E8B30220C4CD1708E8C30220F0
:1000C00060940220904B022074C1022001207047EE
:1000D0000020704738B5044614482DED028BE1F03E
:1000E0007BFE054642F0F8FA1148B0EE408A12F065
:1000F0004DFA30B1DFED0F7AB4EEE78AF1EE10FA87
:1001000004DC94ED080ABDEC028B38BDD5ED000A85
:1001100095ED010A5EF184FCDFED077A20EE270AF7
:1001200084ED080ABDEC028B38BD00BF68B3022025
:10013000E833022000401C46E02E6542174A92F93F
:100140009132022B09D0032B15D073B10368012B18
:100150000AD00122C0E9002370470029F6D00368C5
:1001600013B10022C0E9002370470268002AFBD0C7
:10017000C0E9003270470368042BF5D043600421C6
:10018000A2F5CE539FED067A0160D3ED007AF8EE2A
:10019000E77A67EE877AC0ED087A7047E873022045
:1001A0000AD7233C074B93F99102022807D0032872
:1001B00003D0003818BF012070470420704781F039
:1001C00001007047E873022003688B4208D00429BD
:1001D000C0E9001305D0072900D0704700238362CF
:1001E0007047074B9FED077A03F5C863D3ED007A9C
:1001F000F8EEE77A67EE877AC0ED087A704700BFBD
:10020000E85302200AD7233C70B5044616460D4633
:100210002DED028BF0EE408AB0EE608AEFF0ECF844
:10022000E061002E40D0236843B9334B03F5C86327
:10023000D3ED007AF8EEE77AC4ED097A9FED2F0A44
:10024000002D28EE800A2CDB84ED050ADFED2C7AE8
:100250002C4BB4EEE78AD3F89C0FF1EE10FA10DACB
:10026000D8F0B8FADFED257A20EE270A84ED060AE9
:100270002368032B02D00322C4E90023BDEC028BC8
:1002800070BDD8F0A7FAB4EE480ADFED1C0AF1EE13
:1002900010FA48BFB0EE408A28EE208A84ED068A24
:1002A000E6E7B1EE400ACFE794ED090ADFED137AF5
:1002B00098EEA70A3CF042FD002D84ED050A0CDB08
:1002C000C4D0DFED117AB4EEE70AF1EE10FABDD832
:1002D000DFED0E7A30EE270AB6E7DFED097AB4EEED
:1002E000E70AF1EE10FAB1DBDFED087A30EE670ACB
:1002F00084ED050AAAE700BFE85302200000C842C7
:1003000000000034E8A30220000000B400A00C4765
:1003100010B504462DED028BB0EE608AF0EE408AF7
:10032000EFF06AF8DFED090A236828EEA00AE06121
:1003300068EE200A062B84ED090AC4ED0A0A02D0F1
:100340000622C4E90023BDEC028B10BD0000C842A8
:1003500010B504462DED028BB0EE408AEFF04CF85C
:1003600094ED090ADFED097AE061A8EE270A3CF076
:100370002FFD2368002284ED090A062BA26202D019
:100380000622C4E90023BDEC028B10BD0000C84268
:1003900070B54B680C4606460BB98B687BB1164DA1
:1003A00095F8B51005F13C008FF0BAF8A8B12246D7
:1003B00095F8B5101148BDE870408FF08DBCC96844
:1003C0000029ECD10E48FFF7B9FE0B48BDE870409C
:1003D00090F8B5103C308FF089BC06F1080120463A
:1003E0001FF0EEF80028E2D0054B1A68022ADED092
:1003F0000221C3E90012DAE7E8B3022024B40220A4
:1004000094CD02200368072B02D00722C0E9002305
:1004100080ED0A0A704700BF08B50368032B0CD1B2
:10042000D0ED057A9FED127AF0EEE77AF4EEC77A16
:10043000F1EE10FA03D4002008BD012008BD0D4BD9
:1004400090ED090A03F5C863D3ED007AF8EEE77A78
:1004500037EEC00A3CF072FCB0EEC00ADFED067A5F
:10046000B4EEE70AF1EE10FA94BF0120002008BDB7
:1004700000000034E85302200000484330B5036810
:1004800085B00446023B082B00F28480DFE803F0CD
:100490001D284F59640513050500424B9FED420A84
:1004A000D3F89C0F6C3042F029FDB0EE410A84ED88
:1004B000091A05B030BD3B4DD5F8B00FDFF024F977
:1004C000002860D194ED090AF3E73848E1F07EFC9A
:1004D00004F108013EF072F984ED090A05B030BD5F
:1004E000EEF08AFFE36902469FED317AD4ED060A09
:1004F000F120D31A94ED050AE26107EE903AF8EE86
:10050000677A67EE877A20EEA71A67EEE00A3CF07A
:10051000C7FCD4ED057A94ED091A77EEC07A30EE77
:10052000010AC4ED057A84ED090A05B030BDFFF774
:10053000D1FD9FED201A20EE010A84ED090A05B0D5
:1005400030BD1D4B03F5936393ED000AB8EEC00A6E
:1005500080ED090A05B030BDEEF04EFFE369DFED36
:10056000146AC31A94ED090A94ED0A7A07EE903AD8
:10057000E061F8EE677A67EEA67AA7EE270A84EDC7
:10058000090A05B030BDD5F8B03F93ED100A84EDEF
:10059000090A8EE7034BD3F8A43F93EDD40A80ED0C
:1005A000090A86E7E8A302209F0CB34568B302203E
:1005B0006F12833A0000C842E8930220F0B53F4D25
:1005C00004463F48D5F84C642DED028B336887B064
:1005D000D3F88030834203D107B0BDEC028BF0BD6D
:1005E00030460F4698470028F6D005F58056D5F8D6
:1005F0004C0403F099FE07EE100AD6F89C0F31491F
:10060000B8EEC78A0268DFED307AD2F89820D6F8C3
:10061000A43F28EE278A8A42D3EDD28A33D1D5F877
:100620004C0493EDD31A03688DED031A9B6C984725
:10063000D5F84C24029011681046CA6C9047029B72
:100640000090F0EE680AB0EE480A9DED031A3A46B3
:1006500005A91E48DDF0B6FA236848B90A2BBBD1BC
:1006600000226168A262A1B92046FFF767FDB3E7E7
:100670000A2B02D00A22C4E90023059BA36207B01B
:10068000BDEC028BF0BD9047D6F8A43F78EEC08A4F
:10069000C5E70A29A0D00429C4E900139CD10C4B5A
:1006A0009FED097A03F5C863D3ED007AF8EEE77A97
:1006B00067EE877AC4ED087A8EE700BFE8930220E0
:1006C000D10001083DAE00080AD7233C6C930220FC
:1006D000E853022070B500233C4D0E460446CB6221
:1006E00095F86534DB072BD4D5F84C04384A0368F9
:1006F0005B6F93424FD104F0A1FCB0EEC07ADFED06
:10070000357A86ED0B0AB4EEE77AF1EE10FA4CD5A5
:10071000BDEEC00A304D10EE103A19B23046FFF768
:100720004DFF2D48FFF7AAFE2B6884ED000A092B28
:100730002FD8DFE803F00E1C0E0E0E0E2E2E0E2705
:100740000021254D2B68092BE8D16B6000232B601D
:10075000E4E700210A46A96262600A2B10D8DFE8AC
:1007600003F0140D0D0D0D0D0D140D1414001B4B85
:10077000D3F8A43FD3F85433AB6263600123A36082
:10078000204670BDEB6AAB62636002232046A36023
:1007900070BDAA6AE0E79847A0B9D6ED0B7AFDEEE6
:1007A000E77A17EE903A19B2CBE70B4DBDEEC00ACF
:1007B0002B68092B1CBF0922C5E9002310EE103A53
:1007C00019B2ABE7D5F84C0495E700BFE8930220D7
:1007D000CD0001080000003494CD0220E8A30220DF
:1007E000034B002201219A60DA6019601A61704798
:1007F00094CD022010B582B0044601A904F500444E
:1008000011F044FDA0B1DFED0D6AD4ED367A9DED17
:10081000017A67EEA67AB8EEC77AB4EEE77AF1EE1F
:1008200010FA54BF0123002384F8E53002B010BD54
:10083000012384F8E53002B010BD00BF0000C842BB
:1008400010B52DED028B84B09FED258A01AA8DEDA8
:10085000018A8DED028A8DED038AE6F083FC044661
:1008600020B9204604B0BDEC028B10BD1D4A9DEDA1
:10087000036AD2F8A83FB4EEC86A9DED017ADDEDB7
:10088000027AD3ED066AF1EE10FA27EE267A67EEC9
:10089000A67A8DED017ACDED027A0EDDD3ED077AE1
:1008A00067EE867ACDED037A01A90F4808F028F8A3
:1008B000204604B0BDEC028B10BDD3ED087AA2F542
:1008C0004053D2F8742FF0EEE77AD3F878329A4298
:1008D00067EE867A27FE888A8DED038AE4E700BFFB
:1008E00000000000E8A302207CCA022030B585B0D9
:1008F000002501AA019502950395E6F033FCA8B105
:10090000DDED017A04469FED1A7AF0EEE77A039561
:10091000F4EEC77AF1EE10FA0CD5DDED027AF0EEC6
:10092000E77AF4EEC77AF1EE10FA03D500242046F8
:1009300005B030BD01A842F085FF01A842F046FB9A
:100940000C4B9DED017A01A9D3F8A83FDDED027AA9
:10095000D3ED066A084827EE267A67EEA67A8DED73
:10096000017ACDED027A07F0CBFF204605B030BD0D
:1009700000000034E8A302207CCA022010B504461F
:1009800048F610302044B9F07FFE48F6404020443D
:10099000BDE81040E6F0A0BA08B50F22094803F000
:1009A00081FE00B108BD0F220621064803F07AFE41
:1009B0000028F7D10F2209210248BDE8084003F0C2
:1009C00071BE00BFE833022070B51A4D95F865344A
:1009D000DA0600D470BD6FF304130C46064685F8A2
:1009E0006534A5F500557CF013F8002214217BF046
:1009F00031FD95F874300E2BECD1022C13D0032C62
:100A000008D0012CE6D196F854103046BDE870406D
:100A1000FFF7C2BF96F854100329DBD13046BDE87A
:100A20007040FFF7B9BF30460621BDE87040FFF7C0
:100A3000B3BF00BFE893022010B50E4C31B1D4F81B
:100A40004C0403681B68984713280AD1D4F84C0457
:100A500003681B689847A0F11300B0FA80F04009C2
:100A600010BD0E221321A4F5C04003F01BFE002888
:100A7000ECD1F5E7E893022030B50D4689B0114678
:100A8000FFF7DAFF044610B9204609B030BD04A8CC
:100A90001EF0C6FB16F0ECFA04A916F06DFA00235E
:100AA000E8B901930293164BD3F8A80FA3F5405170
:100AB000D3F8742FD0ED087AD1F87832F0EEE77AD7
:100AC0009A42F1EE677ACDED037A01DA00230393BF
:100AD00001A90C4807F014FF204609B030BD059964
:100AE0002A69019391420293DDDD054B01A9054876
:100AF000D3F8A83FDB69039307F002FFECE700BFE0
:100B0000E8A302207CCA02202DE9F041494C154699
:100B100006460F4694F86534DA062FD443F01003E6
:100B2000D4F84C044FF0010884F8653403681B685E
:100B3000984786F85400D4F84C0403681B6898471B
:100B4000092817D0D4F84C0403681B68984712286A
:100B500010D0D4F84C0403681B6898470E2809D0BD
:100B6000012D21D8062D13D8DFE805F005120B540E
:100B700044382D0000252846BDE8F0814FF00008DC
:100B8000D9E7424639463046FFF776FF00B90025DF
:100B9000B8F1000FEFD07BF03BFF2A4614217BF029
:100BA00059FC2846BDE8F081234801F095FF002854
:100BB000D8D001220A2121480025F9F799FFB8F180
:100BC000000FD8D0E7E7B8F1000FD4D00E220521EE
:100BD000194803F067FD0028DDD109E0B8F1000FE6
:100BE000C9D00E220621144803F05CFD0028D2D1A2
:100BF0000025D0E741463046FFF71EFF0028C6D04B
:100C000039463046FFF71CFE0028C0D0B8F1000F6F
:100C1000B1D0C0E741463046FFF70EFF0028B6D0FE
:100C200039463046FFF762FE0028B0D0B8F1000F19
:100C3000A1D0B0E7E8930220E8330220D894022044
:100C400000F580432DE9F04F2DED068B93F9E2324C
:100C50008DB0044643B100F5C045D5F8703493F823
:100C6000D580B8F1000F13D1002104F5004504F53B
:100C70001150A5F8A41C019016F0B8FC95F8A51C1D
:100C800001980DB0BDEC068BBDE8F04F16F0B8BC76
:100C900000F5E04AEEF0B0FB8346DAF8A40FD0EDA1
:100CA000E4AADBF039F9002840F0F6809FEDA6AA0F
:100CB00009AE204611F06AFC002800F0908004F58F
:100CC000FF494846E1F088F8002307C886E8070096
:100CD00030460B9342F0B6FDB0EE409AD5F84C0486
:100CE00003681B689847122800F0D080D5F870344C
:100CF00093F8D530002B7DD104F50047D5F84C048E
:100D000003685B699847002800F09E8004F5A043C3
:100D1000D3F8D43FB3F90830002B40F3958097F80F
:100D2000A43C5BB1D7F8A80C41F28833ABEB000BC5
:100D30009B4540F2F780002387F8A43CDAF89C0F2B
:100D40009FED820A6C3042F0D9F80DF10C0C8DED5C
:100D5000090A06ABCDED0A0A8DED0B1A9FED7C0A50
:100D600096E8070083E807008CE80700604642F039
:100D7000C5F82046B0EE408A8DED060AF0EE608A96
:100D8000CDED070A8DED081A11F000FC00286AD09D
:100D9000DFED709AB4EEE99AF1EE10FA68D8DAF85D
:100DA000A40FDBF0B9F878B3B4EEE9AAF1EE10FACB
:100DB0002AD8DAF8A40FDBF0EFFB0546002839D17A
:100DC0004846E1F011F804F5115097F8A41C87F893
:100DD000A55C019016F00AFC97F8A51C50E7204688
:100DE00011F09CFB00287FF46AAF9FED579A04F541
:100DF000FF4973E795F9403404F50047002BBCBF69
:100E0000012387F8A43C79E7DAF8A40FDBF084F833
:100E10000028CED0D5F84C0403681B6898470228F8
:100E20004BD0DAF8A40F4FF00008DBF0B5FB054615
:100E30000028C5D0F5EEC0AAF1EE10FA57D4484606
:100E40000025E0F0D1FFBEE795F94034002BBFF656
:100E500066AF4846C7F8A8BCE0F0BAFF07F6AC4357
:100E600083ED000A5BE7204611F058FB00288FD184
:100E7000DAF8A40FDBF050F80028CBD0DFED357A9C
:100E8000B4EEE7AAF1EE10FA93D9C3E704F50047F0
:100E9000002387F8A43C31E7DAF8A43F09AE002725
:100EA00003F5657393E8070086E8070030460B9763
:100EB00042F0C8FCB0EE40AAFBE6B0EE680A5CF176
:100EC00017FDF0EE407AB0EE480AB0EE678A5CF1AA
:100ED0000FFDDFED217A20EE080AB4EEE70AF1EE0D
:100EE00010FACCBF4FF001084FF0000861E7DFEDCA
:100EF0001B7A4846F4EEE7AAF1EE10FA03DB45460A
:100F0000E0F072FF5FE7E0F06FFFB0EEC00ADFEDE8
:100F1000147A08F00105B4EEE70AF1EE10FA88BF82
:100F2000002550E74846E0F053FF07F6AC43DFEDFD
:100F30000D7A93ED007A30EE470AB4EEE70AF1EE4F
:100F400010FA3FF7F8AEF9E6000000009F0CB34539
:100F5000D30237390000FA4255CF7D3F0000C8C2A6
:100F6000000070420000484238B5044611F00EFB04
:100F7000D0B104F5C04504F51154D5F84C0403680C
:100F80009B6C9847014620B12046BDE8384015F0DB
:100F900073BCD5F84C040368DB6C984701462046C7
:100FA000BDE8384015F068BC204611F0B7FA0028BB
:100FB000DFD1014604F51150BDE8384015F05CBCA6
:100FC000F0B5044685B00D46164604F5115768463F
:100FD0001EF026F96946384615F0FCFF10B90020CE
:100FE00005B0F0BD2946384615F0ACFB0028F6D018
:100FF000002EF5D004F50054304694F8BC3643F08A
:10100000020384F8BC3605B0F0BD00BF30B504461D
:101010008DB004F5115568461EF002F904A81EF0C3
:10102000FFF86946284615F0A7FF08B90DB030BD96
:1010300004A9284615F0CEFF0028F7D0059A2368AA
:101040000192D3F8B030104A934215D108A81EF08F
:10105000E7F808A9284615F0BDFF0028E6D0694644
:10106000284615F06FFB0028E0D045F6CC30012172
:101070002044E6F043FFD9E700226946204698471E
:101080000028D3D0F1E700BFC10F010800F50052DE
:1010900092F8BC26D2070CD400F5C042D2F87024D6
:1010A00092F8D51019B90368D3F8AC301847FFF798
:1010B000ADBF7047F0B5064689B00F4606F511552D
:1010C00068461EF0ADF86946284615F055FF70B128
:1010D00033680446174AD3F8B030934223D104A8AA
:1010E0001EF09EF804A9284615F074FF18B90024D4
:1010F000204609B0F0BD6946284615F023FB0028BC
:10110000F5D03FB106F5005292F8BC3643F0020329
:1011100082F8BC3645F6CC3001213044E6F0EEFED4
:10112000204609B0F0BD3A46694630469847002847
:10113000F0D1DCE7C10F01082DE9F04F2DED0A8B4E
:10114000C1B00B462422044600211CA8029360F182
:1011500045FB2422002125A804F5C04560F13EFB93
:10116000242200212EA860F139FB2422002137A877
:1011700060F134FB0023CDE91133139395F841342A
:1011800013F0080606D00126304641B0BDEC0A8BAC
:10119000BDE8F08F04F5A04243F00803039292F8F3
:1011A000C82F049285F8413420F02CFB90F92530AB
:1011B00043B390F844332BB304F6FC0738461FF0D2
:1011C0009FFF94F822397BB3B146314603E094F88F
:1011D00022398B4228D909F10109384620F048FA12
:1011E0005FFA89F10028F2D180467E4A02210298F6
:1011F00083F0BCFE95F84134012668F3C30385F8FB
:101200004134C1E7784A0298022183F0AFFE0126FB
:1012100095F8413430466FF3C30385F8413441B04B
:10122000BDEC0A8BBDE8F08F46F2F0030121E31814
:1012300018469B46F9F7B8F88046002800F0B981B7
:10124000204610F081FE039BD3F8D43FB3F9088009
:10125000B8F1000F40F0998395F94034002B80F2EB
:10126000898246F29C432046E318099302F046F82F
:10127000424610A9099819F0D7FD002800F07C8299
:101280000A238F21029817AACDF8608008EE102A51
:10129000ADF86480CDE90031F1234D21007C179336
:1012A000032380F08FFD514BDDF8088006211A469C
:1012B0000C930123404653724D4A83F057FE4D4A2A
:1012C0000621404683F052FE02230B9304F580432F
:1012D0004FF00008384683F89E82414620F0D6F849
:1012E00094F82239B3B14FF00009414618EE10AA24
:1012F00008F1010852463846CDF85C90CDF8609070
:10130000CDF864901FF086FD94F822395FFA88F1D9
:101310008B42EDD838461FF0F3FE94F8223933B3F0
:101320004FF000094FF0000AC846494638461FF002
:10133000F5F940AAC0B209F1010908EB480C94F88C
:1013400022E9C0EB401002EB880804EB800302EBBB
:101350008C0C48F8BCAC03F519635FFA89F8ACF162
:10136000900CC64593E807008CE80700DDD841F2F1
:1013700088310EA836F0A6FAD5F8700403689B6A87
:1013800098470121D5F87004E2F096FA1A4B012132
:101390001B68D86A089303681B689847EEF02CF81E
:1013A0000690EEF029F8039B049A93F8C83F079043
:1013B000934240F0D0829FED11AA0023059518EECC
:1013C000105AF0EE4AAA9FED0EBAF0EE4ABA9FED1F
:1013D0000DCADFED0D9A9FED0D9ADFED0D8A0A9390
:1013E0000D9627E034D0170820D0170868D00220C7
:1013F0007CD0170894D0170888CD02200000000088
:101400006F12833A000000340000C842A4707D3F90
:101410000AD7233C089B0521986A03685B689847B4
:101420000FA836F063FA039B049A93F8C83F9342DF
:1014300040F0C68194F8421C384620F019F9002883
:1014400000F0BE81059BD3F8700490F8D560002EA3
:1014500000F09D8241F288310FA836F033FAEDF0AA
:10146000CBFF069BC01A1328D4D9EDF0C5FF069018
:10147000204610F069FD8CF0A7FE80468CF00CFE33
:10148000039BD3F8D43FB3F9082000EE102A059A45
:10149000B8EEC00AD2F8700420EE0B0AE4F018FB94
:1014A00040468CF001FE38461FF02AFEDDF824800D
:1014B000404619F08FFE039BA220B7EE001AD3F826
:1014C000D43FF0EE6B0AB3F9083000EE103AB8EEF4
:1014D000C00A20EE0B0A3BF0E3FCB4EEEA0A00225D
:1014E00010A94046B0EE408AF1EE10FA58BFF0EE77
:1014F00040AA19F099FC002800F0E080DDED107A98
:10150000B4EEE7AA94F82239F1EE10FAB4EECC8AE0
:101510003AFE27AAF1EE10FA4DDA002B3DD04FF03B
:10152000000A04F63C190DF1500853461CAA03EBBF
:101530004303B0EE490A02EB83009E0041F0DEFC5B
:1015400040AB514638461E44CDED150A8DED161AB6
:101550000AF1010A8DED140A1FF0E0F87C23C0B2F5
:10156000B0EE680A03FB0090543041F0C7FC2946F6
:1015700040468DED170ACDED180A8DED191A41F090
:1015800091FC94F822295FFA8AF306ED240A9A4224
:1015900046ED230A06ED221AC8D8EDF02DFF079B71
:1015A000C01AB0F5FA7F00F28E800FA836F09EF9CF
:1015B00039E7AA4A1AE6002B00F0EC814FF0000947
:1015C00004F63C1A0CEE905AC846494638461FF0BD
:1015D000A5F87C235422C0B208EB480809F10109A0
:1015E00013FB002040AB03EB88051CAB504403EB1E
:1015F000880141F06DFC94F822195FFA89F805ED35
:101600001B0A45ED1A0A414505ED191ADDD80B9B59
:101610001CEE905A012B00F02F810029BDD0B0EEB6
:10162000088A4FF000090CEE907ADDF828A005E05A
:1016300009F101095FFA89F399426DD99DED100A0C
:10164000B4EEC80AF1EE10FAF2DB5FFA89F040ABB3
:10165000B24600EB400003EB800825AB870003EBAC
:10166000800041F05BFC37AB08ED120AB0EE490A8E
:10167000D81948ED110A08ED101A41F03FFC2EABC5
:101680008DED140AB0EE680AD819CDED150A8DED6E
:10169000161A41F033FC294614A88DED170ACDED3A
:1016A000180A8DED191A41F013FC94F8221908ED6F
:1016B000090A48ED080A08ED071AB9E7DFED687A6C
:1016C000CDED10BA1CE7EDF097FE039BDDED117A2E
:1016D000F022D3F8D43FB121FCEEE77A029E1B89B9
:1016E0000790ADF86C3017EE903AADF86E301423D9
:1016F000CDE90032379A307C1892389A1992399A8B
:101700001A92109A17922A4680F05CFBBCF012FDE8
:10171000317CBCF0B9F948E71CEE907ACDF828A0EE
:1017200000293FF43AAFCAEE2ACA4FF000084646F5
:1017300037AB06EB460008F1010803EB800042F0EE
:1017400081F858462CEE808AD0F030F807EE900AE7
:1017500040ABB8EE677A03EB860694F82239C8EE00
:10176000077A67EEA97A46ED2F7A5FFA88F6B342D8
:10177000DED812E73B4A39E518900A23ADF8640039
:101780008F2017AA4D21CDE900300298F12308EEF1
:10179000102A17930323007C80F014FB0123DDF84B
:1017A00008800621304A40460B930C9253722F4A10
:1017B00083F0DCFB2E4A0621404683F0D7FB85E50B
:1017C000059D0D9ED5F8700403689B6A984700211B
:1017D000D5F87004E2F070F8089B0021D86A03681D
:1017E0001B6898470A9B002B00F0C5800B99384670
:1017F0001FF04CFE94F8223993B14FF00008414697
:1018000001EB410237AB08F10108384603EB8202D5
:101810001FF000FB94F822395FFA88F18B42EFD871
:1018200038461FF017FB0298124A062183F09EFBF0
:101830000C9B002720465F7201F052FD44F29E206F
:1018400020446BF001FC95F841340EA867F3C30304
:1018500085F8413436F04AF896E400BF20EE1708C8
:101860000000000058D0170868D002207CD017086C
:101870001065170864D0170800296AD04FF0000AD5
:101880000DF150080CEE907A504600EB400040AB52
:10189000B0EE480A0AF1010A03EB800925AB870084
:1018A00003EB800041F03AFB37AB09ED120AB0EED2
:1018B000490AD81949ED110A09ED101A41F01EFB29
:1018C0002EAB8DED140AB0EE680AD819CDED150ACD
:1018D0008DED161A41F012FB404629468DED170A90
:1018E000CDED180A8DED191A41F0F2FA94F822396B
:1018F0005FFA8AF009ED090A984249ED080A09EDF4
:10190000071AC2D31CEE907A1BB34FF00009C846E9
:1019100037AB08EB480009F1010903EB800041F007
:1019200091FF5846B0EE408ACFF040FF07EE900A94
:1019300040ABB8EE677A03EB880894F82239C8EE1A
:10194000077A67EEA97A48ED2F7A5FFA89F843455E
:10195000DED80A9621E6D5F8700403689B6A98479A
:10196000D5F870040021E1F0A7FF089B0021D86A98
:1019700003681B68984702980521094A83F0F6FA24
:10198000384600211FF082FD52E7064A3BE40D9ED7
:101990001D4619E70B9B012B7FF4FFADD9E700BF74
:1019A00054EF1A0844D01708F0B5524D85B0D5F859
:1019B000603FDA0713D400F5C0460446D6F8703409
:1019C00093F8C1205AB993F8D530B3B396F940349F
:1019D000002B32DB00F5004393F8B03C0BB105B0AF
:1019E000F0BD00F5E0479FED440AD7F89C0F6C303E
:1019F00041F084FA60EEA07A9FED407A8DED010A05
:101A0000E0EE007ACDED020A8DED031AF4EEC77A0E
:101A1000F1EE10FA11DCD7F89C3F9FED397AD3ED47
:101A2000377AF4EEC77AF1EE10FA0BD4B5EE007AFD
:101A3000F4EEC77AF1EE10FA0AD5324B00221A8082
:101A400005B0F0BDD6F870341B7A002BEED1F4E768
:101A500004F5FF40E0F0C8F9DFED2B7AB4EEE70AB9
:101A6000F1EE10FAE9D8D7F89C3FB3EE0E7ADFED2D
:101A7000276AD3ED367A67EEA67AF4EEC77AF1EEEE
:101A800010FADADA1F49B4F99C320A88013292B2AC
:101A90000A8023B9B4F89A32A4F89C321BB29BB2E4
:101AA0009A429CD300270F807AF0B2FF01221921BD
:101AB0007AF0D0FCD6F8700403685B699847431C41
:101AC00046F2D810124A394620447EF0F3FED6F88A
:101AD0007034012283F8C120D5F8603F5B077FF5A1
:101AE0007EAF41F66C30204405B0BDE8F040A6F072
:101AF00091BF00BFE88302209F0CB3454054094AC0
:101B00006666663FCECD0220000000B4E02E65423E
:101B10009CD01708514BD3F8603F9B077ED4F0B59B
:101B200000F5E04504462DED028BD5F89C0F85B0FD
:101B300003681B699847DFED4A7A90ED017AB4EEAD
:101B4000E77AF1EE10FA59DB04F5C042D2F87034AE
:101B500093F8C110002955D193F8D530002B51D0FE
:101B600092F94034002B4DDB04F5004797F8B03C68
:101B7000002B47D1D5F89C0F48F6B446036826449D
:101B80001B699847D5F89C3FD0F8B02018460392BF
:101B90001A681369984704F5447200F1B0013046A1
:101BA0007EF006F9DDED037AB0EEC08AF0EEE77A5A
:101BB000F4EEC87AF1EE10FA31D4D5F89C0F036830
:101BC0001B699847DFED267AD0ED040AF4EEE70AA8
:101BD000F1EE10FA12DBF6EE087A60EEA77AF4EE78
:101BE000C87AF1EE10FA1FD5EDF006FCD7F8C02C3C
:101BF00042F210710346821A8A421CD805B0BDEC2D
:101C0000028BF0BD48F6B440002303A9204403939F
:101C10007DF0ACFF05B0BDEC028BF0BD704703A9B1
:101C200030467DF0A3FFC8E79DED030A3AF072FF4E
:101C30000028D9D1E2E79FED0B7A46F2D810C7F819
:101C4000C03C002128EE077A074A2044B7EEC77A45
:101C50008DED007B7EF02EFED0E700BFE8830220F2
:101C6000000000340000C842B8D01708F8B500F5ED
:101C7000004595F92C3103B9F8BD00F5C04795F83A
:101C8000402148F22C16044697F84034064400F5EB
:101C9000FF40DB43C3F3C01363F3C30285F8402165
:101CA000E0F0A2F8DFED457A304620EE670A9BF0BF
:101CB000C9FF95F8B03C002BDED130469BF06AFF9F
:101CC000D7F8703493F8D530002B64D095F84031B4
:101CD000DB07D1D4D7F84C0403689B6B98470028E6
:101CE00059D097F94034002B55DB354F3B88002BFA
:101CF00055D1B5F9323104F5E04543B103EB830327
:101D0000D5F8742F03EB8303B2EB830FB4DB3046BB
:101D10009BF0B4FFD5F89C3FDFED2A6AB3EE0E7A54
:101D2000D3ED367A67EEA67AF4EEC77AF1EE10FAC2
:101D300038D9B4F99C2222B9B4F89A22A4F89C228A
:101D400012B291B23B888B4202D201339BB23B80EC
:101D5000012B2ED01C48D5F84C5F006885421BDA59
:101D600022B9B4F89A12A4F89C1289B28B4283D398
:101D700000233B807AF04CFE0C2102227AF06AFBB1
:101D800030469BF0FFFE48F24C1001212044BDE894
:101D9000F840AEF0E3BE0A4F00233B80F8BD04F5E7
:101DA000E045B4E73B88002B3FF466AF013B3B8046
:101DB000F8BD054BD5F84C2F1A60F8BD0AD7233C67
:101DC000CCCD0220E02E6542C8CD022000F50043B4
:101DD00093F92C2112B300F5C04210B592F94024BA
:101DE0000446002A1BDBB3F9323153B100F5E0425F
:101DF00003EB8303D2F8742F03EB8303B2EB830F5F
:101E00001CDB48F22C1020449BF0BCFE48F24C1026
:101E100001212044BDE81040AEF0A0BE704746F25C
:101E2000D8100E4A062120447EF044FD7AF0F0FDE1
:101E300003220F21BDE810407AF00CBB46F2D81007
:101E4000074A012120447EF035FD7AF0E1FD0222AF
:101E50000F21BDE810407AF0FDBA00BFD0D01708BE
:101E6000E4D0170830B500F5C0452DED028BD5F84C
:101E700070348DB093F8D53073B195F94034002BA0
:101E80000ADB00F58043044693F9BA3223B100F52A
:101E9000004393F8B03C33B1494B00221A800DB097
:101EA000BDEC028B30BD01F0B9FC30B1D5F84C046B
:101EB0000368DB6C98470028EED0D5F84C04036823
:101EC0009B6B98470028E7D047F6507020447DF080
:101ED000A3FE41F0B7FCF0EE087AB0EE408AB4EE13
:101EE000E70AF1EE10FAD7DA04F51155DFED358A7D
:101EF000D5ED937A95ED920A20EE270A5CF128FD44
:101F0000F2EE0E7A20EE280AB4EEE70AF1EE10FAAD
:101F1000C2D904F5E043F3EE0E7AD3F89C3F93ED7B
:101F2000366A66EE288AF4EEE78AF1EE10FAB3D943
:101F30000023284609A909930A930B9315F056F834
:101F400098BB1F49B4F99C220B8801339BB20B80CC
:101F500022B9B4F89A120AB2A4F89C1292B2B3EB66
:101F6000420F9CDB7AF054FD01220C217AF072FAC8
:101F7000B7EEC87AB3EE0E5B134BB7EEE86A0022F9
:101F800046F2D81000212044CDE906238DED047BD4
:101F90000E4A8DED025B8DED006B7EF08BFC012215
:101FA0000C210B48F8F7A4FD79E709A841F04AFC99
:101FB000F2EE047AB4EEE70AF1EE10FAC1DB6BE759
:101FC000C4CD0220E02E654200000840F8D017087A
:101FD000D894022070B500F5C0450446D5F84C04ED
:101FE00003681B68984709282BD01F4BD3F84C0473
:101FF00003681B69984704F5804320B993F9B93207
:10200000032B08D070BD93F9B912022903D195F8BA
:102010006534DB0721D5062120460AF0FBF9D5F807
:102020004C040122114B5A7303681B6C98470346FA
:1020300046F2D8100E4A02212044BDE870407EF0DE
:1020400039BC20460AF0FAF90028CED049F2F43023
:102050002044BDE870400AF0D9B90622204602F0BB
:1020600021FB0028DBD1D6E7E893022068D00220CC
:102070002CD11708F0B500238BB0044600F51150A1
:1020800005AA0793089304F5C046099307AB01928C
:1020900003A9009302AA04AB14F02CFC86F8CC012F
:1020A00018B9002528460BB0F0BD0546EDF09AF9A9
:1020B000D6F8D03107469FED3A7A02A9C31A46F204
:1020C000A81006AA07EE903A2044F8EE677A67EE69
:1020D000877ACDED067A7DF06BFE46F2B41003A947
:1020E00006AA8DED020A20447DF062FE46F2C01081
:1020F00006AA04A9204404F580448DED030A7DF06E
:1021000057FEC6F8D071D4EDAF7AF5EEC07AF1EE95
:1021100010FAC6D9D6F8503143B396F85431DA07DD
:1021200024D5DDED036A9DED077ADDED085A9DEDBE
:10213000096A87FE257A87FE067AF4EEC77AF1EE01
:1021400010FAF4EEE76A94BF01230023F1EE10FACF
:1021500018DBDDED026AF4EEE67AF1EE10FAA1D9B1
:10216000F4EEC77AF1EE10FA9CD99AE737EEA77A27
:10217000DDED036AB4EEE67AF1EE10FAD3D8284624
:102180000BB0F0BD9DED027A03F00105F4EEC77AC5
:10219000F1EE10FA88BF0025002D82D082E700BF43
:1021A000BD37863500F5C04292F8653459071AD517
:1021B00001466FF3820310B50B4C82F86534607BE7
:1021C00038B97AF025FC00221121BDE810407AF0E0
:1021D00041B946F2D8100023044A0844022163732F
:1021E0007EF068FBEDE7704768D0022050D11708F9
:1021F000F0B5044685B004F5115668461DF010F898
:102200006946304614F0E6FE002844D004F58043C9
:10221000D3EDAF7AF5EEC07AF1EE10FA3DD9204653
:10222000FFF728FF0746204610F078F9E0B1404D4F
:1022300087F00102AB78D2B21343AB705BB3DAB173
:102240002A782AB3013A6B78D2B22A700ABB03B358
:1022500000266E707AF0DCFB324610217AF0FAF834
:102260002046FFF79FFF13E0204610F02DF90028CD
:10227000DDD12F4DAB7873B16B7853B92B78013327
:10228000DBB2082B2B7012D0092B41D0092B15D8AB
:102290006B78284AD37305B0F0BD00232449254A42
:1022A00020460B80D373FFF77DFF05B0F0BD002FF4
:1022B000EAD0304614F02AFE2B78E5E74FF4857318
:1022C0002B807AF0A5FB022210217AF0C3F8EDF002
:1022D00093F86A6847F23053801A98421DD804F583
:1022E000C04696F8653443F0040386F865347AF006
:1022F0008FFB012211217AF0ADF8D6F8703493F8F3
:10230000D530002BC4D02046FFF764FE6B78C0E7C1
:10231000304614F0F3FD2B78B8E746F2D810064AA1
:10232000022120447EF0C6FAEDF066F86860D6E738
:10233000D0CD022068D0022068D1170838B500F54A
:10234000C04595F865345A0700D438BD43F00403FE
:10235000044685F865347AF05BFB012211217AF09E
:1023600079F8D5F8703493F8D530002BEDD02046AD
:10237000BDE83840FFF72EBE70B5044682B000F5C8
:10238000115004F5C04601A914F096F8D6F894311E
:1023900083420DD004F5E0430546D3F89C0FD7F0F7
:1023A0005FF8C6F894517AF033FB3E217AF020F8BA
:1023B00004F5005596F9982195F9503795F850177E
:1023C0009A4201D0FF2901D102B070BD04F5E0436B
:1023D000D3F89C0FD7F044F895F8503786F8983129
:1023E0007AF016FB96F8982118217AF033F846F225
:1023F000D81096F998310421024A20447EF05AFA06
:1024000002B070BD78D117082DE9F04104462DEDDA
:10241000028B8EB004F51157ECF0EEFF002204A9F8
:1024200003AB0592064606923846079204F5C0456E
:10243000089209920A920B920C920D9208AA9FEDB3
:10244000568ACDE900310BAB05A914F023FADDED76
:10245000077A95F8CC31F4EEC87AF1EE10FA4DDB3C
:10246000002B4BD0DDED0A8A8046384614F02EFA58
:10247000F4EE488A0746F1EE10FA43DBB8F1000F9C
:1024800040D046F2B41020447DF06EFBF7EE007AA7
:1024900090ED007AB4EEE77AF1EE10FA32DD04F551
:1024A000A04393F9F83E012B3CD095F89C3193B3AF
:1024B000D5F8A40143F69823301A984219D900267A
:1024C00004F5E043C5F8A06185F89C61D3F8A43F0A
:1024D00083F84864C5F8A4617AF09AFA32461D215F
:1024E00079F0B8FF46F2D8102C4A022120447EF041
:1024F000E1F90EB0BDEC028BBDE8F081384614F076
:10250000E5F9074604F5A04393F9F83E002FCCD037
:10251000012BCAD106E0C5F8A0610EB0BDEC028B5C
:10252000BDE8F081D5F8703493F8D530002BBCD0DD
:10253000D5F84C0403685B6998470028B5D195F835
:102540009C2112BBD5F8A031F31AB3F57A7FD0D90C
:10255000012604F5E043C5F8A42185F89C61D3F871
:10256000A43F83F848647AF053FA32461D2179F08B
:1025700071FF46F2D8100A4A022120447EF09AF9EF
:102580000EB0BDEC028BBDE8F081C5F8A4610EB0C1
:10259000BDEC028BBDE8F08100000034ACD117081F
:1025A00090D11708018270472DE9F047054682B0A7
:1025B00044F2B420002305F5C0460DF1070128447C
:1025C0008DF807306CF03AFED6F8700490F9C02010
:1025D000A2F10803DBB2012B00D952BB05F5804301
:1025E0000268B3F8C8129269344B9A4260D10182F2
:1025F00005F11000DFF8D08019F0F8F8304B1C68B6
:10260000E06A0368DB6943451BD10121D6F87004F9
:10261000E1F052F9D6F870040368DB6A98478BF052
:10262000E1F8E06A012103681B6802B0BDE8F047E9
:1026300018470368214A9B6993423BD132230382A6
:10264000D6E746F2D8190027DFF880A0A94416E0A3
:102650001C4B01225A72ECF0CFFE05F500410346F7
:10266000D1F89C2C821A142A1AD8A06A0321036874
:102670005B689847E06A0368DB694345C5D09847C3
:102680000128C2D1ECF0B8FE41F28733C21B9A4256
:10269000DED907465246062148467EF00BF9D7E7B9
:1026A00042F2F030C1F89C3C284464F0E3FDDCE7E2
:1026B00090479DE7322198479AE700BFA52501087A
:1026C00088CD022068D00220599D0008C8D1170883
:1026D0002DE9F84F054642F2F03346F2D810264A6B
:1026E000EB1806212844DFF898A005F50044DFF830
:1026F000949005F5A04805F5C04701262DED028B05
:1027000008EE903A7EF0D6F828469FED1C8AFFF737
:102710004BFF1FE028460FF017FCD9F800300321CB
:10272000986A03685B6898478BF04EFD83468BF090
:10273000B3FCD8F8D42FD7F87004B2F9083000EE03
:10274000103AB8EEC00A20EE080AE3F0C1F9584684
:102750008BF0AAFC8AF80960ECF04EFED4F89C2CB1
:102760000346821A142AD5D918EE900AC4F89C3C64
:1027700064F080FDCEE700BFECD117086F12833AFA
:1027800068D0022088CD02202DE9F84F054646F298
:10279000D8103D4A0621284405F5C04642F2F039DA
:1027A0003A4FDFF8F08041F2873BA9442DED028BD0
:1027B0007EF080F82846FFF7F7FE05F500458BF020
:1027C00003FD04468BF068FCB7EE000AD6F87004EF
:1027D000E3F07EF920468BF067FCECF00DFE8246BC
:1027E00006E0D8F800300321986A03685B689847D0
:1027F000ECF002FE03462046A3EB0A035B451BD820
:102800008BF04AFCB7EE000AD6F87004E3F060F9EA
:1028100020468BF049FC4FF001037B72ECF0ECFD9D
:10282000D5F89C2C0346821A142ADAD94846C5F8F2
:102830009C3C64F01FFDD4E79FED158A4FF0010A20
:1028400006E0D8F800300321986A03685B6898476F
:1028500020468BF021FCB0EE480AD6F87004E3F075
:1028600037F920468BF020FC87F809A0ECF0C4FD76
:10287000D5F89C2C0346821A142AE2D94846C5F89A
:102880009C3C64F0F7FCDCE71CD2170868D00220FF
:102890000000000088CD022000F5C043D3F870345A
:1028A00093F9C030032B5FD0F0B5054683B06424A4
:1028B00000F500463F4F0CE03B681421986A03681E
:1028C0005B68984728460FF03FFB631E13F0FF0438
:1028D00003D0D6F8983C002BEED046F2F000012150
:1028E0002844F7F761FD034648B105F5804393F9A5
:1028F000B432032B5AD8DFE803F0142A535605F5F7
:10290000804292F9B422092A09D042B144F2B4209B
:102910000DF107018DF8073028446CF08FFC03B0EF
:10292000F0BD05F5A04340F2B532D3F8D43FB3F97A
:102930000830934219DC44F2B42000230DF1070162
:1029400028448DF807306CF079FC03B0F0BD05F534
:10295000A04340F2B532D3F8D43FB3F908309342E4
:10296000E9DD2846FFF7B4FE704744F2B4200126A3
:102970000DF1070128448DF807606CF05FFC46F20A
:10298000D8100D4A022128447DF094FF094A0B4BD0
:1029900014685E72A06A052103685B689847F9E7CE
:1029A0002846FFF795FE2846FFF7EEFE092BB6D026
:1029B000C1E700BF88CD022040D2170868D00220AE
:1029C00010B504467AF024F80022052179F042FD82
:1029D00046F2D810034A04212044BDE810407DF09F
:1029E00069BF00BF60D2170838B504460D46ECF049
:1029F00003FD04F5C0443DB9D4F85C34C4F8600468
:102A00000BB9C4F85C0438BDD4F86034C01A64282B
:102A1000F9D90023C4F86034C4F85C3438BD00BF71
:102A200030B5044683B000F5FF40DFF0C3F904F58C
:102A3000C042C0F3803592F84234C3F34001A9424A
:102A40001ED065F3410382F842347DB979F0E0FF8E
:102A50002A460B2179F0FEFC46F2D810094A0221E1
:102A6000204403B0BDE830407DF024BF79F0D0FFB2
:102A700002220B2179F0EEFC46F2D810024AEEE772
:102A800003B030BDCCD21708B0D2170838B50C4609
:102A900015210546224601F005FE28B10C4A13789F
:102AA00043F00803137038BD46F2D8100421094AD8
:102AB00028447DF0FFFE22460621284601F0F2FD63
:102AC0000028EBD121462846BDE8384009F0A2BCD9
:102AD00088D0022004D3170810B500F5C04494F83C
:102AE00042349B0624D4D4F84C0403681B689847EE
:102AF000032813D00CD802280CD0B4F8400420F4DA
:102B0000FE4020F07F0080B2003818BF012010BDC9
:102B10001B2803D094F84004C00910BD94F8400469
:102B200000F0A000A0F18000B0FA80F0400910BDD4
:102B3000012010BD38B5044646F2D8102F4A0221B4
:102B400004F5C045204495F8653443F0080385F842
:102B500065347DF0AFFE79F05BFF0122172179F03B
:102B600079FC95F842349B062AD4D5F84C040368C6
:102B70001B68984703282CD01CD802281CD0B5F815
:102B8000403423F4FE4323F07F039BB2C3B9D5F84E
:102B90004C0403681B689847062821D00B220621A5
:102BA000204601F07FFD10B3154A137843F0080367
:102BB000137038BD1B280CD095F94034002BE6DA91
:102BC00046F2F000012215212044BDE83840F7F715
:102BD0008FBF95F8403403F0A003802BD7D1EFE7E7
:102BE00049F210502044BDE838400BF033B820467D
:102BF0000B21BDE8384009F00DBC00BF50D31708C9
:102C000088D0022038B500F5C04441F28832D4F8AB
:102C10006034D4F85C145B1A934210D894F865348D
:102C200019070BD579F0F4FE0022172179F012FC78
:102C300094F865346FF3C30384F8653438BD0546F2
:102C4000D4F84C0403681B6D984794F8653430B190
:102C50001A07F3D42846BDE83840FFF76BBF1B07BF
:102C6000E0D4EBE738B504461546072914D8DFE869
:102C700001F0190F2C3F04492157152101F012FDD5
:102C800050BB46F2D8102B4A042120447DF012FE9E
:102C90002946204609F0BEFB04F5A043D3F8FC3ECC
:102CA0009B0600D438BD41F66C302044BDE8384066
:102CB000A5F0B0BE1B2101F0F5FC68B946F2D810B2
:102CC00004211D4A20447DF0F5FD2A4606212046B8
:102CD00001F0E8FC0028DBD0184A137843F0080321
:102CE000137004F5A043D3F8FC3E9B06DAD5DAE76F
:102CF0001146FFF7CBFE04F5A043D3F8FC3E9B063C
:102D0000D0D5D0E746F2F000012214212044F7F795
:102D1000EFFE04F5A043D3F8FC3E9B06C2D5C2E704
:102D2000112101F0BFFC0028D6D146F2D810044A88
:102D3000AAE700BFDCD217082CD3170888D00220DE
:102D40003CD3170870B5044682B079F061FE0122C9
:102D5000052179F07FFB04F5804393F89E32072B21
:102D600044D8464A2046D65CFFF7B6FE002843D139
:102D700004F5C045D5F84C040368DB6C984730B1C6
:102D800095F8313A1BB195F9303A012B71DDD5F840
:102D90004C040368DB6C984728B104F5A043D3F8D2
:102DA000FC3E19074DD4D5F84C0403681B689847BE
:102DB000032834D0D5F84C0403685B6A984728B1DF
:102DC00004F5A043D3F8FC3E5B0746D446F2D81086
:102DD0002B4B2C4A042120447DF06CFD032231460C
:102DE000204602B0BDE87040FFF73CBF20460126F8
:102DF000FFF772FE0028BBD0234946F2D810204BC3
:102E0000002620440091214A04217DF053FD46F222
:102E1000F000012210212044F7F76AFEDEE704F5F6
:102E2000A043D3F8FC3EDA07C4D5194946F2D810BE
:102E3000134B002600912044144A04217DF03AFDF2
:102E4000CCE7144946F2D8100D4B009120440F4AAC
:102E5000042101267DF02EFDC0E70F4A46F2D8106E
:102E6000074B042100922044084A00267DF022FDF1
:102E7000B4E7084946F2D810084BE6E748D41708EB
:102E800070D317088CD2170878D3170878D2170890
:102E9000A8D3170894D31708B8D3170884D31708F2
:102EA00030B5044683B0154679F0B2FD0122062103
:102EB00079F0D0FA2046FFF70FFEF8B904F5C043C9
:102EC000EDB2D3F84C040368DB6C984730B104F5DD
:102ED000A043D3F8FC3E1B0700D515BB46F2D81023
:102EE000164B174A042120447DF0E4FC04222946B5
:102EF000204603B0BDE83040FFF7B4BE46F2F00014
:102F00000122072100252044F7F7F2FD0D4946F282
:102F1000D8100A4B009104210B4A20447DF0CAFCD2
:102F2000E4E70A4946F2D810044B012500912044F9
:102F3000054A04217DF0BEFCD8E700BF8CD31708FA
:102F40008CD2170878D3170878D2170894D31708AB
:102F5000F0B5044683B079F05BFD0122082179F0D9
:102F600079FA88F0BFFC04F5804393F88D32072B83
:102F700019D84C4A04F5C045D65CD5F8703493F89E
:102F8000D500C8B9064646F2D810474B0421474A37
:102F900020447DF08FFC05223146204603B0BDE879
:102FA000F040FFF75FBE04F5C0450226D5F8703447
:102FB00093F8D5000028E5D02046FFF78DFD0028C6
:102FC0004CD1D5F84C040368DB6C984730B195F8C8
:102FD000313A1BB195F9303A012B5EDDD5F84C043E
:102FE00004F5A0470368DB6C984778B1D7F8FC3E3E
:102FF00019070BD52E4946F2D8102B4B00912044CF
:103000002C4A042101267DF055FCC4E7D5F84C0478
:1030100003681B6898470328D7F8FC3E10D0DB06EE
:1030200005D5D5F84C040368DB69984748B346F2E8
:10303000D8101D4B1D4A042120447DF03BFCAAE71B
:103040009A07ECD51C4946F2D810174B0026009180
:103050002044184A04217DF02DFC9CE746F2F00044
:103060000122122100262044F7F742FD134946F2BF
:10307000D8100D4B009104210E4A20447DF01AFC1B
:1030800089E70F49064646F2D810074B0091042104
:10309000084A20447DF00EFC7DE7054946F2D81031
:1030A000084BABE750D4170810BD17088CD217088F
:1030B00094D3170878D21708E0D3170878D31708E5
:1030C000F8D31708D0D3170800F5804393F98D3251
:1030D000002B45D070B500F5C0460446D6F8D05355
:1030E00005B970BDECF088F945F65873DFED1D7A2F
:1030F000451B23449FED1C1ADFED1C0A8D2093ED28
:10310000000A20EE270A39F0CBFEBCEEC00A10EE12
:10311000103A9D4216D296F865349A07E1D52046BA
:103120000021F7F767FE46F2D810114A0421204427
:103130007DF0C0FB79F06CFC00220821BDE87040F6
:1031400079F088B9CDD996F865349B07C9D4204663
:103150000121F7F74FFE2046BDE87040FFF7F8BEAB
:10316000704700BF00007A440000804F000000005C
:1031700098D217082DE9F041044682B000F5FF40CF
:1031800004F5C045DEF016FEC0F380480190ECF077
:1031900033F995F8683446460746434569D085F8C3
:1031A00068844EB3C5F86C0446F2D810444B022133
:1031B0002044444A7DF07EFB95F8683463BB04F5F7
:1031C000A04898F96D3F002B95F8653453DDC3F3A3
:1031D0004012B2420DD066F3451385F865349B0664
:1031E00007D5394BD3F84C0403681B69984700286E
:1031F00048D102B0BDE8F08146F2D810304B334AD6
:1032000002212044C5F86C8485F869847DF052FB66
:1032100095F86834002BD2D095F8693404F5A048AD
:10322000002BCED1B8F96E3F40F257109FED280A1F
:1032300007EE903A9FED271ADFED270AF8EEE77ABE
:1032400027EE800A39F02CFEBCEEC00AD5F86C04DB
:1032500010EE103A381A9842B3D9012346F2D8102A
:103260001E4A022185F869342044154B7DF022FB6B
:10327000A7E74346A2E76FF3451385F8653402B02C
:10328000BDE8F08179F0C4FB01221F2179F0E2F85A
:103290002046FFF721FC40B9322298F86D1F2046E6
:1032A00002B0BDE8F041FFF7DDBC46F2F0000122BC
:1032B0002121204402B0BDE8F041F7F719BC00BF5E
:1032C00014D4170824D41708E893022030D4170820
:1032D00000007A440000804F000000003CD4170832
:1032E00008B50122034B1A70ECF07CF8024B186011
:1032F00008BD00BFD9CD0220DCCD0220014B002249
:103300001A707047D9CD02202DE9F0410446ECF047
:1033100069F8314B0546B4F8B6221988914208D0B5
:103320002E492F481A800B780560002B45D1BDE847
:10333000F0812A4E33781BBBDFF8AC8098F8003060
:10334000002BF4D0264F274A3B68C31A9342EED98C
:1033500004F5C043D3F870040123337090F8D530DE
:10336000002B34D179F054FB0122132179F072F84B
:1033700098F80030002BDAD03378002BD7D004E057
:10338000194B1B78002BD2D0154F3B68174AEB1A0C
:103390009342CCD904F5C0443D60D4F8700490F851
:1033A000D530002BC3D00021E0F086FAD4F87004A9
:1033B0000368BDE8F0415B6A184700240C7079F09F
:1033C00027FB22461321BDE8F04179F043B803689A
:1033D0009B6A9847C6E700BFDACD0220D8CD02200D
:1033E000DCCD022080841E00D9CD022040420F0097
:1033F0002DE9F84300F5C04900F540570446D9F8D7
:103400004C0497F8188E0368DB6C9847014648B95E
:1034100099F94034002B43DBD9F8703493F8D50088
:1034200080F0010143F6DC5525442846A6F02AFF2A
:10343000D9F87034064693F8D5307BB358B3484B6F
:1034400093F94034002B51DA97F9E28DB8F1000F6F
:1034500033D099F94034002B5BDBD9F84C04036876
:103460005B69984718B199F94134002B49DB314623
:103470002846A6F091FFDFED3B7AB4EEE70AF1EEC5
:1034800010FA15DCA8F10208B8F1030F60D8DFE8E4
:1034900008F00F580950B8F1000F16D1BDE8F883B5
:1034A0000121BFE70A221121204601F0FBF820B9D3
:1034B0000A220921204601F0F5F879F0A9FA3246EE
:1034C0000921BDE8F84378F0C5BF97F8183E002BF6
:1034D000E4D1234B93F94034002B22DA79F098FAA7
:1034E00000220921BDE8F84378F0B4BF02461E4926
:1034F0002846A6F0DFF997F9E28DB8F1000FDCD08D
:10350000A7E799F86534DA07B1D497F8183EDB07D6
:10351000ADD446F2F00001220F212044F7F7E8FA7B
:10352000CBE746F2D810114A052120447DF0C2F9BC
:10353000D4E70A221521204601F0B4F80028BCD1B6
:10354000B6E70A221521204601F0ACF80028B4D1D4
:103550000A220621204601F0A5F80028ADD1A7E7F0
:10356000E89302200000C84258D4170864D4170812
:1035700070B500F5C04300F5FF4586B0044693F8EA
:103580009C112846DEF0C4FB02A81BF049FE02A9EC
:1035900004F5115013F0F0FC04F5E0432846DDE992
:1035A0000412C3F87C2FC3F8781FDEF003FC8206F8
:1035B00001D406B070BD284647F67075DEF008FCF1
:1035C000FDEEC07A254404F50054022217EE901A4D
:1035D000284617EE906A1BF05BFE94F8BC36DB07BA
:1035E00005D5012128461BF025FF0028E1D1012245
:1035F000314628461BF04CFE06B070BD70B500F594
:10360000004486B00D461646B4F8CC3C8B4203D13C
:10361000D4F8C83C934206D0EBF0EEFED4F8C43C9C
:10362000C31A132B01D806B070BDC4F8C86CA4F837
:10363000CC5CC4F8C40C79F0EBF90446EBF0E4FE82
:1036400002460B460849204604950C680749059434
:10365000CDE90223064A074BCDE90021064A074976
:1036600078F062FD06B070BDE0CD022098D4170856
:10367000B8781708B47817087CD4170890D41708BE
:1036800038B500F5C04494F84134C3F380138B423D
:1036900007D00D4631B994F8413465F3861384F8A8
:1036A000413438BD79F0B4F9112178F0A1FEF2E788
:1036B00070B500F5C04504462DED048BD5F8703487
:1036C0008AB093F8D530EBB195F94034002B19DB73
:1036D000D5F84C0403685B69984720B304F5A04310
:1036E00004F5E044D3F8D43FB3F90830002B15DDDE
:1036F000D4F89C0F0368DB6F0AB0BDEC048BBDE807
:103700007040184704F5E044D4F89C0F03689B6FA1
:103710000AB0BDEC048BBDE870401847D5F84434BE
:10372000022BF1D1E4E704F5E0469FED380AD6F824
:103730009C0F6C303FF0E2FB0AAA0DF1040CCDEDBA
:10374000080A8DED091A04AB8DED070A12E907008E
:1037500083E807008CE8070060463EF0C7FF47F6A5
:103760005070D6F89C3FB0EE408A204493ED369AD4
:103770007CF052FA40F066F8D5F84C04D6F8A42F45
:10378000F0EE408A0368D2EDE49ADB6C9847DFEDF7
:10379000207AB4EEE78AF1EE10FA02DC95F84834AC
:1037A00003B1B0B19FED1B7AF3EE0E7A29EE079AC2
:1037B000B4EEE79AF1EE10FA0BDCF0EE087AF4EED4
:1037C000E78AF1EE10FA04DCF5EEC09AF1EE10FA99
:1037D00016DBD6F89C4F40F2AB10D6F8A42FB7EE0C
:1037E000001A2368DFED0C0A92EDCC0AD3F8805062
:1037F00039F056FB2046A8470AB0BDEC048B70BDDB
:10380000D6F89C0F03689B6F9847F5E79F0CB3456C
:103810000080BB44E02E65420000000000F5C0407F
:1038200090F84804704700BFF8B500F5C04696F818
:103830004034B1EBD31F1ED02C4B002704460D465D
:103840001F60C9B979F0E4F81C2178F0D1FD96F831
:10385000403404F5804465F3C71386F84034BAF069
:1038600027FE0121BAF080FD94F87630002B39D084
:10387000012384F87630F8BD79F0CAF8122178F087
:10388000B7FD96F8403443F0800386F84034BAF030
:103890000FFE3946BAF068FD04F58043B3F8702294
:1038A00083F876705307E6D5D6F8703493F8D530A0
:1038B000002BE0D0D6F84C0403685B6998470028D9
:1038C000D9D1D6F84C04202103689B699847002879
:1038D000D1D046F2F00001220D212044BDE8F8408D
:1038E000F7F706B9EBF088FDA067C1E7E0CD02204D
:1038F0002DE9F04F00F5C04405462DED088BD4F8B6
:1039000070348BB093F8D580B8F1000F00F051817E
:1039100094F94024002AC0F2EC8000F5004797F8A3
:10392000B02C002A40F0528100F5E04B93F807A03C
:10393000DBF89C0F03685B6F98478146D4F84C0412
:1039400003685B69984720B1D4F84434022B00F037
:103950007281BAF1000F40F077815646B7EE00BA97
:10396000B9F1000F40F06D8148F24C199FEDC5AAE6
:10397000A9444846ADF090F90130DBF89C0F0CBF2C
:10398000012302239FEDC00A6C3008EE103A3FF08D
:10399000B5FA0AAA0DF1040CCDED080A04AB8DEDC1
:1039A000091A8DED070A12E9070083E807008CE881
:1039B000070060463EF09AFEDBF89C3F9FEDB37A2D
:1039C00047F6507093ED369AF0EE408ADFEDB07A0C
:1039D000284429EE079AB4EEE70AF3EE0E7AF1EEE8
:1039E00010FAB4EEE79AC8BF46F48076F1EE10FA0A
:1039F000C8BF46F480767CF00FF93FF023FFB8EEA5
:103A0000C88A05F5FF40F0EE409AB4EEC80AF1EE20
:103A100010FA98BF46F08006DEF0E6F928EE0AAA12
:103A20002846F0EEC0AAF4EECAAAF1EE10FA48BF9A
:103A300046F040060EF0A2FB002840F0098146F057
:103A40002006C3464846ADF027F9012800F0F08073
:103A50004846ADF021F9013000F0EA804FF000084F
:103A6000BAF1000F00F0DE80DFED897AF4EEE78A2C
:103A7000F1EE10FA00F3D680F3EE0E7AB4EEE79A88
:103A8000F1EE10FA00F3CE80F4EE489AF1EE10FA5F
:103A900000F2C880F4EE4AAAF1EE10FA40F1C280BA
:103AA000BBF1000F00F0BE80B8F1000F00F0BA804B
:103AB000DFF8EC81B5F99C32D8F8002007EE902AA7
:103AC000B8EE677A23B9B5F89A32A5F89C321BB2E2
:103AD0009BB207EE903AF8EEE77A27EE8BBAB4EE97
:103AE000CB7AF1EE10FA40F1C8800132C8F800201C
:103AF0000CE0D4F84C0403689B6C984706460028F9
:103B00006DD0002605F50047DFF8948194F9403424
:103B1000002B45DBD8F8002007EE902AF8EE676A04
:103B2000B5F99C3223B9B5F89A32A5F89C321BB28C
:103B30009BB29FED587A07EE903A94F84134F8EE34
:103B4000E77A67EE877AF4EEE67AF1EE10FA39D882
:103B50005B0611D478F05CFF112178F049FCD8F8AD
:103B60000020012194F8413461F3861384F8413434
:103B700094F94034002B19DB94F841345B0697F834
:103B8000B03C48BF46F002060BB146F0080631468D
:103B900028460BB0BDEC088BBDE8F04FFFF72EBDFB
:103BA00094F841345806D5D5D8F8002046F00106DF
:103BB000E2E70121464605F50047DFF8E480FFF71C
:103BC00033FEA3E75906D7D50021CBE70022DFF863
:103BD000D080DFED316A1646C8F80020A0E7D4F89F
:103BE0007034284693ED0C8AF7F77AFAB4EEC80AD7
:103BF000F1EE10FA85D5D4F8703493F8A130032B88
:103C00007FF47FAF76F0C4FD42224FF4801105F5BA
:103C1000004776F06FFD31462846DFF88480FFF7D5
:103C200003FE73E7DFF878800023C8F800306DE703
:103C300046F0100614E7B0EE08BABAF1000F19D139
:103C4000564646F480668FE6CA464FF4007685E60F
:103C500045F6F07028447BF087FFDFED107A90ED99
:103C6000007AB4EEE77AF1EE10FA3FF5E8AE4FF0E5
:103C7000000BE7E64FF4C06676E601212846FFF721
:103C8000D3FD43E70000C8429F0CB345E02E6542D8
:103C90000080BB44CDCC4C3E0000000000004843F7
:103CA000E0CD022010B542F29073D0EDA97A88B031
:103CB00047F6507EB0EEE76A0344DFED1D6A0DF172
:103CC000080C04468644B4EEE66ADFED1A5A93E81F
:103CD00007008CE807009DED047AF1EE10FA37EE4C
:103CE000257A8DED047A0BD5B4F99A32F7EE006A95
:103CF00007EE103AB8EEC77AC6EE877AC4EDA97A15
:103D0000704601AA6146CDED017A7CF077F8204635
:103D1000FFF7EEFD2046FDF7A9FF2046FEF7A2F8CB
:103D20002046FDF741FE2046FDF7F4FE08B010BD29
:103D3000000000340AE81C4110B5044682B01D2082
:103D400089F066FD08B902B010BD04F5C043D3F890
:103D50004C0400F0E9FA034641F2A87019210193DE
:103D600020446CF06DFD022819D00338012819D8C1
:103D700045F6F07020447BF0F7FE90ED000ADFED91
:103D80000E7ABDEEC00AB8EEC00A20EE270A48F24D
:103D90004C10204402B0BDE81040ACF081BF9FED54
:103DA000070AF4E7DDED017AB8EEE70ADFED027A03
:103DB00020EE270AEBE700BF0AD7233C00000000F3
:103DC000124A134930B4C0E9001202F1740402F53A
:103DD0007552104DA2F1240142610F4AC0E902451B
:103DE000C0E906120D4C0E4A0E49C0E90842A2F580
:103DF00094620D4CC0E90A120C4A0C3182630C4AE1
:103E0000C0E90C41026130BC704700BF4C76022013
:103E100028F0170890B302202858022084B302200B
:103E200058980220B4930220BC930220F836022056
:103E300094B3022003461C2910D8DFE801F0116B6F
:103E400067635F5B57530F4F0F4B0F0F47433F3B6A
:103E500037332F2B26221E190F0F15000020704715
:103E600049F29C501844704749F654101844704762
:103E700000F5A040D0F8F40E704749F6DC00184475
:103E8000704749F268301844704700F5A040D0F8F8
:103E90009C0C704749F26C701844704749F22870C6
:103EA0001844704749F294601844704749F2D8604A
:103EB0001844704749F254201844704749F27C4036
:103EC0001844704749F294001844704749F214307E
:103ED0001844704749F2D8201844704749F2F4302A
:103EE0001844704749F298201844704749F210501E
:103EF0001844704749F23C401844704749F2B030CA
:103F00001844704748F650501844704748F614500B
:103F10001844704748F6D4401844704770B50B6891
:103F200082B0054608461B6C0C4616469847034669
:103F300046F2D81004210F4A284400967CF0BAFCBF
:103F400078F066FD0346226820461C4613689847B1
:103F50000A210246204678F07DFA074B93F8413457
:103F60009B0604D5054A137843F00403137002B08E
:103F700070BD00BF9CD41708E893022088D00220AF
:103F800038B50D4A182305460C4676F021F960B184
:103F900021462846FFF74EFF044640B10146074A36
:103FA0002846FFF7BBFF002038BD012038BD28465A
:103FB00076F06AF8204638BD34D51708BCD4170807
:103FC00010B50B4B00F5C044002200F5E04084F82A
:103FD000842093F84014D0F89C0FC909D4F06EFCEB
:103FE000D4F84C040368BDE81040DB68184700BFF4
:103FF000E893022070B5064608680C46154603682B
:104000005B69984790B1286803685B69984768B90D
:1040100006F5C043D3F8702492F8D52032B193F955
:104020004034002B02DB3046F7F780F804480EF0EE
:104030008FFF20680368BDE870409B68184700BF89
:10404000D8CE022070B500F5C04504460D4ED5F817
:104050004C040368DB699847D5F84C3430741A680F
:10406000184613689847D5F84C34F0701A6818460B
:10407000536C9847014642F2F0302044BDE870404E
:1040800063F0A4B968D00220264B70B52DED028BE9
:1040900093F8653482B00E461546DB0706D500233B
:1040A00033602B6002B0BDEC028B70BDB0EE408A75
:1040B0000446F0EE608A87F0E5FD037F002BEED02A
:1040C0009FED191A01A99FED190A684668EE811A39
:1040D00028EE011AD4E90A3212681B68B2F90820E6
:1040E000B3F9083000EE902A07EE903AF8EEE00AB5
:1040F000F8EEE77A60EE800A27EE800A3AF0B0F830
:10410000DFED0B6A9DED007ADDED017A27EE267A70
:1041100067EEA67A86ED007AC5ED007A02B0BDECB6
:10412000028B70BDE89302200AD7233C53046939FF
:104130000000C8423B4A002310B52DED028B88B029
:1041400092F8652402930393D3070DD502AB93E84D
:10415000030008AB03E90300DDED070A9DED060A45
:1041600008B0BDEC028B10BDB0EE408A044687F06B
:1041700089FD037F002BE9D0DFED2B6A9FED2B6AD1
:10418000D4E90A3212681B68B2F90820B3F9083082
:1041900007EE902A07EE103AF8EEE77AB8EEC77A03
:1041A00067EEA67A27EE267AF1EE676AF0EEE77AF6
:1041B0008DED037ACDED026AF4EEC67AF1EE10FAD7
:1041C00028D402AC03AA1A482146F6F7EFFFDDED2A
:1041D000027A9DED030A2046F0EEE77AB0EEC00ABF
:1041E000F4EE407AF1EE10FA37FE800A3EF0CCF998
:1041F00004A8CDED050A8DED040A3EF077FA2046BD
:1042000088EE000A3EF0F0F908AB94E8030003E9F9
:104210000300A1E7B0EEC77AB4EEC67AF1EE10FA69
:1042200094D4CEE7E89302205304693900000034A7
:10423000E8330220436A1B6893F8D53043B1054B3D
:1042400093F8400400F0A000203818BF0120704708
:1042500001207047E893022010B50446436AD9B1A3
:1042600002211868DFF03CFB236A9FED0E1A1868E4
:10427000F0EE410A0368B0EE410ADB6A9847226A11
:10428000094B00211068D3ED9B0A03689FED050AD6
:104290005B6EBDE81040184701211868DFF020FB75
:1042A000E2E700BF00000000E873022010B50446FA
:1042B000436A61B302211868DFF012FB236A1868B1
:1042C000D4F0BEFA636A1B6893F8A130012B23D99E
:1042D00063691868D9F018F863691868D9F030F97B
:1042E00063699FED100A1868D7F0D0FF63691868FA
:1042F000D9F0D4FA236A9FED0B1A1868F0EE410A40
:104300000368B0EE410ADB6ABDE81040184701219E
:104310001868DFF0E5FAD1E7236A01211868D5F0C3
:1043200015F9D5E70000000010B582B004460C482E
:1043300001A90DF0ABFF10B1019802B010BD636987
:104340001868D7F0E9FD30B101AA032105481AF039
:10435000C9FF0028F0D1044BD3F8740F02B010BD90
:10436000E833022058B30220E8A30220F0B5044647
:104370002DED048B89B091B100259FED888A63698A
:10438000B0EE480A29461868D7F0B2FF636918688A
:1043900009B0BDEC048BBDE8F040D9F07FBA83686A
:1043A00003F58053B3F9C259FFF7BEFF642DB8BFC0
:1043B0006425A842C0F294806268794EB2F9343024
:1043C00096F84154002BC5F3801540F391805B4271
:1043D00007EE903AB8EEE78AB2F932302046A2688A
:1043E000002B02F58052B8BF5B42B2F9C2799BB292
:1043F0005B4207EE903AF8EEE77AF4EEC87AF1EE17
:1044000010FA38FE278A642FB8BF6427FFF78CFFA5
:10441000A26B3B1AD2ED001A00EE103A63691B68DA
:10442000B8EEC00A93EDC91AD3ED0E0A39F092FA2C
:104430006368F0EE480A40F29720B3F93230002B5F
:10444000B8BF5B429BB25B4201EE103AB8EEC11AB4
:1044500038F026FD6369B0EE408A1868D7F05CFD3D
:1044600096F8423406461A0789D44E48DAF008F91D
:10447000002884D0002E82D0DFED488A01A9494867
:10448000CDED018ACDED028ADAF01CF900286ED15B
:1044900005AF454E3946DFED457A06F63823DFEDA8
:1044A0003F9A06F6142093ED009ACDED059A29EE79
:1044B000279ACDED069ACDED079ADAF049F9F4EE98
:1044C000C98AF1EE10FA18DDB0EEC99ADFED387A3C
:1044D000B4EEE79AF1EE10FA0FD4B0EE698A4EE727
:1044E000626801252E4EB2F93430002B3FF76FAFD2
:1044F00063691B6893EDC78A6EE7DDED077A9FED70
:104500002D7AF4EEC77AF1EE10FA7FF738AF9FED0F
:104510002A7AF4EEC77AF1EE10FA7FF530AFB6F8EA
:10452000503A5B073FF52BAF6368F2EE0E6AB3F9C2
:104530003230002BB8BF5B429BB207EE103ABAEEA6
:10454000EF7AC7EE267A27EEA88AFAEE047AB5EE5D
:10455000C08AF1EE10FA48BF9FED108A38EE478A04
:10456000B4EE678AF1EE10FA37FE888A07E7A06991
:1045700005AFDDF02BFC03AB03C883E8030019464D
:1045800001A83DF0E5FF38468DED050ACDED060AA0
:104590003EF0ACF8F0EE408A7BE700BF0000000080
:1045A000E8930220FCBD0220E8B302200000C842CC
:1045B0000000003400000C4200004843436A0849F0
:1045C0001B681A6812698A4208D1B6EE061A3020B2
:1045D000F4EE000A93ED4B0A38F062BC184610471F
:1045E00049AE000838B52DED028B03680446D3F8B8
:1045F00084309847236B2A48B0EE408A1B68B3F991
:1046000008500DF033FD04464FF47A72002128461D
:10461000002CD8BF4FF4FA7438F0AEFC84422ADD87
:1046200007EE100A07EE904ABAEEEF7AF8EEE77A54
:10463000C7EE278A4FF46D70B6EE000AF5EE087AE1
:10464000B7EE001A38EE400AFEEE000AB1EE400A5C
:1046500080EE270A38F024FCB7EE007A68EE807A04
:1046600037EE407A27EEA80A20EE280AA7EE280A9D
:10467000BDEC028B38BD031BC4F57A74F6EE006AFC
:1046800007EE103A07EE904AB8EEC77AF8EEE77AEE
:1046900027EE267AC7EE278A78EEA68ACAE700BFF9
:1046A000E83302202DE9F04F00F5004800F5C0493D
:1046B00004460E4617462DED028B98F8D05C83B069
:1046C00088F8D02CD9F84C0403681B689847B0428E
:1046D00000F0C780022F00F023811B2E00F02A81FA
:1046E00031462046FFF7A6FB05460190002800F062
:1046F0003F810368D9F870245B6992F8D5B0984778
:1047000049F2D823024601988BF0010A23449842CB
:1047100000F0CB80BBF1000F3BD099F84034DB09AF
:1047200002D0002A40F0CA8003681B69984700281D
:1047300040F011819A480DF03DFF38B9D9F84C048A
:1047400003685B699847002840F0168104F54053E0
:1047500093F8DC2DE2B1B3F8F82DD20718D593F811
:10476000183EABB1D9F8703493F8D53083B104F565
:10477000804393F874300A2B0AD199F94034002B06
:1047800006DB884A204601990025FFF7C7FB62E057
:104790000198036851465B6898470546002800F079
:1047A000B48046F24C4101AA20462144FFF722FC86
:1047B000019804F58043C9F84C0483F874700368C9
:1047C0001B689847014641F658203A46204477F046
:1047D000D7F946F2D8100021204482F03DFAF31EAA
:1047E000062E18BF012B94BF0123002388F8CE3B6F
:1047F00004F5405393F9E23D002B40F0A680D9F830
:104800004C0403681B689847A0F1030004F5A0431B
:1048100004F5E042B0FA80F0012E4FEA501088F81B
:104820002C0003F60470D2F89C1F0068C1F8F80051
:1048300003F63470D2F89C1F0068C1F8FC005CD00D
:104840000B2E5AD02046FFF7FDFB574B93F841340F
:104850009B061ED40125284603B0BDEC028BBDE8A3
:10486000F08F04F580431A2F83F874700AD148B989
:1048700045F6347304F5E0422344D2F89C2F1B68BC
:10488000C2F8FC30484B93F841349906E2D5BD425A
:10489000E0D0464A01251378284643F002031370FE
:1048A00003B0BDEC028BBDE8F08FBBF1000F3FF40D
:1048B00070AF99F94034002BBFF636AF3A4BD3F8BE
:1048C0004C0402685269904705460198002D7FF418
:1048D0002BAFFFF787FE344BB0EE408AA3F5C04004
:1048E000F6F7FEFBB4EEC08AF1EE10FA52DC019846
:1048F000BBF1000F7FF418AF4BE703F61C73D2F83F
:104900009C2F1B68C2F8FC309CE72046284A01997E
:10491000FFF704FB284603B0BDEC028BBDE8F08F27
:1049200031462046FFF72CFB0546002893D01B2E6E
:104930007FF4D6AE48F650503946204403B0BDEC63
:10494000028BBDE8F04F01F00DBB43F6DC50204474
:10495000A5F048FD53E712480DF018FE0546002863
:104960007FF4E8AE134A20460199FFF7D7FA72E7C1
:10497000204675F089FB6EE7019803685B699847EC
:10498000054600287FF4E2AE0B4A20460199FFF766
:10499000C5FA60E7094A20460199FFF7BFFA5AE7CE
:1049A000E833022020D51708E893022088D002209F
:1049B00048F61A08F8D417080CD51708E4D41708D5
:1049C0000148FFF76FBE00BFE83302202DE9F04138
:1049D000DFF8B0810D46044698F86534D9072DED0F
:1049E000028B8EB008D443689A89920700F18B80BD
:1049F00093F95430002B4ED108AF05AE95ED027AF5
:104A0000384695ED005AB1EE477A95ED016AB7EE5A
:104A1000C55AB7EEC66AB7EEC77A9FED520B8DED59
:104A2000085B8DED0A6B8DED0C7B3FF011FA63692D
:104A300039468DED0A1B8DED0C2B8DED080BDFED4E
:104A40004B0A9FED4B0A1868D6F0AAFE63691868F6
:104A5000D8F076FD63691868D8F020FF6269236A90
:104A600010681D68D7F076FF304642498DED020A86
:104A7000CDED030A8DED041AFBF72CFE079C02A96D
:104A8000284696E80C000094D3F0A6FF0EB0BDECCB
:104A9000028BBDE8F0810023226908AF05AE0593C3
:104AA00008931068DCF0E4FE236AB0EE408A1868D0
:104AB00003689B6E98473A46F0EE400A3146B0EEE6
:104AC000480A2046FFF7E0FADDED057A9FED2A7AE5
:104AD000F0EEE77AF4EEC77AF1EE10FA08D5DDEDE4
:104AE000087AF0EEE77AF4EEC77AF1EE10FA85D4A0
:104AF00098F842341B072DD598F8423443F0080348
:104B000088F842347AE71D487BF02EF8DFED1C7AF6
:104B100090ED007AB4EEE77AF1EE10FA06DC636805
:104B200093F95430002B3FF467AFB4E777F070FF90
:104B30003D2177F05DFC09220521A8F5C040FFF773
:104B4000B1FD0028EBD109220221A8F5C040FFF7F2
:104B5000A9FDE4E777F05CFF492177F049FCCBE75A
:104B6000AFF30080000000000000594000007A44CC
:104B70000000000094CD0220000000344CB302205D
:104B800000002F44E8930220F0B5B54D0023044601
:104B90002DED028B95F8412493B0520605930693B0
:104BA00000F1AB8095F86534DB0709D463689A8916
:104BB000970700F1138193F95430002B40F0DA800D
:104BC00095F8433495F842246FF38203110785F872
:104BD000433440F1CB80002095F8433460F38203E6
:104BE0005A0785F8433400F18D800EAE0BAF0023D9
:104BF000626905A90E930F93012310683246D7F01E
:104C000059F863691868D8F09BFC63691868D7F095
:104C1000A1FEA3688DED0B0ACDED0C0A8DED0D1AEA
:104C2000D3ED007AF5EEC07AF1EE10FA11DC236ACA
:104C300030468C491D68FBF74DFD109C39462846CF
:104C400096E80C000094D3F0C7FE13B0BDEC028BC5
:104C5000F0BD854B20469FED858AB3F9603200EEAA
:104C6000903AF8EEE00ACDED030AFFF75DFBA3688A
:104C7000B7EE002A07EE900ADDED030AD3ED001A25
:104C8000B8EEE71A9FED7A0A31EE822A61EE881AB1
:104C900022EE082A37F0CAFF9FED767ADFED767AAA
:104CA00020EE070A20EE270A59F1BEFCDFED737AE9
:104CB000384620EE270A20EE088A3DF017FDB4EEB4
:104CC000C08AF1EE10FAB2D5C8EE006A9DED0B7AFB
:104CD000DDED0C7A636927EE267A67EEA67A8DED14
:104CE0000B7ACDED0C7A1B68D3F8AC23C3F8B8234C
:104CF000D3F8B023C3F8BC2399E743691868D6F00A
:104D000063FF4FE707AE00235D48314607930893E2
:104D100009930A93D9F0D6FC00287FD0A0690BAF85
:104D2000DDF05CF809AA01465548D9F021FD9DED5A
:104D3000086A9DED077A0023B7EEC66A0EAEB7EE9D
:104D4000C77A0B930C9309AA636931468DED106BFA
:104D50008DED0E7B1868012300933B46D6F0E2FFF1
:104D600095F843345B077FF542AF4AE74448D9F0F2
:104D700087FC31E74348F7F741FAE368DFED427A11
:104D80001B6893ED0A0AB4EEE70AF1EE10FA4CDB69
:104D9000F6EE007A20EE270A2046FFF7CBF9B0EEB8
:104DA000C07ADFED397A8DED050AB4EEE77ACDED04
:104DB000060AF1EE10FA06D5F0EEE00AF4EEE70A84
:104DC000F1EE10FA1DD495F84234180742D595F843
:104DD000423443F0080385F84234F1E62B487AF078
:104DE000C3FEDFED237A90ED007AB4EEE77AF1EEC0
:104DF00010FA1DDC636893F95430002B3FF4E0AEE9
:104E0000B8E7234BB3F8503A9E077FF5D9AE95F833
:104E100042346FF3C30385F84234D1E6A069DCF075
:104E2000D5FF03C886E8030078E79FED1A0AB3E7C9
:104E300077F0EEFD3D2177F0DBFA092205211148DC
:104E4000FFF730FC0028D5D1092202210D48FFF7D9
:104E500029FCCFE777F0DCFD492177F0C9FAB6E706
:104E6000E893022094CD0220E87302200000C8429B
:104E700000002F440AD7233C35FA8E3C0AE81C4137
:104E8000FCBD0220E8330220000000344CB30220B5
:104E9000E8B302200000FA4230B585B00023044692
:104EA0001D4801A9019302930393D9F047F9032800
:104EB00012D8DFE800F0020A1C1375F069FC40F21A
:104EC00086324FF4801175F015FC2046FFF75CFE2A
:104ED00000212046FFF74AFA05B030BD0E48D9F050
:104EE0004DF9054648B10128EFD005B030BD01A904
:104EF0002046FFF76BFD05B030BD2046FFF744FEAE
:104F0000636929469FED050A1868D7F0F1F96369CE
:104F10001868D8F0C3FCDFE7F0BE022000000000F4
:104F200038B505460C4619B90B4B93F9142A42B90A
:104F30002846FFF729FE21462846BDE83840FFF7FE
:104F400015BAA3F5005393F842341B07F1D4BDE81A
:104F50003840FFF7A1BF00BFE8B3022010B50446F8
:104F600082B08DED010AAAF01FF9636901A9A26B55
:104F70001B6892ED001A93ED0E0AD3EDC90AA7F053
:104F8000E9FF9DED010A02B010BD00BF436A186839
:104F900003685B6A184700BF10B5436A0446186887
:104FA00090F8D51059B3234B1B7833BB224B93F9A0
:104FB000401493F8402400292EDAB5EEC00AF1EE31
:104FC00010FA05D9D3F8702492F8A120032A14D03E
:104FD000B5EEC00AF1EE10FA03D593F842345B0740
:104FE00023D50221DEF07CFC636A1B6893F8A130B4
:104FF000012B0CBF0220032010BD012010BDDEF0EC
:105000006FFC636A1B6893F8A1000028F4D00128A4
:1050100014BF0320022010BD02F0A002202AD7D125
:105020000221DEF05DFC042010BD0121DEF058FC01
:10503000DAE700BFD8CE0220E8930220164B93F89F
:105040006534DB0702D59FED150A704710B52DEDCD
:10505000028B044686F016FE037FC3B1636B1868AB
:1050600086F01CFFA268DFED0E7A41F6644302F57C
:10507000E351134491ED008AD3ED000A28EE278A0C
:1050800039F0A8F828EE000ABDEC028B10BDBDEC8B
:10509000028B9FED020A10BDE89302200000000081
:1050A0000000C8420148F5F79DBF00BFE833022069
:1050B0000148F7F7A3B800BFE83302200148FFF723
:1050C000F1BA00BFE83302200148FEF7ADBB00BFD4
:1050D000E833022000487047C09502200148F6F7E7
:1050E0007DB800BFE833022030B5174D8BB00023E8
:1050F0000022044604A9D5F8A40FCDE90423CDE984
:105100000623CDE90823D7F03FFC08A9D5F8A40F62
:10511000D7F0A0FC022201A920469DED065B9DED83
:10512000087B9DED046BB7EEC55BB7EEC77BB7EEB2
:10513000C66B8DED025A8DED037A8DED016A1AF082
:1051400079FD20460BB030BDE8A30220014B0122BF
:105150001A707047E4CD022000207047002070478D
:1051600000207047002070470020704700207047E3
:1051700000207047002070470020704700207047D3
:105180009FED010A704700BF00000000002070473B
:1051900000207047002070470020704700207047B3
:1051A00001207047002070470120704701207047A0
:1051B0000020704701207047012070470020704791
:1051C000004870474CD51708004870474CD5170861
:1051D000836803F5805393F8743CDB0706D5002100
:1051E000034B022280F83C10C3F84424012070478E
:1051F000E893022090F83C3053B9836803F580535C
:1052000093F8743CDB0703D5034B0122C3F8442415
:10521000002380F83C307047E8930220012380F897
:105220003C30704720EE007A2DE9F043A0EEA07AE2
:105230001D46002304460F4616462DED0A8B97B0F7
:10524000B0EE408AB7EEC77AB0EE609A0193B0EE46
:1052500041AA0293B5EE407B039304930593F1EECC
:1052600010FA069300F1A381B1EEC76BB7EEC66BDF
:10527000F7EE007AB4EEE76AF1EE10FA05DD87EE9C
:10528000867A28EE078A29EE079AA368B0EE480AC4
:10529000DFEDCABA03F5805303F5436203F63443E6
:1052A000D3ED000A92ED00BA38F094FFA0686BEEDF
:1052B0002B8A00F58050B0EE40BAB0EE490A00F5F6
:1052C000436300F6344028EE8BBAD0ED000AD3EDEC
:1052D00000AA38F07FFFA0686AEEAB8A00F5805024
:1052E000F0EE40AAB0EE4A0A00F6484300F64C4001
:1052F00068EEAAAAD0ED000AD3ED008A38F06AFF62
:10530000636868EEAB8A93F9703068EE808A53B9AF
:1053100087ED00BAC6ED00AAC5ED008A17B0BDEC56
:105320000A8BBDE8F083236A9FEDA50A18686C30EC
:105330003DF0E4FDF0EE609ACDED080A8DED091A1E
:105340008DED070A37F0FAFCBDEEC0CA40F6B83260
:105350009C491CEE100A37F0FFFD4342B0EE690A8B
:1053600007EE903A6368F8EEE77A93ED1A7A67EE03
:10537000877ACDED017A37F0E1FCFDEEC09A40F678
:10538000B832904919EE900A37F0E6FD434207EE35
:10539000903A00230393F8EEE77A636893ED1B7A63
:1053A00093F9703067EE877A022BCDED027A00F028
:1053B0008780236A0DF1480E0DF1380C0DF1280895
:1053C000D3F8009009F184030FCB8EE80F008CE82E
:1053D0000F0088E80F0004AB4146484601AAD4F00C
:1053E00069F8636893F97030022B00F0AD80B0EE7D
:1053F000C88ADFED757AB0EEC99ADFED740AB0EEB7
:10540000CAAAAD20B7EE001AB4EEC89AF1EE10FAAF
:1054100058BFB0EE498AB4EEC8AAF1EE10FA58BFF0
:10542000B0EE4A8A88EE270A31EE400A37F038FD9E
:10543000E36904A8D3ED937A20EE270A3DF05EFDE0
:10544000F0EECB7A8DED061AB520F0EEC06ACDED08
:10545000050AB0EE407A3BEE000A37EEE61A8DED13
:10546000047AB0EEC11AF1EE410A37F019FDDDED14
:10547000057AB0EEEA1ABA20B0EEE77AB0EE40BA9A
:105480003AEEA70A31EE471AB0EEC11AF1EE410A20
:1054900037F006FDDDED067AB0EEE81ABF20B0EE7B
:1054A000E77AF0EE40AA38EEA70A31EE471AB0EEDE
:1054B000C11AF1EE410A37F0F3FCF0EE408A27E71B
:1054C000434BB8EECCCAB3F960320CEE903AF8EE2A
:1054D000ECCAB4EEECCAF1EE10FA42DCB1EE6C0AA2
:1054E000B4EEC0CAF1EE10FA59D4F8EEE99AF4EE2F
:1054F000EC9AF1EE10FA07DCF1EE6CCAF4EEEC9ADD
:10550000F1EE10FA7FF555AFA36B3CEEE90AA26805
:10551000D3ED001A41F630439FED287A1344DFEDB6
:105520002D0AD3ED007A236A67EE877A1B68C7EEEF
:10553000A00A93ED061A38F00DFADDED027A37EE87
:10554000800A8DED020A34E7DDED046A9DED057AEF
:10555000DDED067A3BEE26BA7AEE87AA78EEA78AC8
:10556000D6E6A36B3CEECC0ADFED1A0AD3ED001AA7
:10557000A26841F630431344D3ED007A236A67EE04
:10558000ABBA1B68CBEEA00A93ED051A38F0E2F92E
:10559000DDED017A37EE800A8DED010AA5E7A36BF8
:1055A00030EE4C0ADFED0B0AD3ED001AE0E7B0EE67
:1055B000470B59F1A3F9B0EE406B57E60000C84223
:1055C0009F0CB34548F4FFFF00A08C45000000008D
:1055D000E873022000007A4410B52DED028B836A37
:1055E000044686B0186886F059FCE36AB0EE408A3B
:1055F000186886F053FC636B8DED010A186886F01D
:105600004DFC05ABB0EE401A03A92046B0EE480AA7
:10561000DDED010A04AAFFF705FE636A186890F839
:10562000D51081B1304B93F94124002A06DBD3F821
:105630004434022B06D190F8A1301BB90121DEF0D1
:105640004FF902E00221DEF04BF92046FEF7CAFFD7
:10565000636AB0EE408A1B6893F8A110012938D024
:1056600003292FD011B3A3689DED051A03F58053CC
:10567000DDED040A9DED030A93F8743C13F0020F6C
:10568000236A1868036814BFDB6B9B6B9847226A18
:10569000164BB0EE480A10680021D3ED9B0A036850
:1056A0005B6E984706B0BDEC028B10BD236A0121EA
:1056B0009FED0F8A1868D3F0B1FE236A1868D3F003
:1056C000A9F8D0E7D9790029CDD12046FFF7FCFC15
:1056D000C9E7236A9FED068A1868D3F09FFE236A04
:1056E0001868D3F0ADF8BEE7E8930220E873022013
:1056F00000000000836803F6A82393ED000AB5EECE
:10570000C00AF1EE10FA00DD7047FEF757BF00BF88
:10571000704700BF0020704701207047022070478B
:10572000002070470020704701207047002070471C
:1057300081F00100704700BF0120704701207047D1
:1057400000487047E8D5170800487047F4D5170897
:1057500038B5436904461868D6F01EFFB8B36369CC
:1057600020461D68FFF7BAFC626803462846B2F976
:1057700038105B42B2F9362001EE101A00EE103AF2
:1057800000EE902AB8EEC11AF8EEE00AB8EEC00AB0
:10579000D6F0D0FB636920461D68FFF79FFC626866
:1057A00003462846B2F938105B42B2F9362001EEC2
:1057B000101A00EE103A00EE902AB8EEC11AF8EE78
:1057C000E00AB8EEC00AD6F033FC012038BD6369A8
:1057D0001868D6F039FCC2E730B504462DED028BCF
:1057E000436985B01D68FFF779FC62680346284667
:1057F000674DB2F938105B42B2F9362001EE101A4B
:1058000000EE103A00EE902AB8EEC11AF8EEE00A67
:10581000B8EEC00AD6F08EFB2046FFF749FC236A9B
:10582000B5F96022186808EE102A0368B8EEC88A35
:105830009B6E984702AAF0EE400A01A9B0EE480A12
:105840002046FEF721FC2046FFF7F8FB236BF0EE25
:10585000408A20461B68B3F9083000EE103AB8EED3
:10586000C00AFFF71FFC2046B0EE408A8DED030A08
:10587000FFF734FC43422B2000EE903A6368B0EE11
:10588000480AB3F93630F8EEE00A01EE103AB8EE05
:10589000C11A37F005FB20468DED030AFFF77CFBAC
:1058A000042813D8DFE800F0465603082500236AD1
:1058B00001211868D3F04AFE236A1868D2F0C0FFAD
:1058C00063699FED340A1868D6F0E0FC236AB0EEF5
:1058D000681ADDED020A18689DED010A0368DB6AAB
:1058E000984763691868D7F0D9FF05B0BDEC028B03
:1058F00030BD636A02211868DDF0F2FFB5F960324D
:1059000002AA01A900EE103A2348B8EEC00AA9F095
:10591000BFFB20469DED030AFFF720FB1F488DEDDE
:10592000030A0CF0D1FC63699DED030A1868D6F0F8
:10593000CFFCCBE7236A1868D2F06CFF236A002102
:105940001868D3F003FE63699FED120A1868D6F059
:105950009DFCBBE7124D2B785BB120469DED030A01
:10596000FFF7FCFA03A90E488DED030A0DF012FBB8
:10597000ACE7636845209FED0B1ADFED060A93ED57
:10598000040A37F08DFA28460DF0D0FAE5E700BF9B
:10599000E873022000000000A8B4022060940220F6
:1059A000D8CE022000007A44007900F00100704750
:1059B0000020704790F80D33002B14BF1B200320EC
:1059C000704700BF002070470120704790F8E40244
:1059D0000A2818BF06280CBF01200020704700BF0E
:1059E0000120704701207047044A054B90F80D03D1
:1059F000002814BF10461846704700BF90D61708FD
:105A00009CD61708044A054B90F80D03002814BFD4
:105A100010461846704700BFA4D617089CD6170832
:105A200090F8E4020B3818BF0120704790F80D334E
:105A30002BB9044BD3F8500F00F001007047002041
:105A4000704700BFE8830220024BD3F8500FC0F329
:105A5000C0107047E883022090F8E43223B9034B6A
:105A6000187880F00100704700207047B0CE022007
:105A7000034600220120DB681B6883F8B8287047C2
:105A800070B52DED028BB0F87030002284B0012B80
:105A900094BF0D4641F0010580F80D23002D38D04C
:105AA000436A0446274E1B6893F8D5301BB196F91C
:105AB0004034002B32DB0723234884F8E4320368A8
:105AC000022B3AD09FED218AE368F0EE480AB0EE4F
:105AD000481A1868F0EE481AB0EE480ADBF058F899
:105AE000012304F5227084EDCE8A84F80C3384ED12
:105AF000CF8A84EDD08A3EF0AFFA154806F02EFB2F
:105B000096F8423413486FF3C30386F84234D8F052
:105B100001FA284604B0BDEC028B70BD3C3040F069
:105B2000F1FA03460028C6D120461D46FFF7D2FAF7
:105B3000094A02217AF0BEFEEBE70021FAF744FBA6
:105B4000C0E700BFE893022094CD022000000000CF
:105B500098C70220F0BE0220ACD6170838B50A4D0F
:105B6000044695F8903D012B08D095F8B5100748EC
:105B700089F0ECFC002384F80D3338BD05F68C5019
